:020000040800F2
:1000000000040020E1010008090E00080D0E0008A0
:10001000610E00080D0E0008350E0008E30100080F
:10002000E3010008E3010008E3010008392F00089C
:10003000E3010008E3010008E3010008E301000810
:10004000E3010008E3010008E3010008E301000800
:10005000E3010008E301000899310008C5310008F8
:10006000F13100081D32000849320008E3010008A0
:10007000E3010008E3010008E3010008E3010008D0
:10008000E3010008E3010008E3010008E3010008C0
:10009000E3010008E3010008E301000875320008ED
:1000A000E3010008E3010008E3010008E3010008A0
:1000B000B52F0008E3010008E3010008E301000890
:1000C000E3010008E3010008E3010008E301000880
:1000D000E3010008E3010008E3010008E301000870
:1000E000DD320008E3010008E3010008E301000835
:1000F000E3010008E3010008E3010008E301000850
:10010000E3010008E3010008E3010008E30100083F
:10011000E3010008E3010008E3010008E30100082F
:10012000E3010008E3010008E3010008E30100081F
:10013000E3010008E3010008E3010008E30100080F
:10014000E3010008E3010008E30100088D26000830
:10015000E3010008E3010008E3010008E3010008EF
:10016000E3010008E3010008E3010008E3010008DF
:10017000E3010008E3010008E3010008E3010008CF
:10018000E3010008E3010008E3010008E3010008BF
:10019000E3010008E3010008E3010008E3010008AF
:1001A000E3010008E3010008E3010008E30100089F
:1001B000E3010008E3010008E3010008E30100088F
:1001C000E3010008E3010008E3010008E30100087F
:1001D000E3010008E3010008E3010008E30100086F
:1001E00002E000F000F8FEE772B6394880F30888B4
:1001F000384880F3098838484EF60851CEF200019D
:10020000086040F20000CCF200004EF63471CEF2ED
:1002100000010860BFF34F8FBFF36F8F40F2000003
:10022000C0F2F0004EF68851CEF200010860BFF334
:100230004F8FBFF36F8F4FF00000E1EE100A4EF6C4
:100240003C71CEF200010860062080F31488BFF3F1
:100250006F8F01F0E3FE02F005FE4FF055301F49AD
:100260001B4A91423CBF41F8040BFAE71C49194A6A
:1002700091423CBF41F8040BFAE71A491A4A1B4B5A
:100280009A423EBF51F8040B42F8040BF8E70020F5
:100290001749184A91423CBF41F8040BFAE701F0B4
:1002A000C1FE02F03BFE144C144DAC4203DA54F88C
:1002B000041B8847F9E700F03FF8114C114DAC42A0
:1002C00003DA54F8041B8847F9E701F0A9BE0000DF
:1002D000000400200024002000000008000000208E
:1002E00000040020F036000800240020282400200C
:1002F0002824002018300020E0010008E001000858
:10030000E0010008E00100082DE9F04F2DED108A12
:10031000C1F80CD0C3689D46BDEC108ABDE8F08FD3
:10032000002383F311882846A047002001F0FAFA41
:1003300001F0AAFA00DFFEE71A4B6FF0790270B500
:1003400000241A700F225C709C70DC701C715C7150
:100350009C71DC711C725C729A72DC7201F030FE6E
:10036000064601F055FE054650B90F4B9E4217D088
:1003700001339E4241F2883412BF05460024012514
:10038000002001F027FE0DB100F0B4F800F010FDE0
:1003900000F0F4FB204600F00BF900F0ABF8F9E7B1
:1003A0000446EDE728240020010007B008B500F05E
:1003B00087FBA0F120035842584108BD07B5054B03
:1003C00002211B88ADF8043001A800F0C7FB03B080
:1003D0005DF804FBC0330008064991F8243033B1BE
:1003E00000230822086A81F8243000F0E9BB0120CC
:1003F000704700BF482400202DE9F84F234C94F8A3
:1004000024300546884617468BBB2E46DFF87C9085
:10041000002F38D094F824A0BAF1000F05D1202283
:10042000FF214846266200F0B1FCCAF10805BD4232
:1004300028BF3D465FFA85FBAD0041462A4604EBE6
:100440008A0000F079FC94F82430A7EB0B079B445A
:100450005FFA8BFBBBF1080F2E44A844FFB284F86F
:1004600024B0D5D1FFF7B8FF0028D1D108E0266A23
:1004700006EB8306B042C9D0FFF7AEFF0028C4D117
:100480000020BDE8F88F0120BDE8F88F4824002047
:1004900010B5202383F311881248C3680BB101F013
:1004A000C7FA0023104A0F484FF47A7101F084FA1A
:1004B000002383F311880D4C236813B12368013B9B
:1004C0002360636813B16368013B6360084B1B786A
:1004D00033B9636823B9022000F024FC322363603F
:1004E00010BD00BF342400209104000878250020AE
:1004F0007024002010B5254B254953F8042F0132F4
:1005000000D110BD8B42F8D1224C234B22689A4275
:100510003AD9224B9B6803F1006303F580339A427A
:1005200032D2002000F044FB1D4B0220187000F076
:10053000F1FB1C4B1A6C00221A64196E1A66196EB4
:10054000596C5A64596E5A665A6E5A6942F0800262
:100550005A615A6922F080025A615A691A6942F056
:1005600000521A611A6922F000521A611B6972B6B0
:100570000D4A0E4B13601B682268202181F31188FD
:100580009D4683F30888104710BD00BFFCFF00089C
:100590001C00010804000108FFFF000828240020B7
:1005A000702400200038024008ED00E0000001083F
:1005B0002DE9F04F99B0B34C01902022FF2110A8F3
:1005C000A66800F0E3FBB04A1378A346A3B9AF488E
:1005D0000121C3601170202383F31188C3680BB11C
:1005E00001F026FA0023AA4AA8484FF47A7101F0D4
:1005F000E3F9002383F31188019B13B1A54B019A02
:100600001A60A54AA349019F0292002313704B6010
:1006100099461C461D469846012000F07BFB002FA2
:1006200000F012829B4B1B68002B40F00D8219B02A
:10063000BDE8F08F0220FFF7B9FE002840F0FB81F3
:10064000019BB9F1000F08BF1F46944B1B88ADF802
:100650002C3002210BA800F081FADDE74FF47A700C
:1006600000F02EFA031E0393EADB0220FFF79EFE42
:1006700082460028E4D0039B581E042800F2DD8146
:10068000DFE800F0030E1114170018A8052340F846
:10069000343D042100F062FA54464FF0000856E061
:1006A00004217848F6E704217D48F3E704217D48DA
:1006B000F0E71C24204600F07DFA04340B9004215E
:1006C0000BA800F04BFA2C2CF4D1E5E7002DB7D0A5
:1006D000002CB5D00220FFF769FE0546002800F087
:1006E000AF8101206C4C00F063FA0220207000F012
:1006F00011FB4FF000095FFA89FA504600F068FAE2
:10070000074658B1504600F073FA09F10109002874
:10071000F1D12C46A9460027634B97E7012302201D
:10072000237000F0EDFA3E46DBF808309E4206D218
:10073000304600F03FFA0130EBD10436F4E7029B7B
:1007400000261E70534BA9465E602C46374600F0CB
:1007500025FB15B1002C18BF0027FFF72FFE5BE724
:10076000002D3FF46DAF002C3FF46AAF029B0220D6
:10077000187000F0CFFA322000F0A2F9B0F1000AB0
:10078000C0F25E811AF0030540F05A81DBF80820C0
:1007900006EB0A03934200F25381BAF5807F00F220
:1007A0004F8155450DDA4FF47A7000F089F90490C5
:1007B000049B002BC0F244813C4A049BAB5401359E
:1007C000EFE7C820FFF7F2FD0546002800F038816A
:1007D0001F2E11D8C6F12004544528BF544610AB33
:1007E00026F0030022463149184400F0A5FA2246BB
:1007F000FF212E4800F0CAFA4FEAAA0A5FFA8AF2ED
:100800002A493046FFF7F8FD0446002800F01A8117
:1008100006EB8A0605469AE70220FFF7C7FD002887
:100820003FF40EAFFFF7D8FD00283FF409AF4FF0BB
:10083000000A5346DBF8082092451CD2BAF11F0F7C
:1008400012D8109A01320FD02AF0030218A90A44D4
:1008500052F8202C0B92184604220BA900F014FB2E
:100860000AF1040A0346E5E75046039300F0A2F9B3
:10087000039B0B90EFE718A8042140F84C3D00F0D3
:100880006DF964E72824002074250020342400201A
:10089000910400087825002070240020C23300084D
:1008A0002C24002030240020C433000874240020AD
:1008B00018A8002340F8343D642100F02BF90028EB
:1008C0007FF4BEAE0220FFF771FD00283FF4B8AE02
:1008D0000B9800F09FF918AB43F8480D0421184617
:1008E000CDE718A8002340F8343D642100F012F948
:1008F00000287FF4A5AE0220FFF758FD00283FF442
:100900009FAE0B9800F094F918AB43F8440DE5E75F
:100910000220FFF74BFD00283FF492AE00F08EF965
:1009200018AB43F8400DD9E70220FFF73FFD002840
:100930003FF486AE0BA9142000F086F9824618A871
:10094000042140F83CAD00F009F951460BA896E7A8
:10095000322000F0B5F8B0F1000AFFF671AE1AF0DF
:10096000030F7FF46DAEDBF808200AEB0803934217
:100970003FF666AE0220FFF719FD00283FF460AE97
:100980002AF0030AC244D0453FF4E1AE404600F0ED
:1009900011F904210A900AA800F0E0F808F104080F
:1009A000F1E74FF47A70FFF701FD00283FF448AEFD
:1009B000FFF712FD00283FF4AFAE109B01330CD0BF
:1009C000082210A90020FFF717FD00283FF4A4AE6D
:1009D0002022FF2110A800F0D9F9FFF7EFFC3748DB
:1009E00000F0A6FF23E6002D3FF42AAE002C3FF4D2
:1009F00027AE18A8002340F8343D642100F08AF89F
:100A0000824600287FF41CAE0220FFF7CFFC0028AE
:100A10003FF416AE0390FFF7D1FC41F2883000F0AE
:100A200087FF0B9800F0EEF900F0B8F9039B5746EA
:100A30001C461D46F0E5054689E64FF00008FFE537
:100A40002546FDE52C4667E6002000F039F80490C5
:100A5000049B002BFFF6E3AD012000F051F9049B4D
:100A6000213B122B3FF6D8AD01A252F823F000BF74
:100A7000350600085D060008CD06000819060008C6
:100A80001906000819060008610700085109000846
:100A900019080008B1080008E30800081109000857
:100AA000190600082909000819060008A30900080A
:100AB0004F07000819060008E7090008A086010092
:100AC00037B5114B1A780132D2B20024012A0146FF
:100AD0008DF8074011D80D4803681D6A4FF47A73EA
:100AE0004B4301220DF10701A847012805D1084B0E
:100AF0009DF807001C7003B030BD4FF4FA7000F091
:100B000017FF4FF0FF30F6E70024002048260020B2
:100B10008425002038B50E4B1A780132D2B2012A52
:100B200005460ED80B4803681C6A4FF47A734B4392
:100B300004222946A047042803D1074B002018703F
:100B400038BD4FF4FA7000F0F3FE4FF0FF3038BDBF
:100B500000240020482600208425002030B4054CC5
:100B60002368DD69044B0A46AC460146204630BC8A
:100B7000604700BF48260020A086010070B501F044
:100B800023F9094C094E20700025306823788342F0
:100B900008D901F013F9336805440133B5F5803FF6
:100BA0003360F2D370BD00BF852500208025002072
:100BB00001F0B8B900F1006000F5803000687047BE
:100BC00000F10060920000F5803001F043B90000B0
:100BD000054B1A68054B1B789B1A834202D91044B7
:100BE00001F0ECB80020704780250020852500200A
:100BF00038B5074D04462868204401F0E7F828B9C5
:100C000028682044BDE8384001F0F8B838BD00BF7E
:100C10008025002010F0030308D1B0F5007F05D82F
:100C200000F10050A0F508400068704700207047B0
:100C3000014BC058704700BF107AFF1F014B186866
:100C4000704700BF002004E070B52A4B1C68C4F355
:100C50000B03240C63B140F21342934231D040F2B3
:100C6000194293422FD040F2214293422DD10323C7
:100C7000214A0C2505FB03235D6893F9082042F205
:100C800001039C4224D0B4F5805F23D041F20103DC
:100C90009C4221D041F203039C421FD041F2070342
:100CA0009C4208BF3122441E0C44013D0B46A34226
:100CB0001ED215F9016F581C96B1034600F8016C5D
:100CC000F5E70123D4E70223D2E73F220B4DD6E715
:100CD0003322E3E74122E1E75A22E4E75922E2E73F
:100CE0002C2584421D7001D9981C5A70401A70BD81
:100CF0001846FBE7002004E0D4330008C83300089E
:100D0000022802BF024B4FF400129A61704700BFE5
:100D100000040240022802BF014B20229A61704762
:100D200000040240022801BF024A536983F02003F5
:100D3000536170470004024010B50023934203D072
:100D4000CC5CC4540133F9E710BD000030B5441E3B
:100D500014F9010F0B4660B193F90050854201F17F
:100D6000010106D11AB993F90020801A30BD013A69
:100D7000EEE7002AF7D1104630BD000002460346D8
:100D8000981A13F9011B0029FAD17047024403464F
:100D9000934202D003F8011BFAE77047024B1A781E
:100DA000024B1A70704700BF8425002000240020E9
:100DB00038B5104D104C284600F002F9214628465F
:100DC00000F02AF924680D48626DD2F8043843F027
:100DD0000203C2F8043800F0ABFD0949204600F0D8
:100DE00027FA626DD2F8043823F00203C2F80438FF
:100DF00038BD00BF48260020A034000840420F0044
:100E0000C834000870470000FEE7000000B59BB042
:100E1000EFF3098168226846FFF78EFFEFF3058341
:100E2000034B9A6B9A6A9A6A9A6A9A6A9B6AFEE775
:100E300000ED00E000B59BB0EFF309816822684641
:100E4000FFF77AFFEFF30583044B9A6B9A6A9A6A6D
:100E50009A6A9A6A9A6A9B6AFEE700BF00ED00E010
:100E600000B59BB0EFF3098168226846FFF764FF85
:100E7000EFF30583034B5A6B9A6A9A6A9A6A9A6AE5
:100E80009B6AFEE700ED00E030B5084D0A44914250
:100E90000BD011F8013B09245840013CF7D040F336
:100EA00000032B4083EA5000F7E730BD2083B8ED04
:100EB000002304491A465A50C8180833802B426050
:100EC000F9D170478825002002684368114301600A
:100ED00003B118477047000013B5446BD4F894343D
:100EE0001A681178042915D1217C022912D11979A7
:100EF000128901238B4013420CD101A904F14C004B
:100F000001F02AFED4F89444019B2179024620681E
:100F100000F0DAF902B010BD143001F0ADBD0000F0
:100F20004FF0FF33143001F0A7BD00004C3001F04A
:100F30007FBE00004FF0FF334C3001F079BE00005F
:100F4000143001F07BBD00004FF0FF31143001F090
:100F500075BD00004C3001F04BBE00004FF0FF3279
:100F60004C3001F045BE0000D0F8942438B5136829
:100F700019780429054601D0012038BD017C0229D9
:100F8000FAD112795C89012090400440F4D105F136
:100F9000140001F00DFD02460028EDD0D5F8945460
:100FA0004FF480732868697900F07CF9204638BDD9
:100FB000406BFFF7D9BF000000207047704700006A
:100FC0007FB5124B0360002343608360C36001253B
:100FD00002260F4B057404460290019300F184022F
:100FE000294600964FF48073143001F0BDFC094B84
:100FF0000193029400964FF4807304F523722946FE
:1010000004F14C0001F084FD04B070BD24340008EC
:10101000B10F0008D90E00080B68202282F3118856
:101020000A7903EB820290614A79093243F822007F
:101030008A7912B103EB8203986102230374C0F82A
:101040009414002383F311887047000038B5037FA0
:10105000044613B190F85430ABB9201D012502218C
:10106000FFF732FF04F1140025776FF0010100F063
:1010700087FC84F8545004F14C006FF00101BDE886
:10108000384000F07DBC38BD10B501210446043065
:10109000FFF71AFF0023237784F8543010BD0000B7
:1010A00038B504460025143001F076FC04F14C00FC
:1010B000257701F045FD201D84F854500121FFF7EC
:1010C00003FF2046BDE83840FFF74EBF90F844309C
:1010D00003F06003202B19D190F84520212A0AD073
:1010E000222A4FF000030ED0202A0FD1084A826333
:1010F0000722C26304E0064B83630723C363002314
:101100000364012070478363C363F9E700207047DD
:1011100001240020D0F8943437B51A6811780429D6
:1011200004461AD1017C022917D1197912890123A9
:101130008B40134211D100F14C05284601F0C0FD4F
:1011400058B101A9284601F007FDD4F89444019B49
:1011500021790246206800F0B7F803B030BD0000E6
:1011600000EB8103F7B59C6905460E46F4B12023D8
:1011700083F3118805EB8607201D0821FFF7A4FEE5
:10118000FB685B691B684C3413B1204601F0F2FC2C
:1011900001A9204601F0E0FC024648B1019B31461E
:1011A000284600F091F8002383F3118803B0F0BDC6
:1011B000FB685A691268002AF5D01B8A013B13406C
:1011C000F1D105F14402EAE7093138B550F8214080
:1011D000DCB1202383F31188D4F894241368527966
:1011E00003EB8203DB689B695D6845B104216018ED
:1011F000FFF76AFE294604F1140001F0E3FB2046E4
:10120000FFF7B2FE002383F3118838BD704700005A
:1012100000F08EBF0123037000234360C36183622B
:101220000362C3624362036303814381704700002A
:1012300038B50446202383F3118800254160C5603A
:1012400005614561856100F083FF0223237085F30A
:10125000118838BD70B500EB810305465069DA602E
:101260000E46144618B110220021FFF78FFDA06929
:1012700018B110220021FFF789FD31462846BDE84C
:10128000704001F02FB80000028902F001020281D3
:10129000428902F0010242810022026142618261C0
:1012A00001F0B4B8F0B400EB81044789E46801258B
:1012B000A4698D403D43458123600023A2606360A3
:1012C000F0BC01F0CFB80000F0B400EB8104078956
:1012D000E468012564698D403D4305812360002356
:1012E000A2606360F0BC01F049B9000070B5022350
:1012F000002504460370A0F84C5080F84E5080F84A
:101300004F5005814581C56005614561856180F863
:10131000345000F083FF63681B6823B129462046E0
:10132000BDE87040184770BD436802781B6880F8BC
:101330005020052202700BB10421184770470000AD
:10134000436890F850201B6802700BB105211847C4
:101350007047000090F8343070B5044613B1002394
:1013600080F8343004F14402204601F071F86368DB
:101370009B6863BB94F8445015F0600615D194F84F
:10138000453005F07F0545EA032540F202339D42D2
:1013900000F00E815BD8022D00F0DC803FD8002DDC
:1013A00000F08780012D00F0CF800021204601F061
:1013B000A7FA0021204601F099FA63681B6813B16F
:1013C000062120469847062384F8343070BD204615
:1013D00098470028CED094F84B2094F84A3043EA3E
:1013E0000223E26B934238BFE36394F94430E56B28
:1013F000002B4FF0200380F2FD80002D00F0EC80E8
:10140000092284F8342083F311880021E36BA26B56
:101410002046FFF759FF002383F3118870BDB5F50F
:10142000817F00F0B180B5F5407F49D0B5F5807F70
:10143000BBD194F84630012BB7D1B4F84C3023F02F
:101440000203A4F84C30A663E6632664C3E740F2C7
:1014500001639D421ED8B5F5C06F3BD2B5F5A06FB4
:10146000A3D1B4F84430B3F5A06F0ED194F8463050
:1014700084F84E30204600F029FF63681B6813B1E2
:10148000012120469847032323700023A363E363CD
:101490002364A0E7B5F5106F32D040F602439D42B9
:1014A00052D0B5F5006F80D104F14F03A36301233F
:1014B00024E004F14C03A3630223E36325648AE779
:1014C00094F84630012B7FF470AFB4F84C3043F001
:1014D0000203B6E794F84920616894F848304D68F3
:1014E00094F8471043EA0223204694F84620A84780
:1014F00000283FF45AAF4368A3630368E363A4E79B
:101500002378042B10D1202383F311882046FFF782
:10151000BBFE86F31188636884F84F601B68032163
:1015200021700BB12046984794F84630002BACD080
:1015300084F84F300423237063681B68002BA4D009
:10154000022120469847A0E7374BA3630223E363B9
:1015500000239DE794F8481011F0800F204601F019
:101560000F010ED000F066FF012806D002287FF49C
:101570001CAF2E4BA363E06367E72D4BA363E563CA
:1015800063E700F049FFEFE794F84630002B7FF463
:101590000CAF94F8483013F00F013FF476AF1A0601
:1015A000204602D501F0C0F96FE701F0B3F96CE70E
:1015B00094F84630002B7FF4F8AE94F8483013F0DE
:1015C0000F013FF462AF1B06204602D501F098F9E7
:1015D0005BE701F08BF958E7142284F8342083F399
:1015E00011882B462A4629462046FFF75BFE85F3E5
:1015F000118870BD5DB1152284F8342083F3118801
:101600000021E36BA26B2046FFF74CFE03E70B22A1
:1016100084F8342083F311882B462A462946204635
:10162000FFF752FEE3E700BF543400084C340008D3
:101630005034000838B590F834300446152B29D8BA
:10164000DFE803F03E28282828283E28280B2939DF
:1016500028282828282828283E3E90F84B1090F863
:101660004A20C36B42EA01229A4214D9C268128A04
:10167000B3FBF2F502FB15356DB9202383F3118816
:101680002B462A462946FFF71FFE85F311880A23B9
:1016900084F8343038BD142384F83430202383F3A5
:1016A000118800231A4619462046FFF7FBFD002348
:1016B00083F3118838BD036C03B198470023E7E733
:1016C000002101F01DF90021204601F00FF96368A7
:1016D0001B6813B10621204698470623D8E700006F
:1016E00090F83420152A38B5044622D801239340B7
:1016F00040F6416213421DD113F480150FD19B02B5
:1017000017D50B2380F83430202383F311882B4620
:101710002A462946FFF7D8FD85F3118838BDC368EE
:101720009B695B682BB9036C03B19847002384F86D
:10173000343038BD002101F0E3F80021204601F0EB
:10174000D5F863681B6813B1062120469847062325
:10175000EDE70000024B00221B605B609A6070475F
:1017600008260020002303748268054B1B689968D3
:101770009142FBD25A680360426010605860704723
:101780000826002008B5202383F31188037C032B4F
:1017900005D0042B0DD02BB983F3118808BD436904
:1017A00000221A604FF0FF334361FFF7DBFF002395
:1017B000F2E790E80C001A6002685360F2E700005C
:1017C000002303748268054B1B6899689142FBD81B
:1017D0005A68036042601060586070470826002015
:1017E000054B19690874186802681A60536018611B
:1017F00001230374FEF788BD0826002030B54B1C7A
:1018000087B005460A4C10D023690A4A01A800F0A7
:10181000D3F82846FFF7E4FF049B13B101A800F0BA
:1018200007F92369586907B030BDFFF7D9FFF8E71A
:10183000082600208517000838B50C4D41612B693A
:1018400081689A689142044603D8BDE83840FFF7A2
:1018500089BF1846FFF786FF01232C6101462374D8
:101860002046BDE83840FEF74FBD00BF08260020E7
:10187000044B1A681B6990689B68984294BF0020CB
:10188000012070470826002010B5084C2368206905
:101890001A6822605460012223611A74FFF790FFD6
:1018A00001462069BDE81040FEF72EBD0826002045
:1018B0008260022202740022427470478368A3F19E
:1018C0007C0243F80C2C026943F83C2C426943F833
:1018D000382C074A43F81C2CC26843F8102C02220B
:1018E00003F8082C002203F8072CA3F11800704716
:1018F0002103000810B5202383F31188FFF7DEFFD2
:1019000000210446FFF798FF002383F31188204647
:1019100010BD0000024B1B6958610F20FFF760BF2C
:1019200008260020202383F31188FFF7F3BF00006F
:1019300008B50146202383F311880820FFF75EFFD6
:10194000002383F3118808BD49B1064B42681B6927
:1019500018605A60136043600420FFF74FBF4FF0D8
:10196000FF307047082600200368984206D01A68A6
:101970000260506059611846FFF7F4BE70470000DE
:1019800038B504460D462068844200D138BD03684E
:1019900023605C604561FFF7E5FEF4E7054B03F16A
:1019A00014025A619A614FF0FF32DA6100221A6222
:1019B000704700BF08260020F8B503614FF0804350
:1019C000C2605C6A194B1A46022952F8145F38BF8C
:1019D0000221954206461F460AD1586198611C6251
:1019E0000560456081600819BDE8F84001F08AB9DA
:1019F000186AAB68241A0C1902D3E41A2D6804E0A3
:101A00009C4202D2204401F08BF9AB689C42F4D88E
:101A10006B68736035601E606E60B460A9684FF0DB
:101A2000FF33091BA960FB61F8BD00BF0826002039
:101A300010B41B4C234653F8141F814210D0416848
:101A400002680A60026851609A424FF00001C1606A
:101A500003D0936881680B4493605DF8044B704732
:101A60000A68626100209A425360C86003D15DF841
:101A7000044B01F04FB993688868034493604FF0BA
:101A80008042206A526A121A9342E6D9991A0129B1
:101A900098BF931C18445DF8044B01F041B900BF96
:101AA0000826002000207047FEE700007047000075
:101AB0004FF0FF3070470000022906D0032906D0FE
:101AC0000129064818BF0020704705487047032ABF
:101AD0009ABF044800EBC20000207047243500087C
:101AE000D83400080824002070B59AB001AD06462D
:101AF00008462946144600F095F82846FFF73EF9B7
:101B0000C0B2431C5B0086E8180023700323637097
:101B1000002302341946DAB2904204F1020401D8DB
:101B20001AB070BDEA5C04F8022C04F8011C013301
:101B3000F1E7000008B5202383F311880348FFF77D
:101B4000E9FA002383F3118808BD00BF482600206E
:101B500010B50446052916D8DFE801F0161503165E
:101B6000161D202383F311880E4A0121FFF772FB13
:101B700020460D4A0221FFF76DFB0C48FFF790FA53
:101B8000002383F3118810BD202383F311880748B5
:101B9000FFF75CFAF4E7202383F311880348FFF78B
:101BA00073FAEDE7583400087C340008482600201A
:101BB00038B50C4D0C4C0D492A4604F10800FFF7CE
:101BC00093FF05F1CA0204F110000949FFF78CFFE9
:101BD00005F5CA7204F118000649BDE83840FFF760
:101BE00083BF00BF102B002008240020A834000869
:101BF000B2340008BD34000870B5044608460D46EE
:101C0000FFF7BCF8C6B22046013403780BB918467A
:101C100070BD32462946FFF799F80028F3D101201C
:101C200070BD00002DE9F84F05460C46FFF7A6F8F9
:101C30002C49C6B22846FFF7DFFF08B10436F6B2DA
:101C400029492846FFF7D8FF08B11036F6B2632EAF
:101C50000DD8DFF89090DFF890A0DFF89880DFF8DB
:101C600098B0224F2E7846B92670BDE8F88F2946E5
:101C70002046BDE8F84F01F09BBB252E2DD1072251
:101C800049462846FFF762F850B93B6823607B68F5
:101C900063603B892381BB7AA37207350B34E1E78C
:101CA000082251462846FFF751F8B0B9104BA21C44
:101CB00013F8011F09095B4511F8081002F8021C0E
:101CC000197801F00F0102F1020211F8081002F870
:101CD000031CEDD118340835C4E7267001350134F2
:101CE000C0E700BF44350008BD3400084C3500088B
:101CF0000F7AFF1F583500081B7AFF1FBFF34F8F65
:101D0000024AD368DB03FCD4704700BF003C0240AA
:101D100008B5094B1B7873B9FFF7F0FF074B1A6939
:101D2000002ABFBF064A5A6002F188325A601A6818
:101D300022F480621A6008BD6E2D0020003C024033
:101D40002301674508B50B4B1B7893B9FFF7D6FF06
:101D5000094B1A6942F000421A611A6842F4805233
:101D60001A601A6822F480521A601A6842F480627B
:101D70001A6008BD6E2D0020003C02400B2870B593
:101D800013D80B4A0B4C137863B90B4E4FF000611C
:101D900044F8231056F8235001330C2B2944F7D173
:101DA0000123137054F8200070BD002070BD00BFE7
:101DB000A02D0020702D00206C350008014B53F839
:101DC000200070476C3500080C2070470B2810B5B8
:101DD000044601D9002010BDFFF7D0FF064B53F891
:101DE00024301844C21A0BB9012010BD1268013208
:101DF000F0D1043BF6E700BF6C3500080B2810B5A6
:101E0000044621D8FFF77AFFFFF782FF0F4AF3233A
:101E1000D360C300DBB243F4007343F002031361E9
:101E2000136943F480331361FFF768FFFFF7A6FFE0
:101E3000074B53F8241000F0DDF8FFF783FF20462E
:101E4000BDE81040FFF7C2BF002010BD003C0240BB
:101E50006C3500082DE9F84312F00103154640D116
:101E60008218B2F1016F3CD22C4B1B6813F00103B6
:101E700037D02B4CFFF74CFFF323E360FFF73EFF17
:101E800040F20127032D01D9830713D0244C0F46BC
:101E9000401A40F20118EB1B0B44012B00EB070624
:101EA000236924D823F001032361FFF74BFF0120AE
:101EB000BDE8F883236923F44073236123693B431E
:101EC000236151F8046B0660BFF34F8FFFF716FFD5
:101ED00003689E4208D0236923F001032361FFF7C2
:101EE00031FF0020BDE8F883043D0430CAE723F445
:101EF00040732361236943EA08032361B94637F835
:101F0000023B3380BFF34F8FFFF7F8FE3688B9F8F6
:101F10000030B6B2B342BED0DDE700BF00380240A9
:101F2000003C0240084908B50B7828B153B9FFF7C7
:101F3000EFFE01230B7008BD23B1BDE80840087017
:101F4000FFF700BF08BD00BF6E2D002010B5024492
:101F5000064B0439D2B2904200D110BD441C00B2ED
:101F600053F8200041F8040FE0B2F4E75028004095
:101F7000104B30B51C6F240407D41C6F44F400745C
:101F80001C671C6F44F400441C670B4C236843F42B
:101F9000807323600244094B0439D2B2904200D1CD
:101FA00030BD441C00B251F8045F43F82050E0B249
:101FB000F4E700BF003802400070004050280040A5
:101FC00007B5012201A90020FFF7C0FF019803B067
:101FD0005DF804FB13B50446FFF7F2FFA04206D0FC
:101FE00002A9012241F8044D0020FFF7C1FF02B011
:101FF00010BD000070470000034B1B689B0042BFF0
:10200000024B01221A70704774380240A12D002043
:10201000014B1878704700BFA12D002070470000C9
:10202000FEE70000084A094B09498B4204D3094ADC
:102030000021934205D3704752F8040F43F8040B74
:10204000F3E743F8041BF4E71437000818300020C6
:102050001830002018300020836D30B500229D68B4
:10206000446D11464FF0FF3004EB421301329542AC
:10207000C3F80019C3F81019C3F80809C3F8001B06
:10208000C3F8101BC3F8080BEED24FF00113C4F8CD
:102090001C3830BD890141F02001016103699B06B4
:1020A000FCD4122000F0C4BE204B03EB80022DE9CB
:1020B000F047D2F80CE05D6DDEF81420461CD2F833
:1020C00000C005EB063605EB4018516861450BD39F
:1020D000D5F83428012303FA00F022EA0000C5F8FD
:1020E00034081846BDE8F087BEF81040ACEB010399
:1020F000A34228BF2346D8F81849A4B2B3EB840FF3
:1021000010D894681F46A4F1040959F804AFC6F822
:1021100000A0042F01D9043FF7E71C440B4494604E
:102120005360D2E70020BDE8F08700BFA42D002057
:1021300010B5054C2046FFF76DF84FF0A0436365DE
:10214000024BA36510BD00BFA42D0020C0350008C0
:102150000378012B70B5054650D12A4B446D984247
:102160001BD1294B5A6B42F080025A635A6D42F0E0
:1021700080025A655A6D5A6942F080025A615A6962
:1021800022F080025A610E2143205B6900F0D6FBE9
:102190001E4BE3601E4BC4F800380023C4F8003E19
:1021A000C02323606E6D4FF40413A3633369002BC7
:1021B000FCDA012333610C2000F03AFE3369DB07BF
:1021C000FCD4122000F034FE3369002BFCDA002628
:1021D000A6602846FFF740FF6B68C4F81068DB680C
:1021E000C4F81468C4F81C684BB90A4BA3614FF0DB
:1021F000FF336361A36843F00103A36070BD064B26
:10220000F4E700BFA42D0020003802404014004035
:1022100003002002003C30C0083C30C0F8B5446DDB
:10222000054600212046FFF735FFA96D00234FF03A
:1022300001128F68C4F834384FF00066C4F81C28C7
:102240004FF0FF3004EB431201339F42C2F80069A4
:10225000C2F8006BC2F80809C2F8080BF2D20B688A
:102260006A6DEB65636210231361166916F0100640
:10227000FBD1122000F0DCFDD4F8003823F4FE631B
:10228000C4F80038A36943F4402343F01003A3616A
:102290000923C4F81038C4F814380A4BEB604FF027
:1022A000C043C4F8103B084BC4F8003BC4F81069A5
:1022B000C4F80039EB6D03F1100243F48013EA65B2
:1022C000A362F8BD9C35000840800010426D90F874
:1022D0004E10D2F8003823F4FE6343EA0113C2F82B
:1022E000003870472DE9F0410EB200EB86080D462C
:1022F000D8F80C100F6807F00303022B50D0032B03
:1023000050D03D4A3D4F012B18BF1746446D4FEA50
:10231000451E04EB0E030022C3F8102B8A6905F159
:10232000100C002A40D04A8A05F158035B013A4359
:10233000E2500123D4F81C2803FA0CF31343A644FB
:102340004A69C4F81C380023CEF8103905F13F0360
:10235000002A39D00A8A898B9208012988BF4A430A
:10236000C16D04EB8303561841EA0242C665294653
:102370005A602046FFF78EFED8F80C301B8A43EADD
:1023800085531F4305F148035B01E7500123D4F84F
:102390001C2803FA05F51543C4F81C58BDE8F08164
:1023A000174FB3E7174FB1E704EB4613D3F8002BF1
:1023B00022F40042C3F8002BD4F81C28012303FAAE
:1023C0000CF322EA0303BAE704EB83030E4A5A60D4
:1023D00004EB461629462046FFF75CFED6F8003986
:1023E00023F40043C6F80039D4F81C38012202FA5D
:1023F00005F523EA0505CFE70080001000800410F2
:102400000080081000800C1000040002826D126829
:10241000C265FFF721BE00005831436D49015B588A
:1024200013F4004004D013F4001F14BF0120022055
:10243000704700004831436D49015B5813F4004078
:1024400004D013F4001F14BF0120022070470000C5
:1024500000EB8101CB68196A0B6813604B6853600D
:102460007047000000EB810330B5DD68AA6913688E
:10247000D36019B9402B84BF402313606B8A146862
:10248000426D1C44013CB4FBF3F46343033323F07B
:10249000030302EB411043EAC44343F0C043C0F8D6
:1024A000103B2B6803F00303012B09B20ED1D2F8C5
:1024B000083802EB411013F4807FD0F8003B14BFC2
:1024C00043F0805343F00053C0F8003B02EB41124D
:1024D000D2F8003B43F00443C2F8003B30BD00009B
:1024E0002DE9F041244D6E6D06EB40130446D3F800
:1024F000087BC3F8087B38070AD5D6F814381907C3
:1025000006D505EB84032146DB6828465B689847BF
:10251000FA072FD5D6F81438DB072BD505EB840343
:10252000D968CCB98B69488A5E68B6FBF0F200FBCB
:1025300012628AB91868DA6890420DD2121A83E8DA
:102540001400202383F311880B482146FFF78AFFEC
:1025500084F31188BDE8F081012303FA04F26B894A
:1025600023EA02036B81CB6823B121460248BDE810
:10257000F0411847BDE8F081A42D002000EB810355
:1025800070B5DD68436D6C692668E6604A0156BB2C
:102590001A444FF40020C2F810092A6802F003021E
:1025A000012A0AB20ED1D3F8080803EB421410F442
:1025B000807FD4F8000914BF40F0805040F00050F4
:1025C000C4F8000903EB4212D2F8000940F00440BD
:1025D000C2F80009D3F83408012202FA01F10143DC
:1025E000C3F8341870BD19B9402E84BF4020206054
:1025F00020682E8A841940F00050013C1A44B4FB34
:10260000F6F440EAC440C6E7F8B504461E48456DF6
:1026100005EB4413D3F80869C3F80869F10717D527
:10262000D5F81038DA0713D500EB8403D9684B6965
:102630001F68DA68974218D2D21B00271A605F60C1
:10264000202383F311882146FFF798FF87F3118831
:10265000330617D5D5F834280123A340134211D0EF
:102660002046BDE8F840FFF71FBD012303FA04F23E
:10267000038923EA020303818B68002BE8D02146FB
:102680009847E5E7F8BD00BFA42D002096482DE946
:10269000F84F456D6E69AB691E4016F4805F6E6140
:1026A000044605D0FEF722FEBDE8F84F00F054BC0A
:1026B000002E12DAD5F8003E8B489B071EBFD5F8D6
:1026C000003E23F00303C5F8003ED5F8043823F09C
:1026D0000103C5F80438FEF733FE370502D58248FA
:1026E000FEF722FEB0040CD5D5F8083813F0060F1B
:1026F000EB6823F470530CBF43F4105343F4A0531E
:10270000EB60310704D56368DB680BB17648984706
:10271000F2025AD4B3020CD5D4F85480DFF8C8A121
:1027200000274FF00109A36D9B68F9B28B4280F03E
:102730008780F70619D5616D0A6AC2F30A1702F09D
:102740000F0302F4F012B2F5802F00F0A180B2F571
:10275000402F0AD104EB830301F58051DB68186A2E
:1027600000231A469F4240F087803003D5F818486E
:1027700013D5E10302D50020FFF7B2FEA20302D574
:102780000120FFF7ADFE630302D50220FFF7A8FE8C
:10279000270302D50320FFF7A3FE750384D5E007C6
:1027A00002D50020FFF730FFA10702D50120FFF777
:1027B0002BFF620702D50220FFF726FF23077FF5D4
:1027C00073AF0320FFF720FF6EE7D4F85480DFF8E3
:1027D00018A100274FF00109A36D9B685FFA87FBE2
:1027E0005B4597D308EB4B13D3F8002902F4402242
:1027F000B2F5802F22D1D3F80029002A1EDAD3F8AF
:10280000002942F09042C3F80029D3F80029002A99
:10281000FBDB5946606DFFF73DFC228909FA0BF39B
:1028200022EA0303238104EB8B03DB689B6813B16B
:102830005946504698475846FFF736FC0137CBE7D4
:1028400008EB4112D2F8003B03F44023B3F5802F8C
:1028500010D1D2F8003B002B0CDA628909FA01F39F
:1028600022EA0303638104EB8103DB68DB680BB1BD
:1028700050469847013756E79C0708BF0A68072B60
:1028800098BF027003F101039CBF120A013069E78F
:10289000023304EB830201F58051526890690268AB
:1028A000D0F808C04068A2EB000E00221046974204
:1028B0000AD104EB830463689B699A683A449A607E
:1028C0005A6817445F6050E712F0030F08BF0868AA
:1028D000964588BF8CF8000002F1010284BF000A0F
:1028E0000CF1010CE3E700BFA42D0020436D03EBC6
:1028F0004111D1F8003B43F40013C1F8003B70478D
:10290000436D03EB4111D1F8003943F40013C1F8D2
:1029100000397047436D03EB4111D1F8003B23F4BC
:102920000013C1F8003B7047436D03EB4111D1F830
:10293000003923F40013C1F80039704700F16043F7
:1029400000F01F02400903F5614309018000C9B28C
:1029500000F1604083F8001300F5614001239340CB
:10296000C0F880310360704730B5039C01720433B6
:1029700004FB0325C361049B03630021059B0060E6
:102980004060C160426102618561046242628162AD
:10299000C162436330BD00000022416A41610161B0
:1029A000C2608262C2626FF00101FEF7E9BF0000FF
:1029B00003694269934203D1C2680AB1002070479B
:1029C000181D704703691960C2680132C260C2698C
:1029D000134482690361934224BF436A0361002167
:1029E000FEF7C2BF38B504460D46E3683BB16269E5
:1029F000131D1268A3621344E362002038BD237ADA
:102A000033B929462046FEF79FFF0028EDDA38BD8E
:102A10006FF00100FBE70000C368C269013BC360BF
:102A20004369134482694361934224BF436A43610B
:102A300000238362036B03B11847704770B52023EE
:102A4000044683F31188866A3EB9FFF7CBFF05463B
:102A500018B186F31188284670BDA36AE26A13F89C
:102A6000015BA362934202D32046FFF7D5FF002308
:102A700083F31188EFE700002DE9F84F04460E4676
:102A800090469946202787F311880025AA46D4F856
:102A900028B0BBF1000F09D149462046FFF7A2FF3D
:102AA00020B18BF311882846BDE8F88FA16AE36A4C
:102AB000A8EB050B5B1A9B4528BF9B46BBF1400F5B
:102AC0001BD9334601F1400251F8040B43F8040BC3
:102AD0009142F9D1A36A40334036A3624035A26ADD
:102AE000E36A9A4202D32046FFF796FF8AF31188E1
:102AF0004545D8D287F31188C9E730465A46FEF7D4
:102B00001BF9A36A5B445E44A3625D44E7E70000EF
:102B100010B5029C0172043303FB0421C36100233E
:102B20008362C362039B0363049B00604060C460D4
:102B300042610261816104624262436310BD000030
:102B4000026AC260426A4261026100228262C2621B
:102B50006FF00101FEF714BF436902699A4203D185
:102B6000C2680AB100207047184650F8043B0B6059
:102B700070470000C368C2690133C36043691344EE
:102B800082694361934224BF436A43610021FEF797
:102B9000EBBE000038B504460D46E3683BB123693F
:102BA0001A1DA262E2691344E362002038BD237A51
:102BB00033B929462046FEF7C7FE0028EDDA38BDB6
:102BC0006FF00100FBE7000003691960C268013A79
:102BD000C260C269134482690361934224BF436A9D
:102BE000036100238362036B03B118477047000041
:102BF00070B5202304460E4683F31188856A35B9E3
:102C00001146FFF7C7FF10B185F3118870BDA36AA5
:102C10001E70A36AE26A01339342A36204D3E1699E
:102C200020460439FFF7D0FF002080F3118870BDE3
:102C30002DE9F84F04460D4691469A464FF020087C
:102C400088F311880026B346A76A4FB9514620463B
:102C5000FFF7A0FF20B187F311883046BDE8F88F59
:102C6000A06AE76AA9EB06033F1A9F4228BF1F46E6
:102C7000402F1BD905F1400355F8042B40F8042BD5
:102C80009D42F9D1A36A4033A3624036A26AE36A47
:102C90009A4204D3E16920460439FFF795FF8BF38C
:102CA00011884E45D9D288F31188CDE729463A4696
:102CB000FEF742F8A36A3B443D44A3623E44E5E785
:102CC000026943699A4203D1C3681BB91846704729
:102CD0000023FBE7836A002BF8D0043B9B1AF5D056
:102CE0001360C368013BC360C3691A44836902610E
:102CF0009A4224BF436A0361002383620123E5E70C
:102D000000F06CB94FF08043002258631A61022230
:102D1000DA6070474FF080430022DA6070470000AD
:102D20004FF0804358637047FEE7000010B5174C22
:102D3000FEF710FDFEF732FE802215492046FEF711
:102D4000B7FD012344F8180C0374124B124AD968DA
:102D500021F4E0610904090C0A431049DA60CA68E9
:102D600042F08072CA600E490A6842F001020A60AD
:102D70001022DA77202283F82220002383F311889F
:102D800062B60848BDE81040FEF7B4BD302600200A
:102D9000CC35000800ED00E00003FA05F0ED00E09E
:102DA000001000E0D43500082DE9F84F1F4C4FF01B
:102DB0000008656904F11407C1464FF08043266A94
:102DC0005B6AAA689E1B96421DD34FF0200AAA6830
:102DD000236AD5F80CB0134423622B68BB425F60B2
:102DE000A6EB02066361C5F80C8001D1FFF792FFE4
:102DF00089F311882869D8478AF311886569AB6817
:102E00009E42E4D2D9E76269BA420CD0916823624B
:102E10008E1B9660A86802282CBF1818981CBDE865
:102E2000F84FFFF77DBFBDE8F88F00BF08260020F0
:102E3000034B59685A68521A9042FBD8704700BF3A
:102E4000001000E04B6843608B688360CB68C36010
:102E50000B6943614B6903628B6943620B680360D2
:102E60007047000008B5224B22481A6940F2FF1152
:102E70000A431A611A6922F4FF7222F001021A61F0
:102E80001A691A6B0A431A631A6D0A431A651A4AB9
:102E90001B6D1146FFF7D6FF184802F11C01FFF722
:102EA000D1FF174802F13801FFF7CCFF154802F1B6
:102EB0005401FFF7C7FF144802F17001FFF7C2FF8A
:102EC000124802F18C01FFF7BDFF114802F1A80181
:102ED000FFF7B8FF0F4802F1C401FFF7B3FF0E4838
:102EE00002F1E001FFF7AEFFBDE8084000F0E0B8F6
:102EF0000038024000000240F4350008000402409F
:102F000000080240000C0240001002400014024081
:102F100000180240001C02400020024008B500F0EA
:102F200037FAFFF703FFFFF767F8BDE80840FEF741
:102F30003FBE000070470000064A536823F00103BB
:102F40005360EFF30983683383F30988002383F325
:102F50001188704730EF00E010B5202383F311880B
:102F6000104B5B6813F4006318D0F1EE103AEFF3E6
:102F700009844FF0807344F84C3C0B4BDB6844F8F9
:102F8000083CA4F1680383F30988FEF771FC18B1CB
:102F9000064B44F8503C10BD054BFAE783F311880B
:102FA00010BD00BF00ED00E030EF00E0310300088D
:102FB000340300084FF0804310B51A69920708D512
:102FC00000241C61202383F31188FFF7EDFE84F3B6
:102FD0001188BDE81040FFF7BFBF0000104B1A6C0E
:102FE00042F001021A641A6E42F001021A660D4A9A
:102FF0001B6E936843F0010393604FF080435322AC
:103000009A624FF0FF32DA6200229A615A63DA6004
:103010005A6001225A6108211A601C20FFF78EBCF9
:1030200000380240002004E01F4B1A696FEAC252C8
:103030006FEAD2521A611A69C2F308021A614FF09C
:10304000FF301A695A69586100215A6959615A69F1
:103050001A6A62F080521A621A6A02F080521A6288
:103060001A6A5A6A58625A6A59625A6A1A6C42F063
:1030700080521A641A6E42F080521A661A6E0B4A17
:10308000106840F480701060186F00F44070B0F564
:10309000007F1EBF4FF4803018671967536823F410
:1030A0000073536000F054B90038024000700040D3
:1030B000304B4FF080521A642F4A4FF44041116058
:1030C0001A6842F001021A601A689207FCD59A68E1
:1030D00022F003029A60274B19469A6812F00C02FC
:1030E000FBD1186800F0F90018609A601A6842F481
:1030F00080321A600B689B03FCD54B6F43F00103D1
:103100004B671C4B5A6F9007FCD51C4A5A601A68D3
:1031100042F080721A60184A53685904FCD5154B66
:103120001A689201FCD5164A9A60164B1A68164B1B
:103130009A42164B1BD1164A1168164A914216D173
:1031400040F205121A600B4B9A6842F002029A6034
:103150009A6802F00C02082AFAD15A6C42F48042B2
:103160005A645A6E42F480425A665B6E704740F26F
:103170000572E7E70038024000700040085440073D
:1031800000948838002004E011640020003C0240D4
:1031900000ED00E041C20F41084A08B553691168CB
:1031A0000B4003F00103536123B1054A13680BB1CF
:1031B00050689847BDE80840FFF7CEBE003C01408C
:1031C00088250020084A08B5536911680B4003F0B0
:1031D0000203536123B1054A93680BB1D068984745
:1031E000BDE80840FFF7B8BE003C0140882500203C
:1031F000084A08B5536911680B4003F00403536192
:1032000023B1054A13690BB150699847BDE80840DE
:10321000FFF7A2BE003C014088250020084A08B5FF
:10322000536911680B4003F00803536123B1054A49
:1032300093690BB1D0699847BDE80840FFF78CBE91
:10324000003C014088250020084A08B553691168F0
:103250000B4003F01003536123B1054A136A0BB10D
:10326000506A9847BDE80840FFF776BE003C014031
:1032700088250020174B10B55C691A68144004F4C7
:1032800078725A61A30604D5134A936A0BB1D06AC7
:103290009847600604D5104A136B0BB1506B9847E2
:1032A000210604D50C4A936B0BB1D06B9847E2050D
:1032B00004D5094A136C0BB1506C9847A30504D58B
:1032C000054A936C0BB1D06C9847BDE81040FFF7EE
:1032D00043BE00BF003C0140882500201A4B10B5BA
:1032E0005C691A68144004F47C425A61620504D592
:1032F000164A136D0BB1506D9847230504D5134A38
:10330000936D0BB1D06D9847E00404D50F4A136E4E
:103310000BB1506E9847A10404D50C4A936E0BB1C3
:10332000D06E9847620404D5084A136F0BB1506FF2
:103330009847230404D5054A936F0BB1D06F984783
:10334000BDE81040FFF708BE003C01408825002082
:10335000062108B50846FFF7F1FA06210720FFF716
:10336000EDFA06210820FFF7E9FA06210920FFF708
:10337000E5FA06210A20FFF7E1FA06211720FFF7F8
:10338000DDFA06212820BDE80840FFF7D7BA000083
:1033900008B5FFF749FEFDF78BFDFDF739FFFDF797
:1033A0000DFEFFF7C7FDBDE80840FFF7A9BC000010
:1033B000034611F8012B03F8012B002AF9D17047BD
:1033C000121012131211000053544D3332463F3F76
:1033D0003F00000000000000C83300083F0000006C
:1033E00013040000043400083F000000190400002A
:1033F0000E3400083F0000002104000018340008CB
:103400003F00000053544D3332463430780053545B
:103410004D3332463432780053544D3332463434CF
:103420003658580000000000350F0008210F000832
:103430005D0F0008490F0008550F0008410F0008F4
:103440002D0F0008190F0008B90F00080000000038
:103450000100000000000000020000000000000069
:1034600061110008C911000840004000E02A002056
:10347000F02A00200200000000000000030000000D
:10348000000000000D120008000000001000000005
:10349000002B0020000000000100000000000000E0
:1034A000A42D0020010102004172647550696C6F07
:1034B000740025424F415244252D424C002553456E
:1034C0005249414C25000000511B0008B91A000860
:1034D000CD100008351B000843000000E034000850
:1034E00009024300020100C0320904000001020287
:1034F000010005240010010524010001042402023A
:103500000524060001070582030800FF09040100E5
:10351000020A0000000705010240000007058102C1
:1035200040000000120000002C35000812011001BC
:10353000020000400912415700020102030100008D
:103540000403090425424F41524425007370656508
:10355000647962656566340030313233343536372C
:103560003839414243444546000000000040000015
:10357000004000000040000000400000000001008A
:103580000000020000000200000002000000020033
:103590000000020000000200000002000000000025
:1035A0005513000835160008E116000840004000D9
:1035B000042E0020042E002001000000142E002004
:1035C0008000000040010000030000006D61696E92
:1035D00000000000EC350008202E002018300020EC
:1035E00001000000292D00080000000069646C65DE
:1035F000000000000000800200000000AAAAAAAAA1
:1036000000000000FFFF00000000000000A00A0012
:103610000004500000000000AAAAAAAA000050005E
:10362000DFFF0000000000000000000001000000BB
:1036300000000000AAAAAAAA01000000FFFF0000E3
:10364000000000000000000000000000000000007A
:10365000AAAAAAAA00000000FFFF000000000000C4
:10366000000000000000000000000000AAAAAAAAB2
:1036700000000000FFFF000000000000000000004C
:103680000000000000000000AAAAAAAA0000000092
:10369000FFFF00000000000000000000000000002C
:1036A00000000000AAAAAAAA00000000FFFF000074
:1036B000000000000000000000000000000000000A
:1036C0000A000000000000000300000000000000ED
:1036D00000000000000000000000000000000000EA
:1036E00000000000000000000000000000000000DA
:1036F000FF009600000000080400000040350008AC
:1037000000000000000000000000000000000000B9
:103710000000000000000000FFFFFFFFFFFFFFFFB1
:10372000FFFFFFFFFFFFFFFFFFFFFFFFFFFFFFFFA9
:10373000FFFFFFFFFFFFFFFFFFFFFFFFFFFFFFFF99
:10374000FFFFFFFFFFFFFFFFFFFFFFFFFFFFFFFF89
:10375000FFFFFFFFFFFFFFFFFFFFFFFFFFFFFFFF79
:020000040801F1
:1000000000060020891201080D890808698808087F
:10001000D588080869880808A18808088B12010893
:100020008B1201088B1201088B1201089DA60A0889
:100030008B1201088B1201088B1201088B12010828
:100040008B1201088B1201088B1201088B12010818
:100050008B1201088B120108B9B80A08E1B80A0826
:1000600009B90A0831B90A0859B90A08BD620A086B
:10007000E5620A0811630A083D630A0869630A0811
:1000800091630A08BD630A0841620A088B120108DD
:100090008B1201088B1201088B12010881B90A0822
:1000A000A5BA0A08B9BA0A08CDBA0A08D1BA0A0824
:1000B000D5BA0A088B1201088B12010849690A088F
:1000C000F16A0A088B1201088B1201088B120108D1
:1000D0008B12010855BA0A088B12010869BA0A087E
:1000E000E5B90A088B1201088B120108F9BA0A084F
:1000F000FDBA0A0811BB0A0815BB0A08E9630A0819
:100100008B1201088B120108E9BA0A088B12010848
:100110007DBA0A0891BA0A088B1201088B120108ED
:1001200015640A083D640A0869640A0895640A08A7
:10013000C1640A088B1201088B1201088B12010896
:100140008B1201088B1201088B120108C9AD0A0835
:10015000E9640A0815650A0841650A088B12010856
:100160008B1201088B1201088B1201088B120108F7
:100170008B1201088B1201088B1201088B120108E7
:100180008B1201088B1201088B1201088B120108D7
:100190008B1201088B1201088B1201088B120108C7
:1001A0008B1201088B1201088B1201088B120108B7
:1001B0008B1201088B1201088B1201088B120108A7
:1001C0008B1201088B1201088B1201088B12010897
:1001D0008B1201088B1201088B1201088B12010887
:1001E000654201088D1D0208C9830308912D050889
:1001F00099330508019E0508C1EC050885F405083A
:10020000BDF7050869580608D57706089D0A07084E
:1002100065720708D9810808097C090829DD0908E1
:1002200081030A08010E0A08C13B0A0889410A082D
:1002300081F0004102E000BF83F0004330B54FEA97
:1002400041044FEA430594EA050F08BF90EA020F04
:100250001FBF54EA000C55EA020C7FEA645C7FEA97
:10026000655C00F0E2804FEA5454D4EB5555B8BFBA
:100270006D420CDD2C4480EA020281EA030382EA2B
:10028000000083EA010180EA020281EA0303362DBD
:1002900088BF30BD11F0004F4FEA01314FF4801C90
:1002A0004CEA113102D0404261EB410113F0004FA2
:1002B0004FEA03334CEA133302D0524263EB430359
:1002C00094EA050F00F0A780A4F10104D5F1200EF7
:1002D0000DDB02FA0EFC22FA05F2801841F1000152
:1002E00003FA0EF2801843FA05F359410EE0A5F126
:1002F00020050EF1200E012A03FA0EFC28BF4CF057
:10030000020C43FA05F3C01851EBE37101F000450C
:1003100007D54FF0000EDCF1000C7EEB00006EEB19
:100320000101B1F5801F1BD3B1F5001F0CD34908A3
:100330005FEA30004FEA3C0C04F101044FEA4452FA
:1003400012F5800F80F09A80BCF1004F08BF5FEA81
:10035000500C50F1000041EB045141EA050130BD61
:100360005FEA4C0C404141EB0101013C28BFB1F573
:10037000801FE9D291F0000F04BF01460020B1FABE
:1003800081F308BF2033A3F10B03B3F120020CDA91
:100390000C3208DD02F1140CC2F10C0201FA0CF06F
:1003A00021FA02F10CE002F11402D8BFC2F1200CD4
:1003B00001FA02F120FA0CFCDCBF41EA0C0190408A
:1003C000E41AA2BF01EB0451294330BD6FEA0404D3
:1003D0001F3C1CDA0C340EDC04F11404C4F12002BE
:1003E00020FA04F001FA02F340EA030021FA04F3D0
:1003F00045EA030130BDC4F10C04C4F1200220FA27
:1004000002F001FA04F340EA0300294630BD21FA64
:1004100004F0294630BD94F0000F83F4801306BF2A
:1004200081F480110134013D4EE77FEA645C18BF1E
:100430007FEA655C29D094EA050F08BF90EA020FB5
:1004400005D054EA000C04BF1946104630BD91EAAD
:10045000030F1EBF0021002030BD5FEA545C05D1B0
:100460004000494128BF41F0004130BD14F58004EF
:100470003CBF01F5801130BD01F0004545F0FE4163
:1004800041F470014FF0000030BD7FEA645C1ABF98
:10049000194610467FEA655C1CBF0B46024650EACF
:1004A000013406BF52EA033591EA030F41F40021FB
:1004B00030BD00BF90F0000F04BF0021704730B581
:1004C0004FF4806404F132044FF000054FF0000156
:1004D00050E700BF90F0000F04BF0021704730B517
:1004E0004FF4806404F1320410F0004548BF4042EC
:1004F0004FF000013EE700BF42004FEAE2014FEA41
:1005000031014FEA02701FBF12F07F4393F07F4F1B
:1005100081F06051704732F07F4208BF704793F01E
:100520007F4F04BF41F40021704730B54FF4607431
:1005300001F0004521F000411CE700BF50EA010234
:1005400008BF704730B54FF000050AE050EA0102DD
:1005500008BF704730B511F0004502D5404261EB4D
:1005600041014FF4806404F132045FEA915C3FF48E
:10057000D8AE4FF003025FEADC0C18BF03325FEA2B
:10058000DC0C18BF033202EBDC02C2F1200300FADC
:1005900003FC20FA02F001FA03FE40EA0E0021FA01
:1005A00002F11444BDE600BF70B54FF0FF0C4CF4EF
:1005B000E06C1CEA11541DBF1CEA135594EA0C0FA1
:1005C00095EA0C0F00F0DEF82C4481EA030621EADC
:1005D0004C5123EA4C5350EA013518BF52EA033517
:1005E00041F4801143F4801338D0A0FB02CE4FF0C9
:1005F0000005E1FB02E506F00042E0FB03E54FF0F9
:100600000006E1FB03569CF0000F18BF4EF0010EF0
:10061000A4F1FF04B6F5007F64F5407404D25FEAEC
:100620004E0E6D4146EB060642EAC62141EA55519F
:100630004FEAC52040EA5E504FEACE2EB4F1FD0CE1
:1006400088BFBCF5E06F1ED8BEF1004F08BF5FEA5F
:10065000500E50F1000041EB045170BD06F0004611
:1006600046EA010140EA020081EA0301B4EB5C04BE
:10067000C2BFD4EB0C0541EA045170BD41F48011B6
:100680004FF0000E013C00F3AB8014F1360FDEBFDB
:10069000002001F0004170BDC4F10004203C35DAB7
:1006A0000C341BDC04F11404C4F1200500FA05F33A
:1006B00020FA04F001FA05F240EA020001F00042DB
:1006C00021F0004110EBD37021FA04F642EB060151
:1006D0005EEA430E08BF20EAD37070BDC4F10C047B
:1006E000C4F1200500FA04F320FA05F001FA04F23F
:1006F00040EA020001F0004110EBD37041F100012B
:100700005EEA430E08BF20EAD37070BDC4F1200535
:1007100000FA05F24EEA020E20FA04F301FA05F29D
:1007200043EA020321FA04F001F0004121FA04F245
:1007300020EA020000EBD3705EEA430E08BF20EA15
:10074000D37070BD94F0000F0FD101F0004640004F
:1007500041EB010111F4801F08BF013CF7D041EAD1
:10076000060195F0000F18BF704703F000465200D5
:1007700043EB030313F4801F08BF013DF7D043EAA6
:100780000603704794EA0C0F0CEA135518BF95EA5C
:100790000C0F0CD050EA410618BF52EA4306D1D1E3
:1007A00081EA030101F000414FF0000070BD50EA02
:1007B000410606BF1046194652EA430619D094EA8C
:1007C0000C0F02D150EA013613D195EA0C0F05D176
:1007D00052EA03361CBF104619460AD181EA0301CA
:1007E00001F0004141F0FE4141F470014FF0000082
:1007F00070BD41F0FE4141F4780170BD70B54FF01D
:10080000FF0C4CF4E06C1CEA11541DBF1CEA13559C
:1008100094EA0C0F95EA0C0F00F0A7F8A4EB05047E
:1008200081EA030E52EA03354FEA013100F0888075
:100830004FEA03334FF0805545EA131343EA12633E
:100840004FEA022245EA111545EA10654FEA0026F3
:100850000EF000419D4208BF964244F1FD0404F5AC
:10086000407402D25B084FEA3202B61A65EB030508
:100870005B084FEA32024FF480104FF4002CB6EBC5
:10088000020E75EB030E22BFB61A754640EA0C0045
:100890005B084FEA3202B6EB020E75EB030E22BF85
:1008A000B61A754640EA5C005B084FEA3202B6EBC6
:1008B000020E75EB030E22BFB61A754640EA9C0085
:1008C0005B084FEA3202B6EB020E75EB030E22BF55
:1008D000B61A754640EADC0055EA060E18D04FEA13
:1008E000051545EA16754FEA06164FEAC30343EAB3
:1008F00052734FEAC2025FEA1C1CC0D111F4801F80
:100900000BD141EA00014FF000004FF0004CB6E778
:1009100011F4801F04BF01430020B4F1FD0C88BF17
:10092000BCF5E06F3FF6AFAEB5EB030C04BFB6EB22
:10093000020C5FEA500C50F1000041EB045170BD15
:100940000EF0004E4EEA113114EB5C04C2BFD4EB42
:100950000C0541EA045170BD41F480114FF0000EC6
:10096000013C90E645EA060E8DE60CEA135594EA42
:100970000C0F08BF95EA0C0F3FF43BAF94EA0C0F45
:100980000AD150EA01347FF434AF95EA0C0F7FF4BA
:1009900025AF104619462CE795EA0C0F06D152EA0E
:1009A00003353FF4FDAE1046194622E750EA4106F2
:1009B00018BF52EA43067FF4C5AE50EA41047FF403
:1009C0000DAF52EA43057FF4EBAE12E74FF0FF3C68
:1009D00006E000BF4FF0010C02E000BF4FF0010C39
:1009E0004DF804CD4FEA410C7FEA6C5C4FEA430CB2
:1009F00018BF7FEA6C5C1BD001B050EA410C0CBF01
:100A000052EA430C91EA030F02BF90EA020F002062
:100A1000704710F1000F91EA030F58BF994208BFC9
:100A200090422CBFD8176FEAE37040F00100704786
:100A30004FEA410C7FEA6C5C02D150EA013C07D1DD
:100A40004FEA430C7FEA6C5CD6D152EA033CD3D028
:100A50005DF8040B704700BF8446104662468C4622
:100A60001946634600E000BF01B5FFF7B7FF002855
:100A700048BF10F1000F01BD4DF808EDFFF7F4FF7E
:100A80000CBF012000205DF808FB00BF4DF808ED09
:100A9000FFF7EAFF34BF012000205DF808FB00BF2C
:100AA0004DF808EDFFF7E0FF94BF012000205DF84E
:100AB00008FB00BF4DF808EDFFF7CEFF94BF012003
:100AC00000205DF808FB00BF4DF808EDFFF7C4FFFC
:100AD00034BF012000205DF808FB00BF4FEA410C45
:100AE0007FEA6C5C02D150EA013C0AD14FEA430C28
:100AF0007FEA6C5C02D152EA033C02D14FF0000065
:100B000070474FF0010070474FEA410212F50012A2
:100B100015D211D56FF47873B3EB625212D94FEA44
:100B2000C12343F0004343EA505311F0004F23FA2E
:100B300002F018BF404270474FF00000704750EA83
:100B4000013005D111F0004008BF6FF00040704740
:100B50004FF00000704700BF4A0011D212F500129A
:100B600011D20DD56FF47873B3EB62520ED44FEA05
:100B7000C12343F0004343EA505323FA02F0704785
:100B80004FF00000704750EA013002D14FF0FF30C3
:100B900070474FF0000070474FEA4102B2F1E04366
:100BA00024BFB3F5001CDCF1FE5C0DD901F0004C54
:100BB0004FEAC0024CEA5070B2F1004F40EB8300A4
:100BC00008BF20F00100704711F0804F21D113F1D0
:100BD0003872BCBF01F00040704741F480114FEA09
:100BE0005252C2F11802C2F1200C10FA0CF320FA92
:100BF00002F018BF40F001004FEAC1234FEAD323AF
:100C000003FA0CFC40EA0C0023FA02F34FEA430318
:100C1000CCE77FEA625307D150EA01331EBF4FF0A1
:100C2000FE4040F44000704701F0004040F0FE40BC
:100C300040F40000704700BF80F0004002E000BFB9
:100C400081F0004142001FBF5FEA410392EA030FB7
:100C50007FEA226C7FEA236C6AD04FEA1262D2EB01
:100C60001363C1BFD218414048404140B8BF5B4206
:100C7000192B88BF704710F0004F40F4000020F09F
:100C80007F4018BF404211F0004F41F4000121F0B5
:100C90007F4118BF494292EA030F3FD0A2F10102FF
:100CA00041FA03FC10EB0C00C3F1200301FA03F13D
:100CB00000F0004302D5494260EB4000B0F5000F60
:100CC00013D3B0F1807F06D340084FEA310102F11F
:100CD0000102FE2A51D2B1F1004F40EBC25008BFD1
:100CE00020F0010040EA03007047490040EB00009B
:100CF000013A28BFB0F5000FEDD2B0FA80FCACF19C
:100D0000080CB2EB0C0200FA0CF0AABF00EBC250C8
:100D100052421843BCBFD0401843704792F0000FB6
:100D200081F4000106BF80F400000132013BB5E709
:100D30004FEA41037FEA226C18BF7FEA236C21D07F
:100D400092EA030F04D092F0000F08BF08467047E4
:100D500090EA010F1CBF0020704712F07F4F04D1B2
:100D6000400028BF40F00040704712F100723CBFC5
:100D700000F50000704700F0004343F0FE4040F4EF
:100D8000000070477FEA226216BF08467FEA2363AD
:100D90000146420206BF5FEA412390EA010F40F498
:100DA000800070474FF0000304E000BF10F00043E4
:100DB00048BF40425FEA000C08BF704743F09643CB
:100DC00001464FF000001CE050EA010208BF7047E6
:100DD0004FF000030AE000BF50EA010208BF70476D
:100DE00011F0004302D5404261EB41015FEA010C82
:100DF00002BF84460146002043F0B64308BFA3F17A
:100E00008053A3F50003BCFA8CF2083AA3EBC2535B
:100E100010DB01FA02FC634400FA02FCC2F120027A
:100E2000BCF1004F20FA02F243EB020008BF20F0B1
:100E30000100704702F1200201FA02FCC2F1200217
:100E400050EA4C0021FA02F243EB020008BF20EA0C
:100E5000DC7070477BB972B90029BEBF00204FF02B
:100E6000004106E008BF00281CBF6FF000414FF0B2
:100E7000FF3000F007BAADF1080C6DE904CE00298F
:100E800009DB002B1ADB00F095F8DDF804E0DDE962
:100E9000022304B07047404261EB4101002B1BDB91
:100EA00000F088F8DDF804E0DDE9022304B04042F8
:100EB00061EB4101524263EB43037047524263EBE3
:100EC000430300F077F8DDF804E0DDE9022304B025
:100ED000404261EB41017047524263EB430300F033
:100EE00069F8DDF804E0DDE9022304B0524263EB67
:100EF0004303704753B94AB9002908BF00281CBFF3
:100F00004FF0FF314FF0FF3000F0BCB9ADF1080CED
:100F10006DE904CE00F04EF8DDF804E0DDE90223CF
:100F200004B07047430803F05533C01A830803F038
:100F3000333300F03330184400EB101000F00F3062
:100F400000EB002000EB0040000E704707EE900A17
:100F5000F5EEC07AF1EE10FA01D400F00BB8F1EE24
:100F6000677A08B517EE900A00F004F8404261EB8A
:100F7000410108BDD0B5FFF7BFFA0C4B0022064671
:100F80000F46FFF711FBFFF7E7FD0446FFF792FA64
:100F9000074B0022FFF708FB02460B463046394656
:100FA000FFF74AF9FFF7D8FD2146D0BD0000F03D1C
:100FB0000000F0412DE9F047089D04468E46002BC5
:100FC0004DD18A42944669D9B2FA82F252B101FAFD
:100FD00002F3C2F1200120FA01F10CFA02FC41EA0D
:100FE000030E94404FEA1C48210CBEFBF8F61FFA92
:100FF0008CF708FB16E341EA034306FB07F199422D
:101000000AD91CEB030306F1FF3080F01F819942DF
:1010100040F21C81023E63445B1AA4B2B3FBF8F0B9
:1010200008FB103344EA034400FB07F7A7420AD940
:101030001CEB040400F1FF3380F00A81A74240F268
:1010400007816444023840EA0640E41B00261DB1D3
:10105000D4400023C5E900433146BDE8F0878B4208
:1010600009D9002D00F0EF800026C5E900013046C7
:101070003146BDE8F087B3FA83F6002E4AD18B42A1
:1010800002D3824200F2F980841A61EB030301204B
:101090009E46002DE0D0C5E9004EDDE702B9FFDE37
:1010A000B2FA82F2002A40F09280A1EB0C014FEAE2
:1010B0001C471FFA8CFE0126200CB1FBF7F307FB3F
:1010C000131140EA01410EFB03F0884208D91CEBE2
:1010D000010103F1FF3802D2884200F2CB8043467F
:1010E000091AA4B2B1FBF7F007FB101144EA01445E
:1010F0000EFB00FEA64508D91CEB040400F1FF31ED
:1011000002D2A64500F2BB800846A4EB0E0440EADA
:1011100003409CE7C6F12007B34022FA07FC4CEAE3
:10112000030C20FA07F401FA06F31C43F9404FEAD6
:101130001C4900FA06F3B1FBF9F8200C1FFA8CFEEB
:1011400009FB181140EA014108FB0EF0884202FA3F
:1011500006F20BD91CEB010108F1FF3A80F0888000
:10116000884240F28580A8F102086144091AA4B2BD
:10117000B1FBF9F009FB101144EA014100FB0EFE3E
:101180008E4508D91CEB010100F1FF346CD28E456D
:101190006AD90238614440EA0840A0FB0294A1EBFE
:1011A0000E01A142C846A64656D353D05DB1B3EB5B
:1011B000080261EB0E0101FA07F722FA06F3F1408B
:1011C0001F43C5E9007100263146BDE8F087C2F132
:1011D0002003D8400CFA02FC21FA03F391400143AA
:1011E0004FEA1C471FFA8CFEB3FBF7F007FB1036E3
:1011F0000B0C43EA064300FB0EF69E4204FA02F48F
:1012000008D91CEB030300F1FF382FD29E422DD9E1
:10121000023863449B1B89B2B3FBF7F607FB163316
:1012200041EA034106FB0EF38B4208D91CEB010196
:1012300006F1FF3816D28B4214D9023E6144C91A16
:1012400046EA004638E72E46284605E70646E3E626
:101250001846F8E64B45A9D2B9EB020864EB0C0E30
:101260000138A3E74646EAE7204694E74046D1E73F
:10127000D0467BE7023B614432E7304609E76444ED
:10128000023842E7704700BF02E000F000F8FEE7D6
:1012900072B6374880F30888364880F309883648A4
:1012A0003649086040F20000CCF200004EF634717E
:1012B000CEF200010860BFF34F8FBFF36F8F40F293
:1012C0000000C0F2F0004EF68851CEF20001086036
:1012D000BFF34F8FBFF36F8F4FF00000E1EE100AA6
:1012E0004EF63C71CEF200010860062080F31488AF
:1012F000BFF36F8F99F030FA9AF07AF94FF05530CA
:101300001F491B4A91423CBF41F8040BFAE71D49B3
:10131000184A91423CBF41F8040BFAE71A491B4AAC
:101320001B4B9A423EBF51F8040B42F8040BF8E7FE
:1013300000201849184A91423CBF41F8040BFAE7D3
:1013400099F00EFA9AF0A8F9144C154DAC4203DA54
:1013500054F8041B8847F9E702F074FF114C124D52
:10136000AC4203DA54F8041B8847F9E799F0F6B960
:1013700000060020002200200000010808ED00E027
:10138000000000200006002028F70C0800220020A2
:101390004C2600205026002050470120E001010883
:1013A0003002010830020108300201082DE9F04F37
:1013B0002DED108AC1F80CD0C3689D46BDEC108A93
:1013C000BDE8F08F002383F311882846A047002052
:1013D00098F046F9FEE797F0A3FF00DFFEE7000074
:1013E00001F0FF01102A2BDB10F0070F08D010F8D6
:1013F000013B013A8B422DD010F0070F42B3F6D1DA
:10140000F0B441EA012141EA014122F007047FF0F2
:1014100000070023F0E80256083C85EA010586EA49
:10142000010685FA47F5A3FA87F586FA47F6A5FA85
:1014300087F68EB9EED1F0BC01F0FF0102F0070291
:1014400032B110F8013B013A83EA010313B1F8D13C
:101450000020704701387047002D06BF354603381D
:10146000073815F0010F07D1013015F4807F02BF56
:10147000013015F4C03F0130F0BC0138704700BFA7
:1014800010F8012B11F8013B012A28BF9A42F7D02E
:10149000D01A7047034613F8012B002AFBD1181A03
:1014A0000138704738B50022002304460D46FFF787
:1014B000EDFA28B920462946BDE8384000F00AB8C0
:1014C000204605F1004100F005F8404261EB410182
:1014D00038BD00BFD0B50C4B002206460F46FFF7C3
:1014E00063F8FFF739FB0446FEF7E4FF074B0022E1
:1014F000FFF75AF802460B4630463946FEF79CFE87
:10150000FFF72AFB2146D0BD0000F03D0000F0416E
:10151000036800221B68184770B50D4B1C68E56A0C
:101520002B681E686FF036FD014630B1E06A036833
:10153000DB699847411E18BF01212846B0474AF091
:10154000BFFAE36ABDE8704093F89C1049F0F2BB23
:101550005826002013B50191202104466FF026FD86
:1015600090B10A4BDFED0A7A93EDB27A019AB4EEAC
:10157000E77AF1EE10FA05DA2046064B20216FF0EB
:101580001DFD002002B010BD0120FBE760560020C9
:1015900000000034B42A0B0837B5094B0191054609
:1015A000D3F8F80503689B6998470199044618B970
:1015B000044A28466FF0E4FE204603B030BD00BF69
:1015C00060760020C82A0B0830B585B00446039128
:1015D00040216FF0EBFC90B31A49039AD1F8B03D6B
:1015E000D1F8B41DB3F90A5040F21450854214DC0E
:1015F000B3F90E5040F2A3639D421ADDB1F90A50CF
:10160000854214DCB1F90E10994216DD11462046D0
:1016100005B0BDE830406FF005BD0B4B00930B4BA0
:10162000204640216FF0CAFC002005B030BD084BB9
:10163000F4E7054B0093074BF2E7054BFAE701206F
:10164000F3E700BF60560020AC2A0B08DC2A0B0829
:101650000C780B08F22A0B082DE9F041DFF8A48082
:101660000546D8F8F80503688EB05B6A0E469847C1
:10167000F0B1314628466FF0A7FD044600B30AF0EA
:1016800065FD002704462E22394602A801979CF0EA
:10169000F9FF2046322301AA01210AF0BFF80446CF
:1016A00090B9144A01AB314628466FF069FE07E055
:1016B000D8F8F80503689B6A98470028D9D1012417
:1016C00020460EB0BDE8F08198F8103633B10A4AD2
:1016D000314628466FF054FE3C46F1E7074803F0D8
:1016E000C9F804460028EAD1054A314628466FF079
:1016F00047FEE5E7082B0B08112B0B08602600209E
:101700001E2B0B0860760020A7B5C57F0191074608
:1017100065B91F4B1B68986A03685B6B9847019912
:10172000054630B91B4A38466FF02AFE284603B0FA
:10173000A0BDBB6833B93B685B6B384603B0BDE8FE
:10174000A0401847144890F9F03A002B09DD00F545
:10175000F870019174F010F90199054608B90F4A23
:10176000E1E73846019170F045FC019905460C48C7
:1017700075F090F9019905403846FFF7EBFEEDB2A0
:10178000054001993846FFF707FF0540CEE700BF47
:1017900058260020382B0B08605600204F2B0B08D2
:1017A000D851002083680BB170F048B90120704710
:1017B00038B5054670F0D8FC044630B90C4A1378A9
:1017C00043F001031370204638BD0121094873F02E
:1017D000D3FB094806F026FB084874F05FF9284659
:1017E000FFF79AFE0649284670F0D8FBEBE700BFEA
:1017F0005C870020A056002018860020505800204A
:10180000702B0B0838B5054670F05AFD044688B1B8
:101810000948D0F8F82500F54F639A4203D000F646
:10182000285026F05BFB2846FFF776FE0349284642
:1018300070F0B4FB204638BD60760020802B0B088A
:1018400008B5064BD3F8F80503681B69984720B123
:10185000BDE8084002486FF09DBB08BD60760020DF
:101860009464002030B52DED028B85B00D46B0EEAE
:10187000408AFFF7E5FF0446C8B10AF067FC294635
:1018800009F0E0F9B4EE488AF1EE10FAF0EE400A01
:1018900074BF9FED090A9FED090A09487EBF28EE33
:1018A000008A9FED080A28EE000A05F083FD204615
:1018B00005B0BDEC028B30BDE02E6542000000009B
:1018C000D88200200000C842014802F081B800BF61
:1018D0006026002001485DF0EBBC00BFA846002058
:1018E00070470000704700000020704700207047DC
:1018F000012070477047000000207047C8207047E3
:1019000001207047012070470820704790F8903000
:101910008B4286BF00EB8100D0F894000020704716
:1019200090F890308B4286BF00EB8100D0F8940095
:101930000020704708B5034BD3F8F80503681B680F
:10194000984708BD60760020044BD3ED007AFDEE89
:10195000E77A17EE903A18B2704700BF00520020A5
:10196000014B93F85401704760460020034B93F9F4
:101970008801003818BF0120704700BF6046002072
:10198000014B93F95601704760460020044BD3F891
:10199000F80503F69833C01A18BF0120704700BF3E
:1019A00060760020704700007047000008B50448CA
:1019B00007F068FE00280CBF0A200B2008BD00BFFE
:1019C0006026002038B5154DD5F8F8050368DB69A9
:1019D00098470028D5F8F8050368DB680CBF012498
:1019E0004124984708B144F008040D4BD5F8F82578
:1019F00093F9C032002B0B4B0ADD9A420AD044F017
:101A0000400409486FF0C6FA20B144F0800401E0B8
:101A10009A42F6D144F0010038BD00BF6076002044
:101A200060560020F88100209464002000B513EE79
:101A3000103A8DB06222CDF8253013EE903ACDF8F1
:101A400029302123CDE900328DF82410192303AA6F
:101A5000C2218DED030ACDED040A8DED051ACDED01
:101A6000061A8DED072ACDED082A4CF0EDFF0DB0DA
:101A70005DF804FB2DE9F0412DED028B1D4F9FED2C
:101A80001E8A002484B005462646F0EE488A07F5F3
:101A9000516897F8903FE1B28B4216D9404641F029
:101AA00041FE80B1436836B1D3ED007AF4EEE78AA7
:101AB000F1EE10FA07DDD3ED008ADB8808EE103A6C
:101AC000B8EE488A01260134E3E76EB108235322B9
:101AD000CDE90032287CCDED028A0DEB0302AD2169
:101AE0008DED038A4CF0B0FF04B0BDEC028BBDE875
:101AF000F08100BF6026002000000000F8B5BC4C5B
:101B0000B4F86431DA07054639D504F6A44CDCEDA7
:101B1000000ADFEDB87A04F54A6C9CED000A04F681
:101B2000B84304F6AC4204F6C44604F6B44004F5E7
:101B30004B6104F54C6796ED003AD0ED002A91ED2B
:101B4000002A93ED001AD7ED003AD2ED001A287C56
:101B500060EEA70A20EE270A0521FFF767FF287C21
:101B60004CF008FF0646287C4DF008FE00F12103EA
:101B70009E4204D2287CBDE8F8404CF051B9B4F83C
:101B800064319B072ED504F5716304F5736E04F67A
:101B9000347C04F6147204F5726604F61C7004F6C4
:101BA000287104F6247796ED002AD0ED001A91ED05
:101BB000001A93ED000ADEED003A9CED003AD7EDF5
:101BC000002AD2ED000A287C0421FFF72FFF287C91
:101BD0004CF0D0FE0646287C4DF0D0FD00F12103EC
:101BE0009E42C7D3B4F864315F0733D504F67467F7
:101BF000D7ED000ADFED7F7A04F6846104F56767AC
:101C0000D1ED002A97ED000A7B4904F6886304F6BB
:101C10007C6204F5696604F69460D6ED003A90EDB6
:101C2000003A91ED002A93ED001AD2ED001A287CBB
:101C300060EEA70A20EE270A0221FFF7F7FE287CB4
:101C40004CF098FE0646287C4DF098FD00F12103EB
:101C50009E428FD3B4F864311E0723D50021674814
:101C60006DF0BCFC0721D0ED2D3A90ED2E3AD0ED71
:101C70002A2A90ED292AD0ED281A90ED2B1AD0EDC2
:101C8000260A90ED250A287CFFF7D0FE287C4CF030
:101C900071FE0646287C4DF071FD00F121039E4245
:101CA000FFF468AFB4F86431D80623D50121534856
:101CB0006DF094FC0821D0ED2D3A90ED2E3AD0ED48
:101CC0002A2A90ED292AD0ED281A90ED2B1AD0ED72
:101CD000260A90ED250A287CFFF7A8FE287C4CF008
:101CE00049FE0646287C4DF049FD00F121039E4245
:101CF000FFF440AFB4F8643199062DD5DFF808C180
:101D000004F57E6304F6E47204F57F6604F6EC7075
:101D100004F6F87104F6F47796ED002AD0ED001A77
:101D200091ED001A93ED000ADCED003A9CED013ACA
:101D3000D7ED002AD2ED000A287C0921FFF776FEB4
:101D4000287C4CF017FE0646287C4DF017FD00F16C
:101D500021039E42FFF40EAFB4F864315A0620D539
:101D6000274B287CD3ED003A93ED013A53ED032A3B
:101D700013ED042A53ED051A13ED021A53ED070A69
:101D800013ED080A0A21FFF751FE287C4CF0F2FD02
:101D90000646287C4DF0F2FC00F121039E42FFF440
:101DA000E9AEB4F864311B0620D5164B287CD3ED80
:101DB000003A93ED013A53ED032A13ED042A53ED53
:101DC000051A13ED021A53ED070A13ED080A0B2149
:101DD000FFF72CFE287C4CF0CDFD0446287C4DF00E
:101DE000CDFC00F121039C42FFF4C4AEF8BD00BF5E
:101DF00060460020E02E6542E0540020C84F0020DD
:101E00001C620020486200206056002038B5C5786A
:101E10000B46352D044628BF3525352200211846AE
:101E20009CF030FC2A4604F10C01BDE838409CF0DF
:101E3000DFBB000037B504460D4606480192114647
:101E400073F01EFD019A2946204603B0BDE83040DC
:101E500051F006BCA05700202DE9FF414FF00008CB
:101E6000CDE900289FED0F0A0F4F8DED030A0C46B8
:101E7000064615464FF47A73B1F90220D7F8B01D23
:101E800051F0C8FECDE900589DED030AB4F90420D5
:101E9000D7F8B41D4FF47A73304651F0BBFE04B04E
:101EA000BDE8F0810000FA446056002008B54EF00D
:101EB0005BF840F4E67040F0010008BD13B54FF444
:101EC0004470CDE900210FF067FF044628B1DDE939
:101ED000002152F065FC024B2360204602B010BD89
:101EE000BC2D0B0810B504460FF05EFF204610BD58
:101EF0000B4B93F808267AB993F8102662B9D3F8F9
:101F0000F80503F69832904208D003F53D639842F5
:101F100014BF04200320704705207047022070473B
:101F20006076002008B54B69012B07D1084873F093
:101F3000BFFD08B1002008BD0420FCE7022B03D13F
:101F4000034873F0C1FDF4E7BDE808404EF0F2B875
:101F50005058002010B594B0044603A80FF0ECFBD5
:101F60001A4BD3F8F805036803A91B6C984750B3C4
:101F7000247C76F001FD059BDDED047A0893069B39
:101F800009930023F8EEE77A9FED117A0B930C93F7
:101F90000D930E930F931093119312934FF6F853E2
:101FA000ADF84C300023962267EE877A8DF84E30DC
:101FB0003323CDE90032079007AA57212046CDED03
:101FC0000A7A4CF041FD14B010BD00BF60760020CD
:101FD0000AD7233CF0B52DED028B2C4C0546D4F8E6
:101FE000F80503688BB0DB689847002849D0D4F81F
:101FF000F84527482F7CDFED278A70F095FB236892
:1020000020461B6B60EE288A9847BDEEC00A20462A
:1020100010EE103A1EB22368DB6A9847BDEEC00A84
:10202000204610EE103A1DB22368DB6B9847DFEDB7
:102030001A7A2368B4EEE70AB0EE408AF1EE10FA9D
:102040005B6B58BFB0EE678A20469847BCEEC88AE3
:10205000002303930593069318EE103AB722ADF8C8
:1020600024301A23CDE900323E2103AA3846CDEDB3
:10207000048A8DED070AADF82060ADF822504CF0CF
:10208000E3FC0BB0BDEC028BF0BD00BF607600201E
:1020900064520020E02E654200FF7F4770B52DEDB1
:1020A000048B044688B02948DFED298A74F02EFCA1
:1020B000D8B3492054F0A4FF9FED269A20EE090AD8
:1020C0004A2020EE288A54F09BFF20EE090A60EE99
:1020D000288A267C76F050FC0546204651F0D2FF37
:1020E000BDEEC88AFDEEE88A18EE103A18EE902A86
:1020F000ADF80C300023CDE90533ADF80E30ADF866
:102100001020ADF812308DF81C30ED221623CDE9E9
:1021100000328DF81D0002AA2221304602954CF0B3
:1021200093FC08B0BDEC048B70BD1A2054F068FF1E
:10213000DFED097A80EE278A462054F061FFDFED5B
:10214000077A28EE288A20EE270AC0E7D851002017
:1021500000401C466F12833A00A08C450AD7233CEE
:102160002DE9F047044692B0007C4CF003FC054694
:10217000207C4DF003FB00F126039D4205D2207C1C
:1021800012B0BDE8F0474BF04BBE424807F07AFA78
:10219000002878D0404B1F68002F74D01921384692
:1021A00041F044FB00286ED009F0D0FF064604A899
:1021B0000FF0C2FA04A9304609F08AFD4FF0000A78
:1021C00097F88082D1465FFA8AF398455BD994F8F4
:1021D0000F330133DBB2434534BF84F80F3384F847
:1021E0000F9394F80F13384641F09CFA05460028E7
:1021F0004CD0836893F92130192B47D142F090F9E4
:10220000002843D02B6803A91B6A2846984708B9C1
:1022100000230393284642F079F994F8108007468A
:1022200076F0AAFB6A68DDED057A94F80F33126840
:102230009FED1A7A8DF84430F8EEE77A3B1F5F4243
:1022400008900F920698039AD6F80C1209905F41F5
:102250000798109267EE877A2F222623D6F804C2B9
:10226000D6F808420A90CDE900320E9108AA42F64B
:102270001E314046CDED0B7ACDF830C00D948DF86F
:1022800045704CF0E1FB12B0BDE8F0870AF1010A9D
:1022900099E700BF60260020E48700200AD7233C8E
:1022A0002DE9F04300F50057C7B097F85859044698
:1022B0000E46002D35D07022002106A804F5A0445A
:1022C0009CF0E0F904F678331868FEF715F9012D53
:1022D0008046894628D004F67C342068FEF70CF945
:1022E00004460D4676F048FB4FF47A7250430022C4
:1022F00097F858392290239202A9802224A88DF8B9
:102300001031CDE90289CDE904459CF071F97122C3
:102310008923CDE9003242F2283122AA30464CF01E
:1023200093FB47B0BDE8F08300240025DAE7000006
:102330003C2938B5054620D008D81B2911D02429BE
:1023400026D02846BDE8384051F096BF4D29F8D137
:1023500026214BF077FD044640B12846FFF700FFE9
:1023600005E016214BF06EFD044610B9002420460E
:1023700038BD2846FFF792FEF9E789214BF062FD50
:1023800004460028F2D0297C0748FFF789FFEEE7D2
:102390000C214BF057FD04460028E7D0297C034868
:1023A00073F09EFBE3E700BF60260020505800203A
:1023B00030B52DED028BCD7891B0272D0C464FF026
:1023C00027024FF0000106A828BF27259CF05AF9E4
:1023D00004F10C012E4C2A4606A89CF009F9D4F809
:1023E000F80503681B69984700284CD09DF83E50BB
:1023F00015F04001019146D1FFEE000A40F28F3006
:10240000B7EE001A9DED0E0ADFED228A1FF042FFA3
:102410000199D4F8F8058DED0E0AB0EE408A02F06D
:10242000B3FF15F0040F68EE000A9FED1B8A1BD066
:10243000079B0293089B0393099B049302A80A9BA2
:10244000CDED010A059322F069F820EE280ADDEDB2
:10245000010A20EE080A04F6784011B0BDEC028BA8
:10246000BDE8304004F07ABF9DED0D0A20EE280A49
:1024700004F6784020EE080A11B0BDEC028BBDE8EE
:10248000304004F097BF11B0BDEC028B30BD00BFEF
:1024900060760020E02E65420000C84270B50E4E06
:1024A000D6F8F805036886B01B690C46984780B1DA
:1024B00002AD28460FF040F906AB13E903008DE8A2
:1024C000030004F1080195E80C0006F6784005F0D9
:1024D00057F906B070BD00BF6076002070B5304D72
:1024E0002DED028B0646D5F8F80591ED018A0368BB
:1024F0008AB01B690C46984750B9BDEEC88A18EEE1
:10250000103ADB0704D402200AB0BDEC028B70BD88
:10251000D4E9040120F0D0FC0028F4D0236913B9D9
:102520006369002BEFD002A80FF006F902AA21463A
:10253000304651F0DFFA0028E5D0D5F8F8050368F9
:102540001B699847D0B194ED000ADFED167AB4EE1E
:10255000E70AF1EE10FA1ADA06AC20460FF0ECF8B2
:102560000AAB13E903008DE803000F4894E80C0060
:1025700002A905F005F940B10020C5E70B48022289
:102580000F2106F05DFF0028DDD10420BCE7D5F85F
:10259000F8050368DB6C98470028DDD1F5E700BF3C
:1025A0006076002000000034D882002060260020E1
:1025B00030B58C8BC22C85B005460B463AD00CD872
:1025C000B22C26D0C02C30D0142C42D0194628462C
:1025D00005B0BDE8304052F0E7BCD12C3FD0B4F597
:1025E000967FF3D1D1ED007A9FED2D7AF0EEE77A68
:1025F000F4EEC77AF1EE10FA50D5D1ED017AF0EE93
:10260000E77AF4EEC77AF1EE10FA47D525490222AF
:1026100021E0254A91ED010AD2F8F8050268D26C52
:102620009047A0B9042005B030BD05B0BDE83040EA
:10263000FFF754BF1C4A91ED000AD2F8F845F7EEB7
:10264000000A1FF023FD0146204602F0B1FE0020E3
:10265000E9E716490222164806F07CFEE1E7D1EDD3
:10266000017AFCEEE77ACDED027AD1ED007A9DF8A1
:102670000830FCEEE77ACDED037AD1ED027AFDEE7B
:10268000E77A17EE902A12B2009291ED030A9DF8B4
:102690000C200146064805F0ABFEC4E70220C2E765
:1026A000000000345083002060760020A0850020C8
:1026B000602600202DE9F04F2DED028BDFF870A28F
:1026C0009FB0084610A9FFF7A1FBDAF8F8050368E8
:1026D0001B699847002800F0128104AE30460FF0C5
:1026E0002BF88B48314609F037FB002800F00781B2
:1026F0009DF874C0BCF1010F04D0ACF10703022BAC
:1027000000F2FD800AF264530FCBBDF8705008ACA4
:1027100084E80F0015F0030305F0180905F0C00B5D
:1027200005F4806805F4006702931ED1BCF1070F21
:102730009DED110ADDED120A14D0ACF1080CBCF1CC
:10274000010F00F2A480734B93ED037AD3ED007A6E
:1027500060EEC76A67EEA00AE0EE276AE0EE070ABD
:10276000B0EE660A20460FF0E7FAB9F1000F40F02C
:1027700093804946DAF8F80502F006FEDDED157A99
:102780009DED147A8DED030A27EEA70AA7EE070A3E
:102790001FF0B0FC9DED031A40F2E330F1EE410A68
:1027A0001FF078FDDDED140AB0EE408A9DED150AAC
:1027B00099F06EFDDFED587A9DF8743060EE277A5F
:1027C000083B9FED560A012B67EE807A0CD8544BDC
:1027D00003F58D6393ED000AB8EEC00A30EE270AC8
:1027E0001FF002FDF0EE407AB8F1000F1BD19FED13
:1027F0004A0ADDED1A7A9DF8743067EE807A083B5C
:102800009FED460A012B67EE807A0CD8444B03F506
:102810008D6393ED000AB8EEC00A30EE270A1FF070
:10282000E3FCF0EE407A002F3BD19FED3B0A9DED9B
:102830001B7A27EE007A9FED390A27EE000AB9F1DC
:10284000000F4BD105F44065B5F5406F5CD09FEDAE
:10285000357ADDED146AF4EEC76AF1EE10FAFFEE98
:10286000000AB7EE007A88BFF0EE470A029B002B01
:1028700037D0BBF1000F42D0B5F5406F14D168EEF0
:10288000200A2948B0EE670A04F068FD37E096E8B0
:102890000F0084E80F0065E7DFED247AB0EE678A69
:1028A000A2E79FED220ACAE7B8F1000F06D037BBB6
:1028B00068EE200A1C4804F07DFD20E0FFB1DEE751
:1028C000BBF1000F1BD0B8F1000F03D1BFB1DFED9A
:1028D000170AD6E79FB9DFED150AEBE7029B002B3D
:1028E000EED10CAD28460EF027FFDDE90E018DE894
:1028F00003000D4895E80C00214604F041FF1FB08D
:10290000BDEC028BBDE8F08FF7EE000AAEE700BF2A
:10291000C8380020183B0020E02E65420000C84265
:1029200060360020000000B4D882002000000000C3
:10293000607600202DE9F04F2DED028BDFF8D0B14D
:102940009BB008460CA9FFF761FADBF8F8050368AD
:102950001B699847002800F095809DF864300B2B88
:1029600000F29080DFE803F0068E8E068E06068E5B
:102970008E8E06060BF264530FCBBDF8604004AD9B
:1029800014F0030985E80F0004F0180804F0C00AE9
:1029900004F4806704F4006609D1DDE90D0120F03C
:1029A0008BFA00286ED00D9B06930E9B0793B8F10F
:1029B000000F6CD14146DBF8F80502F0E5FCDDEDD7
:1029C000117A9DED107A8DED030A27EEA70AA7EE86
:1029D000070A1FF08FFB9DED031A4FF48A60F1EE9A
:1029E000410A1FF057FCDDED100AB0EE408A9DED64
:1029F000110A99F04DFCDFED417A60EE277A9FEDE8
:102A0000400A67EE807A4FB99FED3C0ADDED167AF9
:102A100067EE807A9FED3A0A67EE807A002E3BD10E
:102A20009FED360A9DED177A27EE007A9FED340A66
:102A300027EE000AB8F1000F53D104F44064B4F556
:102A4000406F4BD09FED2F7ADDED106AF4EEC76A30
:102A5000F1EE10FAFFEE000AB7EE007A88BFF0EE52
:102A6000470AB9F1000F1AD108AC20460EF064FEF7
:102A7000DDE90A018DE80300234894E80C002946AB
:102A800004F07EFE1BB0BDEC028BBDE8F08FDFEDE5
:102A90001F7AB0EE678AB6E79FED1C0ACAE7BAF163
:102AA000000FEFD0B4F5406F07D168EE200A16484A
:102AB000B0EE670A04F052FCE4E73FB1002EE1D12A
:102AC00068EE200A104804F075FCDBE7002ED9D030
:102AD000EBE7002ED6D1DFED0D0AF3E7F7EE000AA3
:102AE000BFE7B9F1000FBFD0BAF1000FCAD0002F75
:102AF000EFD1002EC6D0DFED050AD8E7E02E654203
:102B00000000C842000000B4D8820020000000008D
:102B10006076002010B44B7A8C7ACA7A43EA042398
:102B200043EA0243542B07D0562B09D0522B0BD12A
:102B30005DF8044BFFF73CBC5DF8044BFFF7BABDF2
:102B40005DF8044BFFF7F6BE5DF8044B51F0C4B8D6
:102B5000014B93F85201704760460020084BD3F8B0
:102B6000F81503F6B872914201BFA3F5005393F92B
:102B7000EC01B0FA80F0400918BF0020704700BF98
:102B800060760020084BD3F8F81503F6B87291422E
:102B900007D1A3F5005393F9EC01431E5842584165
:102BA00070470020704700BF6076002038B5036A88
:102BB0001D4D43F4B84303620446D5F8F805036895
:102BC0001B6A984738B1D4E9092342F4406243F4C0
:102BD00040636262A362D5F8F8050368DB68984732
:102BE00038B1D4E9092342F4A04243F4A04362621D
:102BF000A3620E4B1868A8B190F8803293B1236A93
:102C000043F480732362636A43F480736362002138
:102C100040F088FD30B141F083FC18B1A36A43F461
:102C20008073A36238BD00BF60760020E487002077
:102C30007FB500F530560436044630466FF074FD1B
:102C4000DFED1D7A04F5935020EE270A002301A939
:102C5000083001938DED020A039307F0A5FC09F0FB
:102C600075FA09F01FF804F57C6504F5325220323C
:102C70006D21284647F00EFF284606F543726C2169
:102C800047F008FF204601F061FB30B104F53952EE
:102C900030326A21284647F0FDFE04F5405393F98F
:102CA000F03A002B06DD04F53F5220326921284618
:102CB00047F0F0FE04B070BDE02E65422DE9F04F04
:102CC000054695B0344806F0DDFC002861D005F5D6
:102CD00051691921484640F0A9FD002859D010A893
:102CE0000EF02AFD05F5935010A9083008F0F0FF0A
:102CF000DFF8B8B0002795F8903FFEB2B34248D94C
:102D00003146484640F00EFD044600283FD0836817
:102D100093F92130192B3AD141F002FC002836D02A
:102D200063681A6905EB860303F5A043D3F8181608
:102D300091422CD0C3F8182623680FA91B6A20469D
:102D4000984708B900230F9375F01EFE0D900F9859
:102D50008A46FDF7D1FBCDE90A0161680868FDF7F5
:102D6000CBFBCDE9080113990D9A0C4B06911299F2
:102D7000019305F57C680A4B0093CDE90461CDE928
:102D8000022A0849084A5B46404648F0FFFB0137E3
:102D9000B1E715B0BDE8F08F60260020F32E0B08D8
:102DA000FA2E0B08EE2E0B08CF2E0B08C82E0B08A0
:102DB000F0B58BB0154606460F462422002101A827
:102DC0001C469BF05FFCA3238DF8043095238DF8FF
:102DD000053003238DF8063075F0D6FD2B6804937B
:102DE0006B680593AB680693236807936368CDF817
:102DF0000700CDF80B1008932422A3688DF80F70FC
:102E000001A906F57C60099347F0ACFF0BB0F0BD5B
:102E100030B589B01D220446002168469BF032FC83
:102E2000A3238DF8003095238DF8013001238DF810
:102E3000023075F0A9FD04F5A045CDF80300D5F8E2
:102E4000F805CDF807100368DB6B984710EE103AD1
:102E5000D5F8F805CDF80B300368DB6A984710EE1B
:102E6000103AD5F8F805CDF80F3003681B6B98477A
:102E700010EE103ACDF8133004F58053D5F8F8056C
:102E8000D3F86834ADF8173003685B6B984710EEE1
:102E9000103A1D22694604F57C60CDF8193047F0E0
:102EA00061FF09B030BD00002DE9F04F2DED068B1C
:102EB00000F5405591B095F9F03A002B06464CDDEF
:102EC00000F57C6900F54750303072F055FD04463E
:102ED000002847D095ED8F8ADFED247A95F8B0422F
:102EE00028EE278A75F050FD06F52D558046E86FCF
:102EF0000F46FDF701FB8246D5F880008B46FDF7B3
:102F0000FBFA41EC190BD5F88400FDF7F5FA41EC1A
:102F10001A0B06F56B50303005F094FD10EE100AD8
:102F2000FDF7EAFACDE90E0118EE100A8DED0CABB3
:102F30008DED0A9BCDE908ABFDF7DEFA0C4B019352
:102F40000C4B0093CDE90601CDE902870A4B0B4AF1
:102F50000B490494484648F019FB11B0BDEC068BB0
:102F6000BDE8F08F9FED078ABCE700BFE02E654209
:102F7000442F0B084C2F0B08042F0B080C2F0B08A9
:102F80003F2F0B085241C07F30B52DED028B00F56D
:102F900030558BB0043504462B4B009369462846C8
:102FA0006FF0B2FC2122002101A89BF06BFBA32350
:102FB0008DF8043095238DF8053002238DF8063006
:102FC00075F0E2FC04F54053CDF80B10D3F8B03D9A
:102FD000CDF80700B3F90830ADF80F3004F52D53E4
:102FE00038339FED1A8A5B6ACDF8113004F5A0439F
:102FF000D3F8F80503689B6B984710EE103A284603
:10300000CDF81530009BCDF819306FF07DFA20EE29
:10301000080A04F5AB5010EE103A04F5AD511C301F
:10302000CDF81D3022F0D2F820EE080A212210EE51
:10303000103A01A904F57C60CDF8213047F092FEEA
:103040000BB0BDEC028B30BD5241C07FE02E65421B
:1030500070B590F8AB2B00F698030C2101FB0233FE
:1030600000F530558AB004350446D3F888611C4B0E
:10307000019301A928466FF0D9FB1D22002102A867
:103080009BF000FBA3238DF8083095238DF80930C1
:1030900075F07AFC04F54053CDF80B00D3F8B43D3D
:1030A000CDF80F10B3F90830ADF8133004F52D53F7
:1030B000383328469B6ACDF815306FF09FFD10EE2F
:1030C000103A1D22CDF8193002A9019BCDF81D3010
:1030D00004F57C60CDF8216047F044FE0AB070BD75
:1030E0005241C07F13B5044604F5805400F57C605E
:1030F000019047F03DF9019847F0D4F994F9783000
:10310000019823B102B0BDE8104047F073BA02B095
:1031100010BD000010B500F5A0430446D3F8F80533
:1031200003681B68984704F50053014693F804218F
:1031300004F57C6047F0D6FF04F59350083009F0A1
:10314000FBF904F59070BDE8104016F0D7BF000001
:10315000992070472DE9F3410446043052F036FCC3
:103160003E4E3F4B63605425601952F0E5FD6651B9
:103170003035B5F5557FF7D104F5557054F004FAA4
:1031800004F25C7104F5FC65084601916BF0FCFFEC
:10319000019928466CF066F904F67C27294604F567
:1031A0001F6073F0ADFA38466FF0C4F8002104F6E2
:1031B000B86071F015FC04F577605DF0ABFE04F6C5
:1031C000B87072F059F904F5825004F58058103047
:1031D0003FF08EFF04F5CD56224BC8F8503004F571
:1031E000835004F589551C351836083072F07AFB87
:1031F00032463946284670F0D7FA1B4BC8F83C31A6
:1032000004F5C8500EF098FA05F2D4700EF094FA56
:1032100004F5C9500EF090FA05F2F4700EF08CFA35
:1032200004F5CA500EF088FA05F614000EF084FA80
:1032300004F5CB50083005F095FA394630466FF06A
:103240009DFE04F5DC50083003F092FC204607494F
:103250003FF002F8204602B0BDE8F081E8710B08AB
:10326000FC710B08EC2B0B08D4B90C0850690B0847
:10327000F0B500F50551B5B010220831044646F00E
:10328000ADF9574800222B213EF04EFD3FF0EAF900
:10329000544A13881A2143F002030020138054F08B
:1032A000FDF80220462154F0F9F8204601F04EF8CE
:1032B00040B104F544501E2314A938308DF8503025
:1032C0003FF0E0FD484D53F0F3FE95E80F0004AEEB
:1032D00086E80F0002A930463EF02EFCF0B105F161
:1032E000100314AA183518685968164603C608331F
:1032F000AB423246F7D118681B79306033719DF8C4
:1033000008300C2B0AD834AA1344079813F8803CD1
:1033100000EE103AB8EE400A3FF03EFB334D95E820
:103320000F0008AE103586E80F0095E80F000CAFCF
:1033300087E80F0003A930463EF0FEFB0146002857
:1033400049D00021B7EE000A30463EF041FC04F5BA
:1033500006552749802214A89BF04AF90835082110
:1033600014A800223EF0E0FC10A928463EF012FA14
:1033700000282ED01F490B68D8070ED41E4B04F529
:10338000F45210321A6004F501520832DA6004F582
:10339000FF5210329A6101230B602846164903221E
:1033A00001253EF017FD154A0095002304F57C61C8
:1033B000FD203EF0BDFC124B1A68D20705D4114A1D
:1033C0001D6004F58C540C3414600E4801213EF04D
:1033D0001DFD35B0F0BDB7EE000A3846B5E700BFB9
:1033E000A0660B08C887002040280B0860280B083F
:1033F00080280B085026002000220020680F0C08AF
:1034000054260020242200200069C0F34010704799
:103410000F299DBF302303FB01005030002070476F
:10342000014B93F97C01704760460020024B93F8F2
:10343000000600F0010070476076002008B50368C0
:103440009B68984780F00100C0B208BD014BD3F8DB
:10345000B00D70476056002000290DDB074890F83A
:10346000CC2DCBB29A4207D3D0F8C83D0122595C8B
:10347000A0F5405005F0E4BF704700BF6056002043
:1034800008B53AB1022A10D1BDE8084007483522F4
:1034900005F060BF064AD2F8F8258A4205D152F0FD
:1034A00015FCBDE8084052F09BBB08BD602600201B
:1034B0006076002030B589B01C220021104D03AC8D
:1034C00001A89BF0DFF820460EF036F905F26453B0
:1034D0000FCB84E80F00102301A905F62850ADF8A2
:1034E000063022F097FD40B1064BB5F85C2D1B6805
:1034F0000549986903681B68984709B030BD00BF4B
:10350000607600205826002000700B0801290A462A
:1035100003D0022900D019B90122024805F0FEBAF1
:10352000704700BF506100204A2910B40B46044682
:103530002FD026DC3F2921DC292913DC04390C2972
:1035400018D9204619465DF8044B53F0ABB9A3F1E6
:10355000C9000121814040F243400142F1D05DF8B1
:10356000044B70472A39012088400C49014000294A
:10357000E7D0F4E701200A499840F7E74829E0D16D
:10358000EDE7D329DDDCC829E1DC6129E7D09B29FF
:10359000F5E75DF8044B1146FFF7B8BF01FF2200C5
:1035A000900001000B464A2BF7B5064611465FDC3A
:1035B000292B0FDC072B70D056DC002B5DD0042BA1
:1035C00000F0AC800A463046194603B0BDE8F04032
:1035D00052F02CBFA3F12A02202AF3D801A050F800
:1035E00022F000BF21370108C5350108C5350108A3
:1035F000C5350108C5350108C5350108C5350108BF
:10360000C5350108F3360108FF3601080B370108FC
:103610001137010817370108273701082D3701082E
:10362000C5350108C535010833370108C53501081E
:10363000C5350108C53501083F370108C535010802
:10364000C5350108C5350108C5350108C53501086E
:10365000C5350108C5350108C535010839370108E8
:10366000C53501084D370108102BABD14D4949E054
:103670009B2B6FD003DC612BA4D101240AE0A3F1C2
:10368000C9050A2D9ED8012404FA05F540F24342EB
:10369000154297D0204603B0F0BD022AEDD1424D2D
:1036A000D5F8F83505F54F67BB42E6D03F486DF0D9
:1036B00071FC044678B905F6285022F069FA51F0F9
:1036C00051F83B4A05214AF0A1F92146A5F5A04051
:1036D00000F044FED1E7D5F8F835BB42CDD0B5F9BE
:1036E0005C3D13B93046FFF7E5FE3046FFF7E2FEDA
:1036F000D0E70229C1D12F4800F0D0FFBDE70A462C
:103700002D493046FFF7BCFEB7E70A462B49F8E7DC
:103710000A462B49F5E70A462A49F2E72A49F1E722
:103720000A462A49EDE70A462949EAE70A462949AD
:10373000E7E70A462849E4E70A462849E1E71A4B41
:10374000D3F8F80503685B6D984796E73046FFF7B6
:10375000DDFE92E72248019273F0D8F800288CD160
:1037600012486DF017FC0446002886D00E4BD3F8A3
:10377000F82503F6B86082423FF47FAF03F53D635E
:103780009A423FF47AAF019902297FF476AF1A206A
:1037900053F008FE50F0E6FF124A01994AF036F95C
:1037A00078E700BF508300206076002094640020FA
:1037B00014700B086026002068820020A082002080
:1037C0006485002030820020A0850020DC85002058
:1037D000D882002018850020188600207063002001
:1037E000D85100202D700B08002070470020704732
:1037F000002070470020704700207047002070476D
:10380000002070470020704708B50368DB689847C0
:1038100080F00100C0B208BD012070470120704750
:103820009FED010A704700BF0000000000207047B4
:10383000012070470020704770470000102070473B
:103840000048704718720B0870470000002070474E
:1038500001207047002070470020704700F5055098
:103860000C3070470048704710530B0800F5A0401B
:10387000D0F8F80503681B681847000000F5A0435E
:1038800000F5B940D3F8F83570301B1A584258414A
:1038900070470000034808602021117008221A6058
:1038A000704700BFB0740B0803685B6818470000DE
:1038B00000F0A0BF00F0FEBD54F0B6BE45F0B4BAB3
:1038C0001CF066BC47F0B4BB05F0ACBB04F01EBBFB
:1038D00001F0A6B801F03CBA0CF0FAB854F04ABABC
:1038E00056F050BC0BF07ABC52F03EB951F044BED9
:1038F00050F008B805F092BB05F0AEBB72F0CAB943
:103900000AF0B8BD17F052BB00F0C4BC05F04CBCC7
:1039100004F004BF01F0EAB910B50368DB6804469F
:10392000984728B120460021BDE8104001F040BD75
:1039300010BD000003F030B802F06ABD02F0AEBA6C
:1039400070B50A4B0446D3F8F8050368DB680E46E9
:103950009847054640B104F5A044D4F8F80503683B
:10396000DB6B984786ED000A284670BD6076002024
:1039700070B50A4B0446D3F8F8050368DB680E46B9
:103980009847054640B104F5A044D4F8F80503680B
:10399000DB6A984786ED000A284670BD60760020F5
:1039A00070B50A4B0446D3F8F8050368DB680E4689
:1039B0009847054640B104F5A044D4F8F8050368DB
:1039C0005B6B984786ED000A284670BD6076002044
:1039D00070B500F5A0430446D3F8F805036886B037
:1039E0001B690D46984780B102AE30460DF0A4FE2B
:1039F00006AB13E903008DE8030004F5B84096E830
:103A00000C002946783003F0BBFE06B070BD000004
:103A100070B51F4B036000F5A0430446D3F8F804CB
:103A20001C4AC3F8482308B10EF0C2F91A4B2360B0
:103A300004F5805393F82C2E42B9D3F8285E2DB1AB
:103A400028461BF05BFA28460EF0AEF904F58B50C1
:103A500010306CF0E3FD04F58350183054F0BEFBD9
:103A600004F6C44504F66446B54204D0183D284621
:103A70001AF098FEF8E7094BC4F8983804F6941049
:103A800049F02CF904F5106049F028F9204670BD82
:103A900040770B0870270C08D0080C080CD20B08D4
:103AA00038B5484B044640F8043B54F0DDFE04F1C1
:103AB00010000BF0B9FC04F1680044F043FF04F57A
:103AC000907015F0FDFE04F586600AF043FB04F2E9
:103AD00054500EF06FF904F698001CF0FDF904F54F
:103AE000446054F09FFC04F551603FF0C5FD04F5BF
:103AF0007C6047F07FF804F58350183054F056FB93
:103B000004F5855014300CF081FF04F58B50103013
:103B10006CF070FD04F58C500C3045F0D5FA04F5CE
:103B20008F5056F04FF804F580530025264A83F84D
:103B3000045204F5905004F590530433143013608C
:103B40003BF0E8FB04F593502946083006F080FE70
:103B500004F5C550183065F0EBF804F5E5501C305D
:103B600069F030FA04F5EE5014306BF09DFE04F568
:103B7000F15018306CF0D2FA04F5F450103005F022
:103B800089FD04F5FF50103065F030FD04F501505B
:103B900008305BF0BBF804F5005304F5045083F8DB
:103BA00004510A4D1C306DF0F9F82B6813B1084828
:103BB00074F0B0FE204607493EF04EFB2C602046D4
:103BC00038BD00BFD0080C08B49000201888002031
:103BD00020720B08F8070C08F8B50446254601F0DA
:103BE00047FA214B45F8383B204B6465C4E916344D
:103BF0001F4BC4E918341F4BA36604F17C000DF081
:103C00009BFD04F198000DF097FD04F1B4000DF058
:103C100093FD4FF6FF76184BC4F8C830A4F8CC607B
:103C200004F1D0000DF088FD4FF0FF37134B14491D
:103C3000C4F82C7128461D603EF00EFBA4F8747089
:103C4000A4F8906004F5A2700DF076FD04F5BE7046
:103C50000DF072FD04F5CC700DF06EFD04F5DA7018
:103C60000DF06AFD2046F8BD507B0B083539010880
:103C7000393901083D3901080000FFFF0C87002099
:103C800054DF0B082DE9F041044686B0FFF708FF2A
:103C9000874B2360874B8848186004F5055204322F
:103CA000002314269DB206FB05010133097C00297F
:103CB000F8D1824B1D80824B196811B1814874F094
:103CC00029FE04F5065008301A60FFF743FA04F5A0
:103CD000765028306EF014FB04F5405504F505537A
:103CE0003D33C5F8C83D04F57750062385F8CC3D33
:103CF000103053F06DFE04F5785034306DF00AF951
:103D0000714BC5F8343E04F579502C306DF0ECF869
:103D10006E4BC5F86C3E04F57950303004F5A04583
:103D200004F5A6475EF070FC4837694BC5F8483388
:103D300007F1080073F0D6FF04F5A64604F5A7487E
:103D4000743608F15808304614364DF0D3FFB045AC
:103D5000F9D10723C5F8FC340023A5F800354FF44A
:103D6000CB700EF01FF8C5F8F80404F5AA40043033
:103D700073F0B8FF04F5AA40483073F0B3FF554B19
:103D80001A6802B91F60544BC5F8483304F5AA40BD
:103D900064300DF0D1FC04F5AA404FF4805174302A
:103DA0000BF01CFC04F5B7464C4B059318364C4BF6
:103DB000C5F8F8650494009304F5AC4006AB13E92C
:103DC0000C004FF4007144300AF0A0FE304601F0C0
:103DD0004FF9444BC5F8983B04F5B740503001F01B
:103DE00047F9414BC5F8D03B04F5B840083001F025
:103DF0003FF93E4BC5F8083C04F5B840403001F0AF
:103E000037F93B4BC5F8403C04F5B840783001F039
:103E10002FF9384BC5F8783C04F5B94060300DF007
:103E20008BFC04F5BD4604F5B94038367030FFF719
:103E3000D3FE304601F01CF92F4BC5F8B83E06F111
:103E400038000DF079FC04F5BE40043001F010F9A3
:103E50002A4BC5F8043F04F5BE40403001F008F994
:103E6000274BC5F8403F04F5BE407C3001F000F917
:103E7000244BC5F87C3F04F5BF40383001F0F8F81A
:103E8000214BC5F8B83F04F5BF4578354FF0804663
:103E900003A92846039649F0FDF902A905F10C0093
:103EA000029649F0F7F9204606B0BDE8F08100BF60
:103EB00040770B08D8870020A06B0B08D487002020
:103EC0009487002034720B089C2B0B08DC2B0B080A
:103ED00070270C08348B0020902E0B081539010830
:103EE00030770B0858720B089C7D0B08847E0B08FA
:103EF00070790B08307D0B08107E0B0874800B085E
:103F0000047F0B0808800B08787F0B08F0B5044687
:103F100000F5785085B0343004F59356FDF7FCFA7F
:103F20000836204605F054F90021304608F094F890
:103F300004F5AA416431304607F0CAFE04F5A045F5
:103F400004F5805785F8140697F8E41411F0010180
:103F500003D1236820469B6C9847002301A9304673
:103F600001930293039307F003FF28B301A820F005
:103F7000C1FD05F5C86585ED000A0121204605F063
:103F80007DFB28B12046FEF753FE2046FEF78CFF4E
:103F90008021204605F072FB18B11DF073FC1BF068
:103FA00033FE4FF48011204605F068FB10B1304617
:103FB00006F0D4FB05B0F0BD94F8E433B02202FB68
:103FC000034394F8282493F8C131002AD5D1022B59
:103FD00081BF07F26C6705F5C8653B682B60CCE7CD
:103FE000FFF794BF70B500F50053044693F97431A0
:103FF00033B300F5A043D3F8F4540DB374F0BCFC14
:1040000004F5745393ED030ADFED0E7A9FED0E1A5B
:10401000DFED0E0A451B20EE270A40F269101EF064
:1040200039F9FCEEC07A204617EE903A9D42084AD4
:10403000BDE8704034BF00230123022100F09ABD87
:1040400070BD00BF00007A440000804F00000000F7
:1040500036650B08FFF7C6BF37B50221044605F0E9
:104060000DFB50B10121204605F008FB28B9204680
:10407000FEF7DEFD2046FEF717FF1021204605F073
:10408000FDFA10B12046FEF7E3FF2021204605F09F
:10409000F5FAF0B1204604F56D55FEF7B9FE284655
:1040A0006EF0B0FFA8B128466FF0A4F804F57C606C
:1040B0002C461C3404F140026E21019046F0EAFCCB
:1040C000019804F16C026F2103B0BDE8304046F066
:1040D000E1BC03B030BD0000FFF7BEBF10B54FF428
:1040E0000051044605F0CAFA10B12046FEF74CFF15
:1040F0004FF48041204605F0C1FA38B12046FEF762
:10410000F1FF04F5235024306BF03AF9802120466A
:1041100005F0B4FA28B11DF0B5FBBDE810401BF066
:1041200097BD10BDFFF7DABF73B50368354D9B6DC2
:10413000044604F578569847343653F045FB53F05F
:104140002DF800213046FDF7DFFAA87130462E4EDB
:104150000123EB716CF01EFF33682871DB6A2B4A78
:1041600093F89C306B7104F50055B5F8521111703D
:1041700013B9204600F070F93368DB6A93F89C604D
:1041800036B195F806311BB974F0F6FBC5F8080195
:1041900085F8066104F5405604F52D5596ED0E0A96
:1041A000383528468DED010A72F0B0FB014604F562
:1041B0004B509DED010A04306FF038FC96ED0E0A6D
:1041C00028468DED010A72F0A1FB9DED010A014622
:1041D00004F56D506EF056FF44F0DCFE44F044FBF5
:1041E00004F5255028306BF0FFF965F003FB044619
:1041F000284673F0AFFC0146204602B0BDE870408F
:1042000065F0D4BA3D87002058260020892300207D
:10421000FFF78ABF10B5094B1B78044623B100F5A0
:10422000305004306EF09AFE04F5A044D4F8F8053E
:104230000368BDE810409B68184700BF688B0020EA
:10424000FFF7E8BF38B5054B1C6823680A461D68B0
:10425000034B01462046A847002038BD58260020C1
:104260006026002010B573F0B3FF064C064B1860B3
:104270002046FFF707FD2046044A0549BDE81040E7
:1042800097F0BEBC6026002058260020DCE200200B
:10429000113A010813B500F5A043044693F8953B85
:1042A00023B102B0BDE8104003F0D6BF00F5305096
:1042B000002301A9043001936EF0B8FA04F5785098
:1042C00034306CF067FE014604F52D50D4ED460AFB
:1042D0009DED010A383073F0E9FB02B010BD00001B
:1042E00010B500F54053D1ED007A9FED157AD3ED6E
:1042F0004D0A93EDAF0A90ED461A00F5005367EEB4
:10430000C77A9FED107A93F8783B67EEA07A20EE9B
:10431000070A13F00C0F00F530500C46A7EE870A81
:1043200014BF0121002160EE870A04306EF01AF9F3
:10433000DFED057A20EE270A84ED000A10BD00BFEC
:104340000AD7233C35FA8E3C0000C84200F54050A5
:1043500090F9F400C31E5842584170477FB5044697
:1043600004F59355684608350E460DF0E5F92846E4
:1043700006F0FAFD18B90025284604B070BD69465C
:10438000284607F0A5FC0028F5D023683246DB6CF0
:1043900069462046984705460028ECD0012104F5DF
:1043A000415070F0E9FDE7E7F0B52DED028B0446D2
:1043B00000F5935087B008300D46174607F076FB9E
:1043C000064600283DD03FB104F5805292F8E4340F
:1043D00043F0020382F8E43404F5BA40283021F0B7
:1043E00039FED5ED017A9FED197A9FED198AF8EE25
:1043F000E77A04F5A64467EE877A483417EE900A08
:10440000FCF77AF8D5ED037AF8EEE77ACDE9040106
:1044100067EE887A17EE900AFCF76EF8D5ED027A0F
:10442000F8EEE77ACDE9020167EE887A17EE900A96
:10443000FCF762F8074ACDE900010621204649F061
:10444000E5FA304607B0BDEC028BF0BD0AD7233C3D
:1044500095BFD633AC770B087FB500F5805605467F
:1044600096F8E4349A0716D405F593546846083450
:104470000DF062F96946204607F02AFC58B105F5AF
:10448000866009F03BFF96F8E434DB0705D4694603
:10449000204607F00BFB04B070BD04F51B716846A5
:1044A0000DF0DAFBF6EE007AB4EEE70AF1EE10FA60
:1044B000EDD5F0E7F8B500F57856343604463046C9
:1044C0006CF068FD054618B9504B00221A80F8BD03
:1044D00004F5005797F97531002BF5D004F5A0438A
:1044E000D3F8F8050368DB68984720B92046FFF742
:1044F0002DFF0028E8D004F5405393F93831002B04
:1045000042D007EE903A9FED427AF8EEE77A04F552
:10451000805303F58E6267EE877A92ED007AB0EEF3
:10452000C77AB4EEE77AF1EE10FA0CDC03F26C43D2
:1045300093ED007AB0EEC77AB4EEE77AF1EE10FAB6
:10454000CCBF012500252046FFF700FFF0B1002D6C
:10455000BDD047F0B5FA0C21012247F00DFA2046F4
:10456000FFF7F4FE04F5A6434833014600283CD08B
:10457000284A0021184649F049FA30460122BDE890
:10458000F8400C21FDF73EB91D46DCE72DBB04F5D4
:10459000805303F26C629FED207AD2ED007AF4EE44
:1045A000C77AF1EE10FA8FDA03F27C53D3ED027A78
:1045B000F0EEE77AF4EEC77AF1EE10FA84DA07F655
:1045C0007833D3ED0A7AB1EE047AF0EEE77AF4EEBE
:1045D000C77AF1EE10FA3FF577AF0C4A1388013332
:1045E0009BB2132B1380B2D9B3E718460B4A49F09C
:1045F0000DFA04F5B74113225031204604F0AAFE0B
:1046000097F97531022B7FF462AFB6E78086002000
:1046100035FA8E3CCC770B080AD7A33DDD770B0823
:104620002DE9F04D88B0044647F04AFA054674F08B
:10463000ABF904F5C04307461B6904F5BF40B3F16D
:10464000000800F1780018BF4FF001080E4648F04E
:104650008BFD0068FBF750FF824604F5C040043034
:104660008B4648F081FD0068FBF746FFCDE904ABBF
:10467000CDE90601CDE90076054B064A0649CDF89D
:104680000880284646F092FF08B0BDE8F08D00BFD4
:10469000F4770B08F9770B0815780B0873B5044607
:1046A00000F5785034306CF075FC04F5A6454835BB
:1046B00004F5C04640B90023154A3361022128465B
:1046C00049F0A4F902B070BD04F5305069460430D9
:1046D0006EF0ACF80028EED004F5BF4069467830A3
:1046E00048F044FD04F52D53383304F5C0409B6A6F
:1046F000019301A9043048F039FD74F03DF900231D
:10470000306173612046FFF78BFF024AD6E700BF96
:104710001C780B0838780B0870B52DED028B00F56E
:10472000C04686B033690446002B50D03046043072
:1047300048F01AFD90ED008A04F5BF40783048F04B
:1047400013FDB2EE047AD0ED007AB4EEC78A04F518
:10475000A645F1EE10FACDED057A05F148053ADBF4
:104760009FED207AB4EEC78AF1EE10FA33D89FEDB0
:104770001E7AF4EEC77AF1EE10FA2CDBFDEEC87A61
:1047800004F5055017EE903A0DF1130126308DF81F
:1047900013303EF0A5FB04F5055005A918303EF096
:1047A00035FB04F5005292F96631D2F858010393B3
:1047B000FBF7A2FE039B0D4ACDE90001022128462A
:1047C00049F024F9002333612046FFF729FF06B0A2
:1047D000BDEC028B70BD064A0221284649F016F94D
:1047E000F0E700BF0000C8420000003450780B081A
:1047F00073780B087FB500F5C04504462B69002B84
:1048000031D000F5305001A904306EF00FF850B3EC
:1048100004F5BF40154E039603AA01A9783048F06D
:1048200047FD04F52D53383328469B6A029303AAAB
:1048300002A90430039648F03BFD6B690C4A5343D0
:10484000B3F1333F02D82046FFF7EAFE6B6901332C
:104850006B6174F091F82B69C01AB0F5FA6F02D34E
:104860002046FFF759FF04B070BD00BF0AD7A33C34
:10487000CDCCCCCC13B5044600F59350083006F0EF
:1048800073FBD8B101A9134806F02CFE04F578504B
:1048900034306CF07FFB9DF8043088B9DC06C3F33C
:1048A00000100BD49DF805209107C2F3400005D4F9
:1048B0001C07C3F3C00001D402F0010002B010BD18
:1048C000D90603D41A07C3F3C000F7D583F08000DC
:1048D000C009F3E7C838002070B500F50055D5EDE4
:1048E0005E7AF5EEC07AF1EE10FA8AB004464FF027
:1048F000000346D907930893099307AE06AB00F56A
:104900009350019303AA05AB04A90096083007F061
:1049100053F9304620F0DCFFD5ED5E7A9DED047A48
:10492000DDED036AB4EEE70AF1EE10FAF4EEC77AB1
:10493000ACBF01230023F1EE10FAF4EEE67A77EE35
:10494000A76A98BF0133F1EE10FA98BF0133B4EEB5
:10495000E67A98BFDBB2F1EE10FA10DAF4EEC77A1D
:10496000F1EE10FA9CBF0133DBB2012B07D82046D1
:10497000FFF780FF80F00100C0B20AB070BD0120D7
:10498000FBE70020F9E7000070B500F5A0450446FC
:1049900095F810362BBB012685F8106647F090F885
:1049A0003246112146F0E8FFD5F8F80503685B6A46
:1049B0009847B0B104F5005393F976318BB1022BCF
:1049C00006D004F5B74106225031204604F0C2FC5F
:1049D00004F5A640034ABDE870400221483049F082
:1049E00015B870BD112B0B0838B500F5A04304466F
:1049F00093F810268AB1002583F8105647F060F826
:104A00002A46112146F0B8FF04F5A640034ABDE846
:104A100038400221483048F0F9BF38BD8C780B0887
:104A2000F0B585B0054668460CF086FE05F5935056
:104A30006946083007F090F9D8B105F57850343060
:104A40006CF0A8FA344C354E40B105F50053D3ED67
:104A50005E7AF5EEC07AF1EE10FA0CD8238823F4D2
:104A6000FF7323F00103238028460023F373FFF72D
:104A7000BBFF05B0F0BD2846FFF72EFF074688B301
:104A80006378DB0705D423780133DBB2092B05D823
:104A90002370637803F00103F373EAE7238823F4B8
:104AA000FF7323F0010343F48573238047F008F874
:104AB0000222102146F060FF73F05EFF6368C01AA7
:104AC00047F23053984209D905F5A640144A02210D
:104AD000483048F09BFF73F04FFF60602846FFF7B7
:104AE00053FFD6E72378002BD3D0013B23702388D4
:104AF000C3F30803B3F5807FCBD1637860F3000381
:104B0000637046F0DDFF3A46102146F035FF284637
:104B1000FFF76AFFBDE700BF848600203D870020C5
:104B2000A4780B0810B5044673F01AFF0E4AB4F8C7
:104B3000BE1013888B420D4B02D01180186010BD3F
:104B40001B68C01A0A4B9842F9D904F578543434DA
:104B500020466CF01FFA0028F1D020460122BDE863
:104B600010400621FCF74EBE8C8600209086002067
:104B7000400D03002DE9F84F00F5A045914604468D
:104B800095F800260E46002B71D042EA010385F805
:104B9000003622B91BB173F0EFFEC5F8040695F894
:104BA000083653B195F800363BB904F5A6404B4A98
:104BB0004B460621483048F029FF95F8083695F80D
:104BC0000026134085F80836002B40F08580002A27
:104BD00000F0828073F0D0FED5F80436DFED406A35
:104BE000C01A04F5005A07EE900A9AED5B7AF8EEC7
:104BF000677A27EE267AF4EEC77AF1EE10FA6BDDCB
:104C0000D5F8F83504F5BE4808F14008434563D0AF
:104C100004F5B7475037BB4205D104F54053D3F8EC
:104C20003C3BDB0758D504F5A64B95F800362D4ADA
:104C300085F808360BF1480B4B460421584648F0DE
:104C4000E5FE50F043FFD5F8F82504F5B94370337D
:104C50009A4214D1012E0DD19AF97031022B0ED146
:104C60005846214ABDE8F84F042148F0CFBE22EA59
:104C700001038CE7022E02D19AF97431EEE79AF91A
:104C80006831013B042B27D8DFE803F00B11031830
:104C90001D0004F5BE4119227C31204604F05AFB68
:104CA000D0B919224146204604F054FBA0B9394638
:104CB00020461922BDE8F84F04F04CBB04F5BE4174
:104CC00019227C31EFE704F578500122BDE8F84F56
:104CD00014213430FCF796BDBDE8F88FB4780B088A
:104CE00000007A44C8780B08D4780B08013A10B554
:104CF0000446042A2AD8DFE802F00A12031B200027
:104D000000F5BE4104227C3104F024FBF0B904F527
:104D1000BE4104224031204604F01CFBB0B904F52A
:104D2000B74120460422BDE81040503104F012BBC8
:104D300000F5BE4104227C31EDE700F57850BDE876
:104D40001040012207213430FCF75CBD10BD00008B
:104D50002DE9F84300F5015700F5005808370446DF
:104D60000021384698F884905AF044FC04F57856AF
:104D70003436054630466CF00DF9002846D0002D3B
:104D800041D098F94E305BB3294638465AF098FC2A
:104D9000DFED1F7AB4EEE70AF1EE10FA19D898F9B0
:104DA0004E30013B042B1BD8DFE803F00B1303222A
:104DB000270004F5BE410A227C31204604F0CAFADD
:104DC00070B904F5BE410A224031204604F0C2FA0F
:104DD00030B904F5B7410A225031204604F0BAFA3E
:104DE00046F06EFE2A460921BDE8F84346F0C4BDF0
:104DF00004F5BE410A227C31E7E701220F2130464B
:104E0000FCF700FDECE7B9F1000FE9D1BDE8F8834C
:104E10000000C84201207047002070470120704701
:104E20000120704710B50368DB680446984748B115
:104E3000E368DFED067A03F5C75393ED040A20EE2D
:104E4000270A10BD9FED020AFBE700BF0AD7233CEB
:104E50000000000010B50368DB680446984748B1BD
:104E6000E368DFED067A03F5C75393ED030A20EEFE
:104E7000270A10BD9FED020AFBE700BF0AD7233CBB
:104E80000000000010B50368DB680446984728B1AD
:104E9000E36803F5C75393ED050A10BD9FED010AC2
:104EA000FBE700BF0000000010B50368DB680446A4
:104EB000984728B1E36803F5C75393ED020A10BD84
:104EC0009FED010AFBE700BF0000000010B503687A
:104ED000DB680446984738B1E06800F5CB50BDE880
:104EE0001040083003F0D4BE10BD000070B52DEDA9
:104EF000028B5A4D84B0D5ED460A8DED010A044669
:104F0000806A0E466DF088FE8DED010A7EB3E06882
:104F100000F57766A06A6DF053FE6368D5ED461A1A
:104F200093ED831AF6EE000A60EE200A30469FEDFC
:104F30004C0A01A95DF0E2FAE06800F5CB500830B8
:104F400003F03AFE98B1E66873F016FDD6F8983F84
:104F5000C01AB0F5FA7F0AD205F5A043D3F8F805D8
:104F600003F54463984202D003685B6D9847E0689C
:104F70009DED010A0023039300F5805393F96839EE
:104F8000002B10DD00F5CB5003A9083003F0EEFF35
:104F9000E0689DED030A00F51F6071F015FC04B098
:104FA000BDEC028B70BDDFED2F7ADFED2F8A9FED18
:104FB0002F8AB0EEC00AB4EEE70AF1EE10FA1FD461
:104FC000E368A06A93F8F0395A0745D490F844137F
:104FD000D5ED461A9DED010A1B07A36858BF90F84E
:104FE000442393F91E60D3ED040A01EE106AB8EE73
:104FF000C11A48BF012221EE281A6DF069FE1DE09A
:105000001648FFF7A3F90028DAD1A268E36892ED09
:10501000040A93F8F01992F91E3095ED461AA06A29
:1050200007EE903AF8EEE77AC1F3C00267EEA80AFD
:105030000DF10B03C1F380016DF0F8FE20EE080ABC
:1050400006488DED030AFFF781F90028A0D0034838
:1050500003A9FFF745F99BE70121B9E76026002086
:1050600000000000000000340AD7233C0000C842C2
:105070000C4A02600C4A426002F56E6102F57262EF
:10508000C2600A4A0261043242610432826104321F
:10509000C2610432026204324262A2F58E52816021
:1050A00082627047FC780B08C8380020106400202A
:1050B0000368DB6D1847000037B51D4B1B68DB6AC2
:1050C00093F89C3004460BB301A91A4806F00AFA7B
:1050D0001948FFF7CFFB054620B1184B93F810563F
:1050E00085F00105236820465B6A984700B14DB101
:1050F000236820469B6A984740B13DB99DF804302B
:105100009B0703D40025284603B030BD2368204602
:105110009B6D984705460028F5D0236820461B6DF7
:105120009847E06800F5CB50083003F0C3FCEAE78D
:1051300058260020C8380020602600206076002015
:1051400070B52DED028B2F4C94F80036DB070D4621
:10515000164605D500230B601360BDEC028B70BDB5
:10516000836893F91F30012BA4F5005420D0032B42
:10517000D4F8B43DB3F9083007EE903AF8EEE77A88
:10518000C2ED007A35D0002BD4F8B03DB3F9083029
:10519000FFEE007AB7EE007AB8BFB0EE677A07EE9E
:1051A000903AF8EEE77A67EE877AC5ED007AD4E7B1
:1051B000D4F8B00D50F08CFED4F8B40DB0EE408AA7
:1051C00050F086FE78EE007AB6EE007A67EE877AC7
:1051D000DFED0D6A38EE408A67EEA67A28EE078A80
:1051E000C6ED007ADFED097A28EE278A85ED008A80
:1051F000B3E7D4F8B03DB3F9083007EE903AF8EED3
:10520000E77AD2E7607600200000C84200A08C4513
:1052100070B506462DED028B0D461446FFF790FF44
:10522000F06800F51F6071F071FBA0B3DFED317A1B
:1052300095ED000A722080EE270AB7EE001AFFEE05
:10524000000A1DF027F8DFED2C7AB0EE408A94EDCD
:10525000000A732020EE270AB7EE001AFFEE000ABC
:105260001DF018F8B0EEC88AB0EEC00A38EE000A99
:10527000F7EE007AB4EEE70AF1EE10FA0BDD95EDE9
:10528000007AC7EE007AC5ED007A94ED007AC7EE99
:10529000007AC4ED007A194BF068D3ED460A94ED1C
:1052A000000A00F51F6071F019FBDFED157A94ED2F
:1052B000007AB4EEE77AF1EE10FAB4EEE70A94BFA2
:1052C00001220022F1EE10FA94BF012300239A423A
:1052D0000BD0B36893F91F3033F0020302BFD5ED52
:1052E000007AF1EE677AC5ED007ABDEC028B84EDB1
:1052F000000A70BD00A08C450AD7233C6026002020
:10530000000000B40A4B93F80026D2070DD4A3F591
:105310000053D3F8B83D43B1B3F9083007EE903AE3
:10532000F8EEE77AC1ED007A7047DFED027AF9E72F
:10533000607600200000000070B5C369054618685B
:105340000E46144658B150F083FD86ED000A2B6AD4
:10535000186838B150F07CFD84ED000A70BD002360
:105360000B60F4E700232360F8E7000010B5436A00
:1053700018680C4620B150F06BFD84ED000A10BD9A
:1053800000230B60FBE70000C36851B103F66872AD
:1053900092ED000ADFED057AB4EEE70AF1EE10FABD
:1053A00003DA03F5805393ED500A70470000003490
:1053B000C36803F5805383F8CD18704730B52DEDE1
:1053C000028B3C4D9FED3C8A83B000230446284667
:1053D0008DF80330FEF7BAFFD4E90223DFED370A78
:1053E00093F8F01992F91E30002848D001EE103AD7
:1053F000B8EEC11AA06AD5ED461A9FED310A21EE2A
:10540000201AD2ED040AC1F3C002C1F380016DF08D
:105410005FFC20EE080A01A928468DED010AFEF77F
:105420005FFFE06800F5CB50083003F0A3FAE068B6
:105430009DED010A00F51F6071F0C6F99DF803307B
:10544000ABBBE368D5ED460A93F8F0199FED1C0A53
:10545000A06AC1F3400201F001016DF06DFAE0684D
:10546000DFED187A012120EE270A00F51F6071F0A8
:10547000A5F99DF8030003B0BDEC028B30BD07EE2B
:10548000903AF8EEE77A92ED040A95ED461AA06A92
:10549000C1F3C00267EEA00A0DF10303C1F380015E
:1054A0006DF0C4FC20EE080A8DED010AB9E79FED0E
:1054B000040AD4E7602600200000C8420AD7233C33
:1054C0000000000000A08C45B7EE007AF4EEC70A99
:1054D000F1EE10FA18DCDFED107AF4EEE70AF1EEE7
:1054E00010FA11D4C368DFED0D6A03F5CD53D3ED87
:1054F000037AF4EEE67AF1EE10FAB6BFC7EE207A40
:10550000B0EE670A20EE270ADFED050A40F27D10B3
:10551000B3EE0E1A1CF0BEBECDCC4C3D00000034E4
:105520000000000070B52DED028B044682B01546D8
:1055300001AA0E46FFF704FEA3689DED010A93F948
:105540001E20DFED200A07EE902AF8EEE77A20EE23
:10555000208A204667EEA00A93ED040AFFF7B4FF05
:1055600028EE000A184B85ED000AE068D3ED460AE4
:1055700000F67C206DF050FBDFED147A95ED007A9B
:10558000B4EEE77AF1EE10FAB4EEE70A94BF012226
:105590000022F1EE10FA94BF012300239A420BD0AF
:1055A000A36893F91F3033F0020302BFD6ED007AEF
:1055B000F1EE677AC6ED007A85ED000A02B0BDEC27
:1055C000028B70BD0AD7233C60260020000000B487
:1055D000F8B5324F2DED028B0446D7F8B00D0E46CC
:1055E000154650F075FCB7EE001AFFEE000AA62033
:1055F0001CF050FED7F8B40DB0EE408A50F068FCB5
:10560000A720B7EE001AFFEE000A1CF043FEA368C5
:1056100093F91F30012BF0EE408A09D178EE008A11
:1056200038EE407AF6EE007A68EEA78A27EE278AEF
:10563000F0EE680AB0EE480A96F02AFEDFED187A1E
:1056400020EE270A1CF0BAFD86ED000A28EE080AB3
:10565000A8EEA80A1CF04EFDA368DFED120A93F92C
:105660001E20F7EE007AB4EEE70AB0EE408AF1EEC3
:1056700010FA58BFB0EE678A07EE902AF8EEE77A84
:1056800093ED040A67EEA00A2046FFF71DFF20EE07
:10569000080ABDEC028B85ED000AF8BD60560020BB
:1056A000A00CB3450AD7233C30B52DED028B83689F
:1056B0009B7F053B5F2B83B00546F0EE408A0C468E
:1056C00021D801AA6946FFF73BFDAB68DFED200A50
:1056D00093F91E209DED018A93ED040A07EE902AAE
:1056E000F8EEE77A28EE208A284667EEA00AFFF750
:1056F000EBFEDFED187A28EE000AB4EEE70AF1EED1
:1057000010FA03DBE4B1B0EE680A0DE0DFED127AC7
:10571000B4EEE70AF1EE10FA0AD8002CF3D0B4EE9A
:10572000E80AF1EE10FAEEDC03B0BDEC028B30BDFE
:10573000002CF4D1B4EEE80AF1EE10FAE3D4F3E76A
:10574000DFED057AB4EEE70AF1EE10FAF2D8DAE707
:105750000AD7233C00000034000000B410B52DED42
:10576000028B0368DB680446B0EE408A9847A8B114
:10577000E36803F5805393F93831002B0EDDBDEE5D
:10578000C80A10EE103A1BB200EE103A2369B8EEC8
:10579000C00A186850F0D0FCB0EE408AB0EE480A5B
:1057A000BDEC028BE0680121BDE8104000F51F60F0
:1057B00071F004B810B5C36893F8F019094B0446AA
:1057C000C1F34002806AD3ED460A01F001016DF099
:1057D000B3F8DFED057A204620EE270ABDE8104039
:1057E000FFF7BCBF6026002000A08C4510B59FEDE0
:1057F000107AC368DFED0F7A93F8F0190E4B20EEA4
:10580000070A044660EEA70A20EE270A806A93ED95
:10581000461AC1F3400201F001016DF08DF9DFED90
:10582000077A204620EE270ABDE81040FFF796BF12
:105830000AD7233C35FA8E3C6026002000A08C4518
:1058400010B5836ADFED157A93EDB91AB4EEE71A55
:10585000F1EE10FAD8BFB0EE671ADFED117A21EE43
:10586000271A0446F1EE410A4FF4F2701CF012FDC3
:10587000E368A06A93F8F0190A4BC1F34002D3ED34
:10588000460A01F001016DF06FF9DFED077A20465D
:1058900020EE270ABDE81040FFF760BFCDCCCC3D1D
:1058A0000AE81C416026002000A08C45102938D849
:1058B000DFE801F0090D37111519371D37202428AD
:1058C0002B37372F330000F5B8400830704700F50C
:1058D000B8404030704700F5BE400430704700F5D6
:1058E000B7405030704700F5BD403830704700F584
:1058F000BF40FAE700F574501030704700F5B9402A
:105900007030704700F5BE40E3E700F5BE407C30E4
:10591000704700F5B8407830704700F5B740183050
:10592000704700207047000082B073B50E4606A98C
:1059300081E80C00C5680446DDE908018DE8030034
:1059400006AB05F589500CCB31461C306EF0F6FDE8
:1059500040B1E36803F5C75318331B68E3620023C3
:1059600084F8303002B0BDE8704002B070470000EB
:1059700070B52DED028BC368554D03F5805303F6CA
:10598000D40293F8CD1892ED000A0029B7EE007A00
:10599000FFEE007A08BFF0EE477A044682B027EEA9
:1059A000800AFFF781FEE06841F23C16B0EEC00AC3
:1059B00030446DF037FFE06895ED460A30446EF0F4
:1059C000BBFDE06800F5C753183300F5CB501B68EA
:1059D000E362083003F0F0F878B1E66872F0CCFFCB
:1059E000D6F8983FC01AB0F5FA7F06D205F5A04563
:1059F000D5F8F80503685B6D9847E368226803F5FE
:105A0000C753126E93ED000A002120469047E068CC
:105A100000F589501C306EF083FDE06841F6681691
:105A20003044B0EE408A03F047F9E56808B3A8199E
:105A3000B0EE480A03F074F9E0688DED010A3044D5
:105A400003F032F99DED010A80B1E36803F580535C
:105A5000B3F94A3100EE903AF8EEE00A204602B07F
:105A6000BDEC028BBDE87040FFF7C0BEDFED190A48
:105A7000F4E705F5C75393ED018A72F07DFFD5F881
:105A8000983FC01AB0F5FA7F17D2A06A6DF0B6F849
:105A9000A36AD3EDB67AF5EEC07AF1EE10FAD8BF6C
:105AA000DFED0C7AB0EEC00AB4EE670ADFED097ADA
:105AB000F1EE10FA98BFB0EE678AB0EE480A2046C1
:105AC00002B0BDEC028BBDE87040FFF773BE00BFB3
:105AD0006026002000000000012070470048704749
:105AE00060790B080120704700207047F0B52DED5C
:105AF000028B85B001A90446806A3D4D6CF096FE8C
:105B000003AA02A900284DD12046FFF781FB2846B1
:105B1000FEF71CFC18B103A92846FEF7E1FBE0687C
:105B20009DED030A00F51F6070F04EFEDDED027A78
:105B30009FED307AF0EEE77AF4EEC77AF1EE10FAE4
:105B400005D4E06800F5CB50083002F0B3FFE06800
:105B50009FED298A41F66816304403F0A5F8E36802
:105B600058B39819A76A02F0B1FFE36895ED461A99
:105B700093F8F01903F58053C1F34002B3F94A31A9
:105B800000EE903A01F00101F8EEE00A38466CF0C0
:105B9000D3FF20EE080A2046FFF7E0FD05B0BDEC7C
:105BA000028BF0BD2046FFF7BDFC23689DED030A84
:105BB0001B6E012120469847B8E7DDED027A93F885
:105BC000F0199FED0E7AD5ED460AA06A87EE880A95
:105BD00003F6B463C1F3400201F00101D3ED007A92
:105BE00067EE877A20EE270A6CF0A6FED1E700BFA9
:105BF000602600200000003400A08C4535FA8E3C61
:105C000008B5C06800F51F6070F080FE80F00100EC
:105C1000C0B208BDC06800F5CB50083003F00CB826
:105C20000A20704700487047D4790B08012070475C
:105C300090F8300100F0FD00031F584258417047B2
:105C400090F83C30012B02D138301FF089BF7047EB
:105C500090F9702022B190F8711009B9FFF7A8BB34
:105C60007047000010B504460348FFF725FA10B14D
:105C7000022384F8303110BDA085002030B52DED11
:105C8000028B90F8324183B00546002C39D1AB68C5
:105C900093F915104A1C52D1D3ED067A9FED307A54
:105CA000F0EEE77AF4EEC77AF1EE10FA53D4AB686F
:105CB0009FED2B7AD3ED067AF0EEE76AF4EEC76A31
:105CC000F1EE10FA49D4274B93F8AB2B0C2103F6D5
:105CD000980301FB023393ED628AF4EEC87AF1EE89
:105CE00010FA3AD84EF03EFD044618EE100AFAF7C4
:105CF00003FC1D4ACDE900010421204647F086FE41
:105D000029E0836893F915104B1C13D01548C9B2CC
:105D100003F09CFC012809D14EF024FD134A042114
:105D200047F074FE002485F8324103E095F83231E3
:105D3000002BACD0204603B0BDEC028B30BD09482F
:105D4000C9B203F083FC0028B1D14EF00BFD084A24
:105D5000042147F05BFE0124E5E70024EAE700BFE9
:105D60000000003460260020077A0B08DC790B085D
:105D7000EF790B0810B504460348FFF79DF910B101
:105D8000032384F8303110BD1885002010B5B0F819
:105D90006C30012B044607D84EF0E4FC114A052173
:105DA00047F034FE002010BDC0689FED0F0A00F5DB
:105DB00089501C306EF044FA00230C4884F83231CC
:105DC00001F052FB0A4803F05DFC18B12046FFF7D2
:105DD000D1FF10B9052384F83031012084F8310156
:105DE000E1E700BF247A0B0800000000D882002001
:105DF0006026002070B505460E480C46FFF75CF99A
:105E0000B0B1042385F830310A4801F033FBA368B0
:105E10000BB9E36853B194E80F0005F5A27686E864
:105E20000F00054930460BF069FD012385F8543118
:105E300070BD00BFD8820020C47B00201FB590F841
:105E4000543104462BB372F097FDD4F858311BB18E
:105E5000C31AB3F57A7F1CD90DF10F03C4F85801AA
:105E600000930D480DF10E030DF10D02122149F0C2
:105E700007FD70B14EF076FC03689DF80F101B69AA
:105E800098479DF80E209DF80D1004F5A2734DF073
:105E9000EBFA04B010BD00BFF189002010B5144A20
:105EA0001378044643F0800313704EF05BFC114AF4
:105EB000052147F0ABFDE36803F5805393F93031DA
:105EC000022B0BD0032B0FD0012B03D12046FFF761
:105ED00051FF10B9052384F8303110BD064908225E
:105EE000064803F037FAF4E705490822F8E700BF4F
:105EF0005C870020407A0B08A082002060260020EA
:105F0000688200202DE9F04701F108030446884625
:105F100091460FCB92B003AE86E80F00274930467A
:105F20000BF0ECFCB8F9043023EAE372A4F83A2150
:105F3000002293420DAFC4F83C21C8BF4FF00109C5
:105F400038460BF0F9FB07AD0DF1240AB9F1000F4B
:105F500015D0236828465F6C0BF0EEFB9AE803002F
:105F60008DE80300314695E80C002046B84718B18B
:105F7000002384F84031012012B0BDE8F087B8F862
:105F8000001001310BAA89B204F1380021F008FE9B
:105F90000028DED097E80F0085E80F00314628463C
:105FA0000BF0ACFC9AE803008DE80300276895E845
:105FB0000C0031467D6C2046A847D8E7C47B002002
:105FC00037B504460D4672F0D7FCC4F868011C488A
:105FD00003F058FB18B12046FFF7CCFE10B905239B
:105FE00084F83031D5ED027AF5EEC07AF1EE10FA90
:105FF00016DD9FED147A67EE877AFCEEE77AC4ED42
:10600000597A4EF0AFFBD4F864214FF47A73B2FBA7
:10601000F3F30D4A062103B0BDE8304047F0F6BC6B
:1060200058F00CFE0023009395F90D2095F90E30E1
:1060300095F90C1058F09EFDC4F86401E1E700BF2B
:106040006026002000007A44547A0B088B8813B134
:106050000831FFF7CFBE704738B59FED180A0B7CAB
:106060002DED028B91ED028A044628EE008A0D4642
:1060700053B1436893ED800AB8EEC00A30EE080AC7
:106080001CF0B2F8B0EE408AE36895ED030A03F520
:10609000805393ED501A40F22F30F1EE410A1CF07C
:1060A000F9F884ED0D8ABDEC028B002384F83831B9
:1060B000012384ED4D0A84F8303138BD0000C84218
:1060C00073B503689B6C05460E469847044640B37B
:1060D00095F840319BB9B5F83A31012285F8402155
:1060E00013B34EF03FFBB5F83A31134A0093062143
:1060F000338847F08BFC72F03FFCC5F83C01B5F8E3
:106100003A3173B172F038FCD5F83C41041B4FF4BE
:106110007A70B4FBF0F4B5F83A01844234BF00243D
:106120000124204602B070BD4EF01CFB3388034AA8
:10613000062147F06BFCE2E7647A0B08907A0B08C3
:1061400010B5044672F018FCD4F86831C01AD4F8BF
:10615000643198424FF0000084BFC4F8640101200C
:1061600010BD000003689B6C1847000010B5FFF7D6
:10617000A7FF044628B14EF0F5FA034A042147F080
:1061800045FC204610BD00BFA87A0B0810B590F85A
:106190003031042B044618D18B88B3B190F85431B8
:1061A00023B9BDE810400A4801F072B900F5A271A8
:1061B00008480BF051FDE36803F58053D3ED517AA5
:1061C000B4EEE70AF1EE10FAEBD8012010BD00BFE3
:1061D000D8820020C47B00207FB501F108030C4663
:1061E00006460FCB6D4685E80F00124928460BF096
:1061F00085FB6288A388122A4FEA132305D1227EE9
:10620000D20744BF03EB83035B00F068227A07EEFA
:10621000903A00F5DC50B8EE670AC2F34002294616
:10622000083000F02DFF10B1072386F8303104B09C
:1062300070BD00BFC47B00200B799FED0F6A07EE95
:10624000903A0B7E9B07C36848BF9FED0C7AF8EE2F
:10625000677A03F5DC5348BF67EE877A93ED247ABB
:10626000B0EEC77AC7EE066AF4EEE76AF1EE10FA0E
:10627000ACBF012000207047DB0FC9400000803B0D
:1062800038B504460D4672F077FBC4F86001D5EDD1
:10629000027A9FED047A67EE877AFDEEE77AC4ED25
:1062A000577A38BD00007A4410B5044672F064FB9A
:1062B000D4F86031C01AD4F85C3198424FF0000035
:1062C00084BFC4F85C01012010BD000010B5036854
:1062D0000446DB6B9847D4ED577AF8EEE77A002056
:1062E000B4EEE70AF1EE10FA44BFC4F85C010120F5
:1062F00010BD000010B54B885C2B02460C4671D0D7
:1063000041D8103B99B2042936D94EF02BFA638854
:106310003E4A042147F07AFB47E0C23B132BF4D8F6
:1063200001A151F823F000BFAB630108AB63010882
:106330000B630108AB6301080B6301080B630108E1
:106340000B630108AB6301080B6301080B630108D1
:106350000B6301080B630108AB630108AB63010821
:106360000B6301080B6301080B6301080B63010851
:106370000B630108FD630108042BC6D8DFE803F0B6
:106380001A23282D1F00722B34D007D85D2B2DD057
:10639000702BBAD1BDE81040FFF786BFD52B06D8C9
:1063A000C12BBAD8B23B012BAFD801200FE0DE2BB6
:1063B000FBD0AAE72146BDE81040FFF781BEBDE84B
:1063C0001040FFF7CFBE2146FFF77AFE002010BD38
:1063D0002146BDE81040FFF72FBF2146BDE8104021
:1063E000FFF7C4BEBDE81040FFF7D0BEBDE81040C7
:1063F000FFF7A6BEBDE81040FFF768BF92F8303146
:10640000012BD2D192F83801E1E700BFC07A0B0826
:1064100038B50D46FFF76EFF044620B14EF0A2F9E5
:1064200029884BF049FC204638BD000037B5036889
:10643000D1F80920DB6C00EE102A0C46984768B1B1
:106440004EF090F90546D4F80900FAF755F8044AD9
:10645000CDE900010621284647F0D8FA03B030BD47
:10646000DC7A0B0889884B1E59425941FEF7A0BFC0
:106470008B8891ED040A03484FF47A71594300F078
:10648000EFBF00BFD882002030B5684B1B68DB6AC5
:1064900093F89C3085B0044633B9B0F86C30012BCA
:1064A0009CBF052380F8303194F83131E3B1684660
:1064B0000BF042F96068694605F04EFC50B104F1FA
:1064C000380021F061FF002384F8313104F5B67003
:1064D0001FF0DEFA94F83031072B43D8DFE803F0E1
:1064E0002444878D9381969C04F5B6701FF0D0FAF2
:1064F00004F1380580B194F83C30012B0CD194F8AC
:1065000030314BB9284621F0ADFD48B14EF02AF9A3
:10651000474A022147F07AFA284621F0D1FDD9E70F
:106520004EF020F9434AF4E7434803F0ABF828B9AA
:10653000204605B0BDE83040FFF71ABAE06800F524
:1065400089501C306DF0D0FF0028F1D0E36803F5CE
:10655000805393F88C38002BEAD12046FFF70AFCD1
:106560000028E5D005B030BD94F8383183BBDFEDAD
:10657000330A94ED0D0A2046FFF738F9DFED307A43
:1065800094ED4D0A2368B4EEE70AF1EE10FA94BFD9
:106590000121002120461D6EFFF786F801212046CB
:1065A000A8476368D4ED0D7A93ED807AB8EEC77A88
:1065B00077EEC77A9FED237AF0EEE77AF4EEC77AAA
:1065C000F1EE10FA4CBF0123002384F83831C9E7FB
:1065D000194803F057F820B12046FFF7CBFB0028FD
:1065E000C0D1204605B0BDE83040FEF7E7BE1648F2
:1065F00005B0BDE8304001F083BB144805B0BDE8EC
:10660000304001F069B92046FFF718FC104805B08A
:10661000BDE8304000F07CBFE06800F5DC50083099
:1066200005B0BDE8304000F0E7BB00BF58260020B1
:10663000EC7A0B08147B0B08602600200000000099
:10664000000000B40000FA43A08500201885002057
:10665000D882002013B504468DED010A0091FFF7A2
:106660000DFB00999DED010A28B9204602B0BDE856
:106670001040FEF7A3BE204602B0BDE81040FEF772
:1066800035BC000090F83031072B1FD8DFE803F04D
:10669000041E0E11151E1518C36803F5C75393ED9C
:1066A000040ADFED0C7A20EE270A70470A48FEF74D
:1066B000B9BB0A4B93ED000AF3E7094800F0E8BDC7
:1066C000C06800F5DC50083000F018BA9FED050AEC
:1066D000704700BF0AD7233CA08500204C850020CE
:1066E000D88200200000000090F83031072B1FD81E
:1066F000DFE803F0041E0E11151E1518C36803F51C
:10670000C75393ED030ADFED0C7A20EE270A70479A
:106710000A48FEF79FBB0A4B93ED000AF3E70948CE
:1067200000F0D2BDC06800F5DC50083000F0B8B908
:106730009FED050A704700BF0AD7233CA0850020C3
:106740004C850020D88200200000000090F83031F5
:10675000072B17D8DFE803F004160A160D160D10E4
:10676000C36803F5C75393ED050A70470748FEF762
:1067700089BB074800F0C4BDC36803F5DC5393ED43
:10678000260A70479FED030A704700BFA0850020CE
:10679000D88200200000000090F83031072B19D873
:1067A000DFE803F004180A0D0F180F12C36803F591
:1067B000C75393ED020A70470848FEF775BB0848B7
:1067C000FBE7084800F0A4BFC06800F5DC500830C3
:1067D00000F048B99FED040A704700BFA085002073
:1067E00018850020D88200200000000090F8303189
:1067F000072B17D8DFE803F00416070B0D160D1052
:1068000090ED0B0A7047094B93ED000A7047084B57
:10681000FAE7084800F082BDC36803F5DC5393ED46
:106820000D0A70479FED040A704700BFCC85002019
:1068300044850020D88200200000000038B590F880
:1068400030310C46072B2CD8DFE803F0042B141949
:106850001E2B1E23C06800F5805393F8CC583DB121
:1068600000F589501C306DF051FE0FC884E80F0010
:10687000284638BDBDE838400B4801F083BABDE872
:1068800038400A4801F020B8BDE83840084800F018
:1068900055BFC06800F5DC50BDE83840083000F056
:1068A000E7B80025E4E700BFA08500201885002098
:1068B000D882002082B037B50D4606A981E80C00C9
:1068C0000446DDE908018DE8030006AB0CCB294640
:1068D0002046FFF729F810B1002384F8303103B0C7
:1068E000BDE8304002B0704790F83031062B11D827
:1068F000DFE803F004100A100D100D00C06800F569
:1069000089501C306DF0F0BD034801F0F3B9034825
:1069100000F0F2BD01207047A0850020D882002041
:1069200090F83031072B1BD8DFE803F0040A0E1A69
:1069300011041114C06800F589501C306CF062BF5E
:1069400080ED4D0A01207047064801F089B90648DC
:1069500000F0F8BCC06800F5DC50083000F042BB25
:1069600000207047A0850020D88200208B88012B52
:1069700008D1074890F8143623B10021A0F5A040B3
:10698000FDF7ECBC034800220831FDF70DBD00BF48
:10699000607600206026002038B54B88702B0446B6
:1069A0000D4642D010D8142B08D80F2B0AD9113B12
:1069B000032B20D8DFE803F02A2C2A265C2B2BD0CF
:1069C0005D2B2FD0002020E0C22B37D00CD8B22B6B
:1069D0002ED0B32B2FD0722BF4D1D1ED027AFDEE55
:1069E000E77AC0ED577A0FE0D52B18D0DE2BE9D12E
:1069F000FFF73EFD08E0002229462046BDE838406A
:106A0000FFF780BAFFF72EF9012038BD0122F3E726
:106A1000BDE83840FFF7E0BBFFF718FBF4E7FFF7EE
:106A20001BFBF1E7FFF7CCFAEEE7FFF729FCEBE7FA
:106A3000FFF7FCFCE8E7FFF799FFE5E7FFF712FD3A
:106A4000E2E700000920704700487047E5640B0842
:106A50000120704790ED240A7047000090ED0B0A6A
:106A600070470000C36803F5CD5393ED740A704777
:106A700038B500F1440305460C460FCB84E80F00FF
:106A8000DFED067A95ED1B0AD5ED170A204620EEBC
:106A9000270A0BF057F9012038BD00BFE02E6542F0
:106AA00007B5C06800F5CD5018306CF07DFBDFED08
:106AB000107A8DED000AB0EEC00AB4EEE70AF1EEEE
:106AC00010FACDED010A06D5F0EEE00AF4EEE70A81
:106AD000F1EE10FA09D468461DF0C2FFDFED057A29
:106AE00020EE270A03B05DF804FB9FED030AF9E7E7
:106AF00000000034E02E65420000000010B586B0B2
:106B0000002304460093019305F020FB694604F03E
:106B10007FFA18B99FED130A06B010BD636F226F9C
:106B20000492694604A805931DF028FFDFED0E7A54
:106B30008DED020AB0EEC00AB4EEE70AF1EE10FAEB
:106B4000CDED030A06D5F0EEE00AF4EEE70AF1EE29
:106B500010FADFD402A81DF083FFDFED047A20EEE7
:106B6000270AD9E70000000000000034E02E65424B
:106B700010B50446FEF77CFA20460B4B40F8443B28
:106B80000AF0DAFD0023204608496365A365236700
:106B90006367A367E367C4F88030C4F884303BF0D0
:106BA0005BFB204610BD00BF7C7C0B08347C0B08CF
:106BB0001FB5002304460093019305F0C7FA694608
:106BC00004F026FA30B905F0C1FAD0F80C32E366C9
:106BD00004B010BD04F1540168461DF0CFFE02A8B8
:106BE0008DED020ACDED030A1DF084FFDFED077A7B
:106BF000B0EEC00AB4EEE70AF1EE10FAE3D402A850
:106C00001DF02EFF84ED1B0AE2E700BF00000034F8
:106C100013B5D0ED170AC3689FED217A90ED1B0ADA
:106C2000426DF6EE007AF4EEE70ADFED1E7AF1EE41
:106C300010FA03F56B63B8BFF0EE477A93ED007A74
:106C400090F88C300267B4EE677AF1EE10FAC8BFA4
:106C5000F0EE477A90ED247AB4EEE77AF1EE10FA8E
:106C600098BF43F00103DFED107A80F88C3000F11B
:106C70007001836D4367044620EE270A08460191A0
:106C80001DF0DEFFE068094B019993ED460A00F51F
:106C9000CD50183002B0BDE810406CF047BA00BFCC
:106CA000CDCCCC3DCDCC4C3EE02E654260260020C4
:106CB00030B52DED048BC3684B4D90ED180A03F5EC
:106CC000CD5393ED611AF6EE007A21EE271AD5ED39
:106CD000467A21EE271AD0ED1A7A044630EE670A7A
:106CE00085B0D320F1EE410A1BF0D4FAD4ED1A7A24
:106CF00094F8943070EE277AF0EE408AC4ED1A7A58
:106D0000002B6CD1DFED396A94ED177A636E95ED47
:106D1000469A94ED1B0A27EE267A002B87EE878A87
:106D2000BFEE007A28EE268AF7EE007A18BFF0EE62
:106D3000477A28EE278AA9EE080A1BF097FAD4EDC5
:106D4000227A84ED1B0AE9EE087AC4ED227A94EDEA
:106D50001B0ADFED277AA36D626DD4ED170A226757
:106D600004F17001084620EE270A636703911DF0C5
:106D700067FFA36E94ED1B0ADFED1E7AA36704F193
:106D800078020023104630EE270AE36702921DF0D6
:106D90007DFFD4ED1A7AD5ED466A94ED176A94ED2D
:106DA0001B0A67EEE77A88EEA67A04F1800318469C
:106DB0000193C7EE866A84ED217AC4ED206A1DF046
:106DC00065FFE0680399DDE9013200F5CD50183028
:106DD00005B0BDEC048BBDE830406CF0B5B9204681
:106DE000FFF7E6FEB3E700BF60260020DB0FC940D7
:106DF000E02E6542DB0FC93F30B52DED028B8BB025
:106E0000002304460293039305F0A0F902A904F0BD
:106E1000FFF830B92046FEF7D1FA0BB0BDEC028B7B
:106E200030BD04F1540102A81DF0A8FD636F226F6C
:106E3000079302A906A8CDED050A06928DED040A76
:106E40001DF09CFD08A8CDED090A8DED080A1DF086
:106E500051FE04A884ED0B0A1DF04CFED4ED177A08
:106E600094F88C3030EE670AB0EEC00A84ED240A44
:106E7000EBB92046FFF7CCFEE068344B00F5CD506F
:106E800093ED460A18306CF0C3FAE36803F5CD536E
:106E900093ED730A93ED728A2046FEF78BFC23680C
:106EA00001211B6EB0EE480A20469847B5E7B6EEC2
:106EB000007AE368F4EEC77A9FED257ADFED257A54
:106EC000F1EE10FA03F56B63B8BFF0EE477A93ED7D
:106ED000007AB4EE677AF1EE10FAC8BFF0EE477AA6
:106EE00037EEA77AB4EEC70AF1EE10FA1BDD94F87C
:106EF000943023BB9FED187AD4ED187A67EE877A29
:106F0000C4ED187A4DF02EFC0546206EF9F7F4FA20
:106F1000124ACDE900010421284646F077FD0123FD
:106F200084F89430A8E7B4EEE70AF1EE10FA02D53F
:106F300094F8943043B92046FFF7BAFE9CE7B4EECC
:106F4000E70AF1EE10FAF6D50023E9E76026002003
:106F5000CDCCCC3DCDCC4C3ECDCC4C3FB47B0B0806
:106F600037B5C368DFED1B7A03F5566393ED000A6E
:106F7000B4EEE70AF1EE10FAD8BFB0EE670ADFED23
:106F8000167A20EE270AD0ED177A20EE270A04465B
:106F90001BF0B0F8B5EEC00AF1EE10FAD8BF9FEDC5
:106FA0000F0AD4ED187AF4EEC07AF1EE10FA0EDD85
:106FB00084ED180A4DF0D6FB0546206EF9F79CFAD1
:106FC000074ACDE900010421284646F01FFD03B021
:106FD00030BD00BFCDCCCC3D0AE81C410000000014
:106FE000E07B0B08DFED137AB4EEE70AF1EE10FA5E
:106FF00010B504461CDB80ED180AFFF7B1FFE0680E
:1070000094ED180A00F5CD53D3ED607AB4EEE70A9B
:10701000F1EE10FA03F1180308DDD3ED5D1A93EDDC
:107020005C1AD3ED5B0A18466BF0F8FF012000E014
:10703000002010BD0000003437B5C36890ED177A0A
:1070400003F56B63D3ED007AB4EEE77AF1EE10FA54
:10705000044611D5C0ED177A4DF084FBE36803F5C3
:107060006B6305461868F9F747FA044ACDE9000151
:107070000421284646F0CAFC03B030BDFC7B0B0857
:10708000F0B52DED028B0D4683B000230446694612
:107090002846B0EE408A1746009301930AF0A2FCFE
:1070A00028B90026304603B0BDEC028BF0BD236842
:1070B00020469B6D984706460028F2D09FED110AA6
:1070C00068461DF06BFCDFED107A84ED150AB0EE1A
:1070D000C80AB4EEE70AF1EE10FAD8BFB0EE670ABC
:1070E000C4ED160A84ED170A2046FFF7A5FF676670
:1070F0002046FFF75DFD95E80F00443484E80F005B
:10710000D0E700BF0AD7233CCDCCCC3D70B50446B8
:107110002DED048B05F01AF804F1540103F078FF0B
:107120000646002800F09C80D4ED0E7ADFED4E9AE2
:107130009FED4E9ADFED4E8AF0EEE77AF4EEE97AB3
:10714000F1EE10FAD8BFF0EE697AC4ED177A204656
:10715000FFF772FF94F94030D4ED0F7A5A1EF4EE27
:10716000C97A53425341F1EE10FA6366BEBFE36839
:1071700003F58053D3ED507AC4ED187A04F0E6FF9E
:10718000D0F80C32E3663B4BC4ED1A8A0FCB04F106
:10719000440585E80F002046FFF7E2FE002384F84F
:1071A0009430E36803F67C2003F6485393ED008A9D
:1071B000B4EEE88AF1EE10FAD8BFB0EE688A6BF050
:1071C000FFFCB4EE480AF1EE10FAF0EE400AC8BF38
:1071D000F0EE480AE068F4EEC90AF1EE10FAF7EEB4
:1071E000007A00F58053B8BFF0EE670AD3ED577A06
:1071F000F4EEC97AF1EE10FA06DBF4EE670AF1EE6E
:1072000010FAC8BFF0EE670AD3ED581A9FED167A50
:107210009FED191A94ED180A00F55663D3ED007A24
:10722000F4EEC91AF1EE10FAF4EEE97AB8BFF0EE16
:10723000601AF1EE10FAD8BFF0EE477A41F6B815B1
:1072400027EE811A28446BF0E9FEE06828446CF0D0
:1072500067F80023C4ED228A84F88C30C4ED248AB8
:10726000BDEC048B304670BDCDCCCC3D000000346D
:1072700000000000C47B00200AE81C410F2070477A
:1072800000487047E07C0B080120704701207047E0
:1072900090F8383023B1032B0CD09FED080A7047CB
:1072A000C36803F5C75393ED040ADFED057A20EEBA
:1072B000270A7047034B93ED000AF6E70000000031
:1072C0000AD7233C4C85002090F8383023B1032B9B
:1072D0000CD09FED080A7047C36803F5C75393EDC0
:1072E000030ADFED057A20EE270A7047034B93ED82
:1072F000000AF6E7000000000AD7233C4C85002076
:1073000090F838302BB9C36803F5C75393ED050ADD
:1073100070479FED010A70470000000090F8383078
:1073200023B1032B05D09FED050A704790ED0B0AA2
:107330007047034B93ED000A704700BF0000000048
:107340004485002090F838302BB9C06800F589508A
:107350001C306CF057BA00207047000030B52DED9E
:10736000028B012587B080F838500446F0EE408A41
:10737000B0EE608A71F000FB0023E063019302939A
:107380000493059394F838100948C4ED0D8A84EDF0
:10739000128A84F8395003AB6A46CDED008A8DED30
:1073A000038AFBF705FD07B0BDEC028B30BD00BFC3
:1073B0006026002010B52DED028B022386B080F8E8
:1073C00038300446F0EE408AB0EE608A71F0D4FAAC
:1073D000012384F839300023E0630193029304937E
:1073E000059394F838100848C4ED108A84ED128A89
:1073F00003AB6A46CDED008A8DED038AFBF7D8FC1E
:1074000006B0BDEC028B10BD6026002010B504460E
:107410000348FDF751FE10B1032384F8383010BD46
:107420001885002010B504460B4802F02BF918B15E
:107430002046FFF7EBFF10B9052384F83830E068E9
:107440009FED060A00F589501C306CF0F9FE002310
:1074500084F84430012010BD6026002000000000A8
:10746000C16580ED180A70470023C36500230366D9
:107470007047000010B5044671F07EFA034B606659
:107480000FCB683484E80F0010BD00BFC47B002020
:1074900010B5C36D044653B994ED187ADFED107A38
:1074A000B4EEE77AF1EE10FA0ADA002010BD71F0BE
:1074B00063FA636EC01AE36D9842EDD30120F5E7DD
:1074C000084804F168010AF0C7FBD4ED187AB4EE5D
:1074D000E70AF1EE10FACCBF01200020E6E700BF7A
:1074E00000000034C47B0020C36803F58053D3F848
:1074F000780BC0F38010704790F838302BB9C06813
:1075000000F589501C306CF0EFBF0120704700007F
:1075100070B590F838300446052B00F2D880DFE8CB
:1075200003F0032D709FA44AC06800F589501C30F9
:107530006CF0DAFF20B92046BDE87040FEF718BABB
:1075400094F844302BB10021654884F844104AF087
:10755000B3FB644802F096F818B12046FFF756FFD7
:1075600010B92046FDF72AFFE1685F4801F5C551D3
:107570000C310AF071FB84ED0B0A70BD90F83930C4
:1075800083B171F0F9F9E36BC01A40F6B833984251
:1075900016D94DF0E7F8554A042146F037FA002392
:1075A00084F839304F4802F06DF820B12046FFF7DB
:1075B0002DFF0028E1D12046BDE87040FDF7FEBE5A
:1075C00094F83930002BEDD0DFED490A94ED0D0A27
:1075D0002046FEF70BF994ED120ADFED467A236898
:1075E000B4EEE70A1D6EF1EE10FA204694BF0121B9
:1075F0000021FEF759F820462B460121BDE87040D6
:10760000184790F83930002BCCD071F0B5F9E36B06
:10761000C01A40F6B8339842BBD894F83930002BE2
:10762000C0D0E368D4ED107A9FED330A93F8F019D7
:107630002C4BA06AD3ED460A67EE807A9FED2F0AA5
:10764000C1F3400227EE800A01F001016BF074F9EA
:10765000DFED2B7A204620EE270AFEF77FF8BAE707
:10766000BDE87040274800F037B990F84C30002B47
:1076700098D071F081F9236DC01A40F6B833984262
:1076800008D9002384F84C304DF06CF8174A0421D7
:1076900046F0BCF994F84C30002B83D094ED150AD9
:1076A000E068DFED177A00F51F6020EE270A002161
:1076B0006FF084F894ED160AE068DFED137ABDE808
:1076C000704020EE270A00F51F606FF07DB84DF086
:1076D00049F8BDE870400D4A042146F097B900BF53
:1076E000A879002060260020C47B0020E87C0B08DD
:1076F00000000000000000B40AD7233C35FA8E3C9D
:1077000000A08C45188500200000C842117D0B08A0
:1077100090F8383023B1032B08D09FED060A70474C
:10772000C36803F5C75393ED020A70470248FDF79B
:10773000BBBB00BF000000001885002038B590F8E2
:1077400038300C4623B1032B12D00025284638BD13
:10775000C06800F5805393F8CC58002DF6D000F5A2
:1077600089501C306CF0D2FE0FC884E80F00EDE7A2
:10777000BDE83840014800F0A7B800BF18850020D8
:1077800082B070B5054688B00CAC84E80C00FFF7F9
:10779000ABFEEC6804F589540E461C34002833D047
:1077A000DDE90E018DE803000CAB0CCB3146204621
:1077B0006CF0C4FE30B30021012485F8381085F840
:1077C0004440EB68D6ED027A114803F5C653B8EE93
:1077D000E77A1433D6ED037A1B6805930022F8EE9E
:1077E000E77A04920692079205AB02AA8DED027A1F
:1077F000CDED037AFBF7DCFA204608B0BDE8704017
:1078000002B070470020F8E720466CF0D1FCD1E7C9
:10781000602600200420704700487047ED770B0871
:1078200000207047002070470020704713B50023E8
:10783000044610480193FCF789FD18B10D4801A9D1
:10784000FCF74EFDE06800F5CB50083001F092F8EF
:10785000E0689DED010A00F51F606EF0B5FFE0687D
:107860009FED050A012100F51F606EF0A7FF02B031
:1078700010BD00BF602600200000000005207047FA
:1078800000487047007E0B080120704790ED0D0AFC
:10789000DFED027A20EE270A704700BF0AD7233CAB
:1078A00090ED0D0ADFED027A20EE270A704700BF47
:1078B0000AD7233C9FED010A704700BF000000007B
:1078C00090ED0B0A7047000010B538300C460FC819
:1078D00084E80F00012010BD30B52DED028B044669
:1078E00083B000F138017C4801910AF0B5F9E068F5
:1078F00084ED0B0A00F5CB50083001F05DF9E36828
:107900000199002855D003F5CC5292ED027AD4EDBE
:107910000B7AF4EEC77AF1EE10FA4FD841F66815FB
:10792000581901F049F96D4BDFED6D7A9FED6D0A45
:10793000D3ED460A002808BFB0EE670AA06A6BF0D4
:107940006BF9E06884ED120A284401F035F990B92A
:10795000E36803F5805393F96829002A0BDDD3ED22
:107960002C7A9FED617A67EE877A9FED607A67EEF9
:10797000877AC4ED0D7AE06894ED0D0A41F668153A
:10798000284401F099F9002840F08D80DFED540A79
:1079900094ED0D0A2046FDF729FF236894ED120AA5
:1079A0001B6E0121204603B0BDEC028BBDE83040C8
:1079B000184703F5805292ED137AA8E703F5805338
:1079C00003F51B6277EEC77A92ED007A4248DFED4D
:1079D000488A67EE877A93ED507AF4EE477AF1EEB3
:1079E00010FA48BFB0EE677A84ED127A0AF04EF8CA
:1079F000B6EE008A9FED3F7A6368F0EE487AE0EEDB
:107A0000077AFDEEE77AF8EEE77AC4ED0D7A93EDAA
:107A1000800AB8EEC00A37EEC00A1AF0E5FBF0EEB5
:107A2000C07AF4EEE87AF1EE10FAE36804DD03F5CB
:107A3000805292F949202AB103F5805393F94930D5
:107A4000022B18D1DFED2C7A94ED0D0A30EE270AC7
:107A50001AF0CAFB636884ED0D0AD3ED807AF8EE64
:107A6000E77A30EE670A1AF0BFFBD4ED127AF1EE36
:107A7000677AC4ED127AC0EE287A3620DFED180A54
:107A8000B0EEE70AB7EE001A1AF004FCF7EE007A3F
:107A9000E0EE487AB0EE677AD4ED127A67EE877A34
:107AA000C4ED127A67E7E06894ED0D0A284401F00E
:107AB00037F9E06884ED0D0A284401F0F5F8002854
:107AC0003FF464AFE36803F58053B3F94A3100EE45
:107AD000903AF8EEE00A5BE7C47B002060260020C5
:107AE00000000000CDCCCC3DE02E65420000C84235
:107AF00000A00C46A00CB34500A08C4638B5044647
:107B0000C06800F5895004F138011C306BF0ECFEC0
:107B1000054670B1A06A04F148016AF087FE08B911
:107B20000023A3646368D3ED807AF8EEE77AC4EDAE
:107B30000D7A284638BD0000002070470048704785
:107B4000747E0B08012070470020704700207047AA
:107B500000207047C0689FED030A00F51F606EF0BB
:107B60004FBE00BF0000000010B52DED028B86B0A7
:107B7000044601AA6946FDF74BFB204602A9FDF722
:107B8000C1FBE3689FED2D8A9DED000A03F5DC53F0
:107B900080EE080AD3ED000A1BF020F820EE080A58
:107BA00027488DED000AFCF7D1FB18B1244801A944
:107BB000FCF796FB04AA03A92046FDF7BDFB05A927
:107BC0002046FDF7D3FBE0689DED030A00F51F603A
:107BD0006EF026FEE0689DED040A00F51F606EF071
:107BE0002BFEE0689DED050A00F51F606EF032FE89
:107BF000E06800F5CB50083000F0D8FEE0689DED5D
:107C0000010A00F51F606EF0DFFDE0689DED000ADF
:107C100000F5805300F51F60D3F87C1B01F00101D3
:107C20006EF0CCFDE0689DED020A00F51F606EF07D
:107C3000E7FD06B0BDEC028B10BD00BF00A08C4577
:107C4000602600200B20704700487047703A0B08F0
:107C5000012070470020704790ED0B0A704700002C
:107C6000C06800F589501C306BF0CCBD70B58AB08F
:107C7000044604F06BFA90F87C32DB0702D4002053
:107C80000AB070BDE36803F5895003F6687393ED9D
:107C9000000AB5EEC00AF1EE10FA48BF9FED130AD4
:107CA0001C306CF0CDFA6368E66893ED9C0A104ACC
:107CB00006F582511031B8EEC00A02A806AD3BF0BD
:107CC0001FFB284609F038FD0AAB13E903008DE8D5
:107CD000030006F5895095E80C0002A91C306CF0F1
:107CE0002DFC0028CBD001232387C9E7000000002A
:107CF000C47B0020C06800F589501C306CF0F4BBD8
:107D000010B50446C06800F589501C306CF0ECFBDF
:107D100020B92046BDE81040FDF72ABE94F838305F
:107D200043B1002384F838304CF01CFD114A062181
:107D300045F06CFE104801F0A5FC60B92046FDF747
:107D40003DFBE1680D4801F5C5510C3109F084FF98
:107D500084ED0B0A10BD94F839301BB10848FFF7C9
:107D6000BBFDEEE70648FDF7A7F984F839000028C7
:107D7000E4D0F3E7E87E0B0860260020C47B0020F7
:107D80001885002038B5C06800F580530C4693F87C
:107D9000CC583DB100F589501C306CF0B7FB0FC8D2
:107DA00084E80F00284638BD072070470048704718
:107DB000687F0B0813B5044601AA6946FDF708FC65
:107DC000E36803F5805393F964304BB994ED0E0AE0
:107DD000DDED007A30EE270A1AF0F0F98DED000A99
:107DE000DFED0E7A9DED017ADFED0D0AB4EEE77A54
:107DF000F1EE10FAB5BFE36B009B0093E3639DEDDA
:107E0000000A2046FDF7F2FC23689DED010A1B6E77
:107E100001212046984702B010BD00BF0000003489
:107E2000000000004368D3ED807AF8EEE77AC0EDF9
:107E30000E7AD3ED807AF8EEE77AC0ED0F7A7047CC
:107E40000C207047004870476F3A0B0801207047BC
:107E50000020704790ED0B0A7047000090F8380042
:107E6000831E584258417047C06800F589501C3045
:107E70006BF0C8BC30B590F83830012B0C460CD1F3
:107E8000C36803F5805393F8CC5825B103F6AC03CF
:107E90000FCB84E80F00284630BD0025FBE700002B
:107EA0001FB50446684609F047FC6068694603F060
:107EB00053FF10B9002004B010BDE36893F8C42E3E
:107EC000002AF7D003F5895003F6687393ED000A92
:107ED000B5EEC00AF1EE10FA54BFBDEEC00A9FED38
:107EE0000A0A1C30B8EEC00A6CF0AAF9E06800F586
:107EF00089501C306BF044FD0028DBD0002384F84F
:107F0000383084F83A30D6E700000000064BC068ED
:107F1000D3F8F82503F67C73D21A18BF0122012189
:107F200000F6B8606DF070B86076002030B590F85B
:107F30003830012B87B0044615D004D9023B012B01
:107F400072D907B030BDC068002100F6B8606CF08F
:107F50000FFB10B140F201132387204607B0BDE8A4
:107F60003040FDF72BBA90F83930002B3AD0C0687A
:107F70000025694600F6B8600095019502956CF001
:107F800035FF48B94CF0EEFB344A062145F03EFD82
:107F9000022384F83830D4E7E068039503A900F69B
:107FA000B860049505956CF053FFE56841F23C1309
:107FB00038B303AA6946E8186BF060FC78B94CF056
:107FC000D1FB274A062145F021FD032384F83830F0
:107FD00042F082F83D224FF4801142F035F8002340
:107FE00084F839302046FDF7C3FCE06800F589507D
:107FF0001C306CF079FA0028A3D0012384F83930C2
:108000009FE76946E8186BF013FC0028E7D14CF0B5
:10801000A9FB134A062145F0F9FC032384F8383004
:1080200042F05AF84522D6E7012380F830300D4857
:1080300001F028FB002890D094F83A302BB10A4880
:1080400007B0BDE83040FFF747BC0748FDF734F8FC
:1080500084F83A00002880D0F1E700BFE87E0B08E2
:10806000DC7F0B0860260020188500200320704765
:10807000004870477F520B0801207047002070476E
:108080000120704790ED0E0A7047000070B52DED8D
:10809000048B84B0044601A9806A6AF0C7FBB0B9BA
:1080A0009FED4E8AE068B0EE480A00F51F606EF062
:1080B0008BFBE0680121B0EE480A00F51F606EF00E
:1080C0007DFB84ED0E8A04B0BDEC048B70BD03AA69
:1080D00002A92046FDF726FADFED418A9DED039ABD
:1080E000E0689FED408AB4EEE89AF1EE10FA00F5F0
:1080F0001F6094BF012600266EF008FCE368A56AA5
:1081000098B3DDED037A9FED387AF0EEE77AF4EE7E
:10811000C77AF1EE10FA28D5DDED027A9FED337AB9
:1081200087EE880A03F6B4622846D2ED007A002270
:10813000A26393F8F0192E4B67EE877AC1F34002E1
:10814000D3ED460A20EE270A01F001016AF0F4FBA4
:10815000204620EE080AFDF701FB23689DED030A87
:108160001B6E012120469847ADE703F56B63DFEDF9
:10817000210AD3ED007A95EDB97A9DED010A9FEDC4
:108180001E1AF4EEE07AF1EE10FAB4EEE07AD8BFFF
:10819000F0EE607A20EE000AF1EE10FAD8BFB0EEF1
:1081A000607A27EE011A80EE270A26201AF072F86C
:1081B000314620469DED027AC7EE087AB4EEE89A81
:1081C00027EE800AF1EE10FA98BFB1EE400A84ED76
:1081D0000E0A94ED0E0AFDF733FBBEE70000000027
:1081E000000000B400A08C450000003435FA8E3C3D
:1081F00060260020CDCCCC3D0AE81C4170B500F5CE
:10820000A046044696F8953BF3B16AF073F803680C
:10821000012203219B6898470C4B00251D6004F543
:1082200005500B4B34301D603AF0ECF804F5055066
:1082300030303AF0E7F804F5055035303AF0E2F81E
:10824000044B86F8955B5D7270BD00BF9886002078
:108250009C8600203D87002037B500F5A0430446EA
:1082600093F8953B002B34D070F086FB294B1B68AC
:10827000C01A294B1B68984205D3204603B0BDE8BD
:108280003040FFF7BBBF254B1B78012B11D0022BD1
:1082900021D0F3B9224BB3F9003000EE103A214B54
:1082A00004F52D50B8EEC00A197838306FF01EF87A
:1082B0000DE01B4BB3F9003000EE103A194B04F5FA
:1082C0002D50B8EEC00A197838306EF05FFB0028E8
:1082D000D3D003B030BD134B197804F52D550229C6
:1082E00005F1380504F540530BD1D3F8B00D0191D9
:1082F0004DF0EEFDDFED0C7A019920EE270A2846BD
:10830000D4E7D3F8B43DB3F9083000EE103AB8EE34
:10831000C00AF4E7988600209C860020A0860020F2
:10832000A2860020948600200000C8422DE9F84370
:10833000984600F5A0439DF8206093F8F455BDF9E8
:1083400024700C463DB9224A0221204648F0BCFD6B
:108350002846BDE8F8836AB100F578500121343031
:10836000F9F732F930B91B4A0221204648F0ACFD3A
:108370000025EDE7184B1B68D86A0368DB6998474E
:10838000012801D1154AEFE7B8F1040F06D9144AC4
:1083900043460221204648F097FDE9E7022E02D924
:1083A000104A3346F5E7012E06D140F698039F4266
:1083B000CEDD0D4A3B46ECE7002EC9D1642FC7DD68
:1083C0000A4A3B460221204648F07EFD3546BFE77B
:1083D000D8800B08F7800B085826002015810B0861
:1083E0002F810B084E810B0874810B0892810B08BA
:1083F0002DE9F0432DED028B00F5A04583B01E461C
:1084000095F8953BBDF9308004461746B0EE408A9A
:108410002BBB1346721E18BF0122CDE90068FFF77F
:1084200085FF28B9042003B0BDEC028BBDE8F083C2
:108430004FF0010985F8959B04F5785534352846A9
:1084400068F0A8FD50B304F50054002384F874319B
:1084500084F8703184F87531144B01225A7270F02F
:108460008BFA9FED130ADFED137A134B28EE000A07
:108470001860B4EEE70AF1EE10FA58BFB0EE670AE2
:108480000E4BBCEEC00A002083ED000A0C4B1F709F
:108490000C4B1E700C4BA3F80080C4E74A46032126
:1084A0002846F9F785F90028CDD1BBE73D870020A4
:1084B00000007A440060EA46988600209C860020EE
:1084C00094860020A0860020A286002070B500F5CA
:1084D00006560C36054630464DF0D0FB05F54054A7
:1084E000C4F8B00D30464DF0DDFBC4F8B40D304695
:1084F0004DF0E2FB41F29411C4F8B80DD4F8B00D80
:108500004DF02AFCD4F8B40D64214DF025FCD4F8CC
:10851000B80D10B164214DF01FFCC92130464EF05A
:1085200073FBCA21C4F8BC0D30464EF06DFBD3215D
:10853000C4F8C00D30464EF067FBC4F8C40DD4F843
:10854000BC0D40B141F294114DF006FCD4F8BC0DC5
:108550001E214DF005FCD4F8C00D40B141F294113C
:108560004DF0FAFBD4F8C00D1E214DF0F9FBD4F804
:10857000C40D40B141F294114DF0EEFBD4F8C40D9E
:108580001E214DF0EDFB05F56B50303000F0F4F896
:1085900005F57850343068F0FDFC40B905F52D54F0
:1085A000383420466EF0DEF820466EF0BBF8084BFB
:1085B0001B685B6A4FF47A72DA804FF4FA6205F551
:1085C00013501A81BDE8704046211C304EF074BE35
:1085D0005826002010B500F540541E21D4F8B00DE7
:1085E0004DF0BEFBD4F8B40D1E214DF0B9FBD4F80C
:1085F000B80D20B1BDE810401E214DF0B1BB10BD3B
:1086000070B500F50053054693F970210C46DAB1B8
:10861000B3F9726170F0B0F905F5A043D3F80C36E8
:10862000C01AB0F5FA7F0DD8B3B29C422CBF00231C
:108630000123064A93722846054ABDE8704001218D
:10864000FCF798BA0123F4E770BD00BF3D87002016
:10865000B8810B082DE9F84300F54058054698F914
:10866000449EB9F1000F09D0D8F8B40D4DF0E2FCEA
:1086700005F5A04420B90023C4F8743BBDE8F88395
:10868000D4F8F80503685B6998470028F3D005F52E
:1086900078563436304668F07DFC0746B8B9D8F8CD
:1086A000B03DB3F90830B3F57A6FE4DD70F064F9EA
:1086B000D4F8743B73B3C31AB3F5FA6FDED3012257
:1086C00039463046F9F774F8C4F8747BD6E7B9F147
:1086D000020FD3D105F52D5038306FF03BFA054627
:1086E0000028CBD1D8F8B03DB3F9083013F57A6F34
:1086F000C1DA70F041F9D4F8743B5BB1C31AB3F539
:10870000FA6FBBD3012229463046F9F77BF8C4F84B
:10871000745BB3E7C4F8740BB0E7000038B50446E7
:1087200000F506500C304DF08BF904F5405538B982
:10873000D5F8B43D2046D988BDE83840FFF760BF82
:1087400070F01AF904F5A043C3F80C06D5F8B43D4F
:108750002046D988FFF754FF2046BDE83840FFF790
:1087600079BF000010B50349044639F075FD204675
:1087700010BD00BF2C820B0810B504464DF0A6FAC0
:10878000CF214EF041FA48B1606264214DF0E4FA25
:10879000606A1E21BDE810404DF0E2BA024BD3F8EA
:1087A000B43D636210BD00BF6056002038B52DEDAA
:1087B000088BDFED627A624D9FED62BAD5ED460A15
:1087C000DFED61BADFED618AF0EE40AA90ED040AB8
:1087D000044620EE270A5E4805F5405569F0B8FFCB
:1087E000D5ED8C7A9FED5B7A67EE877ABFEE008AD3
:1087F000F4EECB7AF1EE10FAB7EE001AF4EEEBAA33
:1088000088BFB0EE418AF1EE10FA20EE28AAB0EE51
:10881000E79A76DB94ED030A94ED021AD4ED010A8F
:10882000D32039EE400A19F035FDF0EE680AB0EEBB
:10883000401A94ED022AD4ED011A9FED470A19F06F
:1088400069FCDFED450A3AEE000AD820B0EE681A5E
:1088500019F020FD41486EF00BF8F4EECBAAF1EED2
:1088600010FADFED3A7A3D48B4EEE8AAF7EE009A46
:10887000BFEE000A88BFB0EE690AF1EE10FA48BFF9
:10888000F0EE4A7A78EEE78A68EE888A28EE800A67
:108890006EF000F8F4EEEBAAF1EE10FA4BDB94ED7B
:1088A000037AB4EEC97AF1EE10FA44DCDFED2C8ADB
:1088B00077EE287AF4EEC97AF1EE10FA24DDDFEDD6
:1088C000296AF0EE697AEAEE667AF5EEC07AF1EEA0
:1088D00010FAD8BFDFED207AA7EE679A28EE091AC2
:1088E00094ED022ADFED190A9FED1F0AF1EE421AFC
:1088F00019F010FCBDEC088B1848BDE838406DF04D
:10890000DBBFB0EE680AA5E7DFED187AB4EEE79AB0
:10891000F1EE10FA0CDD89204EF072FB9FED141A77
:10892000B4EECB0AF1EE10FA88BFB0EE681AD7E7C2
:1089300028EE281AD4E79FED080ADBE735FA8E3CCB
:1089400060260020000000B4000000340000C8428F
:1089500064520020E02E654200000000D851002043
:108960000000B4420AD7233C0000C8C200000743FD
:108970000000B4C207B59FED0A0A0A486DF078FFFF
:108980009FED090A07488DED010A6DF083FF9DED0B
:10899000010A044803B05DF804EB6DF08DBF00BF21
:1089A0000000C842D85100200000000010B5204B44
:1089B00093F80036DB07044601D4436A23B9204606
:1089C000BDE81040FFF7D6BFB3F908309FED191A84
:1089D000DFED190A00EE103AB720B8EEC00A19F020
:1089E00059FC16486DF044FF636A9FED121AB3F903
:1089F0000830DFED130A00EE103AB820B8EEC00AD6
:108A000019F048FC0D486DF045FF636A9FED091AA7
:108A1000B3F90830DFED0A0A00EE103AB920B8EEDB
:108A2000C00A19F037FCBDE8104004486DF044BF9F
:108A3000607600200000C84200000000D8510020ED
:108A40000000C8C213B5154801A969F0EFFE10B3C4
:108A5000134CD4F8F8050368DB68984718B99DED06
:108A6000010A02B010BD0F4B9FED0F7AD3ED007AD3
:108A7000A4F56E5367EE877A13ED030A9FED0B7A28
:108A800097EE870A19F0F2FB93F0E0F9DDED017A39
:108A900020EE270AE5E79FED060AE2E76452002090
:108AA00060760020D86000200AD7233C35FA8E3C3F
:108AB0000000000010B5002380F8283080F83C301A
:108AC000036304466FF058FFA06310BD10B5114B4F
:108AD00090ED0B0AD3ED007A30EE670A044619F0E8
:108AE000C5FBDFED0D7AB0EEC00AB4EEE70AF1EE99
:108AF00010FA05D52046FFF7DDFF94ED0B0A10BDF7
:108B00006FF03AFF236BC01A41F288339842F1D8D4
:108B1000F3E700BFD43A0020C2B8323E70B5054634
:108B200016460C4609B92C6470BD0C486DF0EEFE7B
:108B30000028F8D146204EF0F3FB0028F3D1084B73
:108B400093F9D031002BEED1002EEDD04BF00AFE80
:108B5000BDE87040034A042144F058BFD8510020BA
:108B600060560020C0810B0810B5036C012B044631
:108B700001D0002010BD90ED067ADFED0C7AB4EE46
:108B8000E77AF1EE10FAF4DB09486CF0FBFE0028FE
:108B9000EFD0084BD4ED067A93EDA57AB4EEE77AE0
:108BA000F1EE10FA4CBF01200020E3E70000003492
:108BB000505800206056002008B590F90020002A87
:108BC00008DD036C022B05D0FFF7CEFF80F001001B
:108BD000C0B208BD0020FCE713B590F90030002BAF
:108BE00004460EDD002311488DF807300DF1070112
:108BF0003AF048F9236C0E4A023B18BF012382F871
:108C0000163A2046FFF7D8FF38B1012309488DF8FE
:108C100007300DF107013AF035F900220121204615
:108C200002B0BDE81040FFF779BF00BF98570020A1
:108C3000605600203158002010B52DED028B0446FF
:108C4000FFF7BAFFE0B194F82830CBB9012384F8DC
:108C500028300D4B93ED008A0C4B93ED8E0A30EECD
:108C6000480A19F003FBF0EE007AA0EE278AB0EE76
:108C7000480A19F0E5FA84ED0B0A6FF07DFE2063D7
:108C8000BDEC028B10BD00BFD43A0020605600201E
:108C900010B50446FFF790FF28B194F8283013B9B7
:108CA0006FF06AFE206310BD10B50446FFF784FF25
:108CB00008B194F8280010BD10B52DED028B0446C4
:108CC000B0EE408AFFF778FF00B394F82800E8B9C7
:108CD000DFED107A104B27EEC87A93ED8E0A9FEDE8
:108CE0000F8AA7EE080A19F0C1FAD4ED057AB2EEA0
:108CF000047A77EE877AB0EEC00A67EE887AB4EE2F
:108D0000E70AF1EE10FA94BF01200020BDEC028BBF
:108D100010BD00BF0AD7233C6056002035FA8E3CB8
:108D20002DE9F8432DED048B0446B0EE408AFFF7A1
:108D300043FF8146002800F0D580DFF82C82DFED6C
:108D40007E7AD8ED8E9ADFED7D8A98F8B07267EE64
:108D5000C87AB0EE699AA7EEA89AB0EE490A19F05F
:108D600085FAD4ED057A67EEA87AB0EEC00AB4EEC3
:108D7000E70AF1EE10FA40F3A48094F82830002BB3
:108D800040F09F80B0EE490A19F070FADFED6C7A7E
:108D9000B4EEE70AF1EE10FA8CBF012300239F42E4
:108DA00000F0A080D8ED8C7AB0EEC00AF0EEE77A41
:108DB00037EE800ADFED637AB4EEE70AF1EE10FADF
:108DC00040F190804E466FF0D7FD236B054653B1BE
:108DD0004EB994F8282032B9C31AB3F5FA7F2CBFE4
:108DE00000260126226308F67C2898ED007AD4ED4F
:108DF000077AF0EEC76AF4EEE76AF1EE10FA1EDBCE
:108E0000DFED516AF0EEE77AF4EEE67AF1EE10FA71
:108E100015D4A6B994F828308BB9B4EEE67AF1EE01
:108E200010FA02DB7B1E5E425E41DFED457AB4EE56
:108E3000E77AF1EE10FA02D8002F08BF4E46D4EDC3
:108E4000057A9FED428AB0EE690AA7EEA80A19F0EA
:108E5000F7F9D4ED057AB0EE409AB0EE690AA7EEC4
:108E6000E80A19F0EDF9DFED3A9AF0EE408A86B3A0
:108E7000A36B41F28832EB1A93422AD94BF072FC71
:108E8000344A062144F0C2FDEFB1012F1ED0012368
:108E900084F828306563304B94ED0B0AD3ED007AEB
:108EA00030EE670A19F0E2F9DFED2C7AB0EEC00A75
:108EB000B4EEE70AF1EE10FA1AD82046FFF7FAFDF1
:108EC0002CE000267FE7C4ED0B8AE0E784ED0B9AE7
:108ED000DDE794F82830002BDDD10FBB29EE299A6D
:108EE00029EE088AB0EE480ABDEC048BBDE8F88391
:108EF000606B41F288332D1A9D420FD9236C012BF0
:108F000013D107EE905A9FED167AF8EE677AF4EED9
:108F1000C77AF1EE10FA08D584F83C30D4ED0B8A0C
:108F200068EEA98A28EE888ADCE74BF01BFC0D4A24
:108F3000062144F06BFDC0E70AD7233C35FA8E3C8E
:108F4000000000B4DB0F4940000000340000C842BC
:108F5000E02E6542E4810B08D43A0020C2B8323ECC
:108F600000606A46F6810B086056002038B52DED8A
:108F7000028B00230B6090F90030002B0446B0EE0A
:108F8000408A0D4606DCBDEC028B2046BDE8384029
:108F9000FFF7F0BC036C022B2ED11D4A9FED1D1A6A
:108FA000D2ED461A02F50053D3ED560A93F9660145
:108FB00093F8781B07EE900AF8EEE77AC1F3C00247
:108FC00027EE811AC1F38001B0EE480A03F604408F
:108FD00069F07EFEDFED107A20EE270A85ED000AAB
:108FE000236C022BCFD0B0EE480ABDEC028B20469A
:108FF000BDE83840FFF7DABB012B03D190F83C30D5
:10900000002BCAD12046FFF7AFFD0028C5D1E7E706
:10901000602600200AD7233C0000C84200F25450CA
:1090200009F052BB10B5044609F03EFC90F921301E
:109030008BB190F8403373B194F978355BB104F596
:109040007850343067F0A6FF28B904F25450BDE8D8
:10905000104009F051B910BD2DE9F0432DED028B00
:1090600000F5005783B097F858390646002B00F0FA
:10907000948000F523542434204666F0CFF84FF056
:10908000000841F2DE6997F858295FFA88F5AA428C
:109090000BD92946204666F015F94D4406EB8505A7
:1090A00085ED000A08F10108EDE706F5A04595F801
:1090B000803BEBB9012285F8802B1D4697F8583983
:1090C0005FFA85F94B4568D94946204666F0DAF8DB
:1090D00006EB890808F5A04808F6843383ED000AFA
:1090E0004946204666F094F90135C8F88C0BE5E74F
:1090F00095F8943B0133DBB2934228BF002385F8F7
:10910000943B95F8941B204666F0BCF895F8941BA8
:109110002046B0EE408A66F07BF907466FF02CFCE3
:1091200095F8941B06EB810303F5A04303F6843204
:10913000D2ED008A82ED008AD3F88C2BA7EB0208CF
:1091400008F1FF3CBCF1630F84BF0746A0EB0208A7
:10915000C3F88C7B204666F08DF895F8941B01903F
:10916000204666F07BF807EE908ADFED0E0A019A42
:10917000F8EE677A78EE688A06F5935067EEA00AF3
:10918000B0EE401A3946B0EE680A083003B0BDECC4
:10919000028BBDE8F04320F081BD03B0BDEC028B33
:1091A000BDE8F0836F12833A10B5044600F55160B4
:1091B0003AF0CEFB2046BDE81040F9F77FBD000035
:1091C000F9F7A8BF0148FBF7ADBC00BF602600203F
:1091D00070B52DED048B00F54053044693F9F4303F
:1091E000022B56D000F5005505F6783393ED0A9A18
:1091F00095F9663108EE103AB8EEC88AF6EE008AA4
:1092000028EE288AF2EE0E7A00F53056B4EEE78AA0
:109210000436F1EE10FA304658BFB0EE678A69F0B6
:10922000DDFC48B1304669F0E9FCB4EEE80AF1EE45
:1092300010FACCBF01200020B4EEC98AF1EE10FA7A
:1092400004F5A0460BD405F6783595ED0A7ADFEDE6
:10925000127AB4EEE77AF1EE10FA16DBA8B16FF0ED
:109260008BFBD6F8703B0BB9C6F8700BD6F8703B89
:10927000C31AB3F5FA6F94BF0023012304F5805499
:1092800084F87135BDEC048B70BD0023C6F8703BCB
:10929000F4E70023F2E700BF0000003408B5044AF9
:1092A0000B2340F08BFD80F00100C0B208BD00BF71
:1092B00058830B0838B5044600F5A640154A062128
:1092C000483044F0A3FB144B1B68986A036804F50C
:1092D00093555B68642108359847284601F026FCC1
:1092E00004F58053012283F8712583F87C24B4F9B6
:1092F000A43004F698001BB9B4F8A230A4F8A43046
:10930000B4F8A41018F030FB2846BDE8384001F04E
:1093100013BD00BFCC820B085826002070B50B6827
:109320000B4EDB68054608460C46984730742368A8
:1093300020461B689847F070236820465B68984772
:10934000014605F590501430BDE8704036F0B8B9CC
:109350003D8700202DE9F04700F5A0470646D7F8E5
:10936000F8358B420C46914664D000F5A648022A97
:1093700008F1480816D10B6808461B689847014653
:109380003046FFF78BFF054660B9236820465B68CF
:109390009847294A03460521404644F037FB2846B2
:1093A000BDE8F0872046D7F8F8A5FBF785FE05460F
:1093B00088B942F085FB236806461B68204698471B
:1093C0000A210246304642F0D7FA1C4A04214046A0
:1093D00044F01CFBE3E706F50150C7F8F8450830F8
:1093E00056F092F9D7F8F80503681B689847A0F182
:1093F0000A035842584106F5005487F8E4055046E0
:10940000FBF756FE84F80491D7F8F80503681B684B
:10941000984794F80421014606F57C6041F062FE0D
:10942000404600214BF098FDD7F8F8153046FFF77D
:1094300075FFB4E70125B2E7FC820B083C830B08FB
:1094400073B505460A4801920E46FCF72FFA019AB9
:10945000044630B10146064802B0BDE87040FFF74F
:1094600079BF2846314640F0EFFB204602B070BD80
:10947000602600200148FFF7E3BF00BF6026002000
:10948000F0B5044604F5A04600F5905087B01430BE
:1094900036F0CAF8D6F8F8152046FFF73FFF04F576
:1094A000AC40443005F0DEFB04F5775010304EF050
:1094B00025FB04F5835018304EF09EFE04F58C51C8
:1094C00004F547500C3104F5866530306CF060FAD5
:1094D000284605F045FA04F5A640483048F054FC0B
:1094E00004F57950303059F095FC09F0DDF94FF46E
:1094F0000063036309F0D8F90AF04EFA04F58053CB
:109500008027C3F8E07F4FF48063C4F8BC3F00219C
:1095100004F551603AF016FE01212846C4F844745F
:1095200005F0B8F80423C4F8743104F5907010F015
:1095300043FA4FF40023C4F8B03B204604F54057EB
:10954000FFF748F804F52D5097F8D01138306DF03A
:10955000E5FC4EF039F94DF021FE04F5235024309E
:1095600065F02AFE04F58F5050F03CFD04F5AA404A
:10957000743006F061FD2F4B2F491B68986A036811
:109580004FF47A72DB6A04F5B7459847183504F54D
:1095900041506BF053F91A2229462046FFF7DAFEB4
:1095A0002046FFF787FE04F5BA4028301DF00CFF77
:1095B0004FF48073C6F81C3E204B0493204B059358
:1095C00006AB13E9060004F57C6041F0A7FB04F547
:1095D0000053204693F85111FCF768F91A2200282D
:1095E00014BF014629462046FFF7B4FE04F5065095
:1095F0000C309922292101904DF048FB9B22052136
:1096000001984DF043FB01984CF008FB0D48FFF723
:10961000E3FA97F9F430022B07D101230A488DF8B9
:109620000F300DF10F0139F02DFC012386F8F435D0
:1096300007B0F0BD58260020C59101086026002023
:10964000C1910108506100201859002070B50A4BE3
:109650001D68E869036800225B680C469847E86962
:10966000036821461B6901229847E869036821467F
:10967000DB68BDE8704018475826002000F57C6084
:1096800042F0E8B900F5405090F9F400831E5842CA
:109690005841704713B50446143000F0F1FE04F150
:1096A0002C0000F0EDFE04F1740070F059FD04F19F
:1096B000F40070F055FD4FF0FF331549C4F85031F8
:1096C000204638F0C9FD00230DF1070104F1280000
:1096D0008DF8073039F0D6FB01230DF1070104F1B5
:1096E00029008DF8073039F0CDFB0F230DF107016C
:1096F00004F125008DF8073039F0C4FB054B1A68DA
:1097000012B105486FF006F920461C6002B010BD8A
:1097100014850B08A486002064830B082DE9F0470C
:109720008CB003A937F0FEFF60B300210D2208A81A
:1097300007AF1C4CDFF87080DFF8709007910B26A4
:1097400094F0A0FF0697237ADFF864A08DF8143018
:10975000002554F825300493D8F80000E368B5B923
:109760000093C06A53461122394615F061FB00216F
:10977000B7EE000A03A838F02BFA35B1013E04F128
:109780001004E0D10CB0BDE8F0870125E1E70193BA
:109790000223009311224B463946C06A15F048FB5C
:1097A000E5E700BFB4850B0858260020C1830B08ED
:1097B000B8830B082DE9F74FD0F85431044683BB2A
:1097C000DFF88CA1074600F1740800F5AA750126A0
:1097D000721ED2B297ED070A0192404670F0E0FC8B
:1097E000FB69C8F83C304FF07E53C8F8483097F911
:1097F0002830019A013B5FFA86FB0E2B20D8DFE868
:1098000003F0133E4A5760691F1F1F1F1F1F891F48
:109810007A00D4F8543103B96361D4F8583103B9EC
:10982000E36203B0BDE8F08F4820019208F0B4FA7B
:10983000814618B1019A21466FF056FCC5F8009098
:10984000286890B103689B689847002874D14AF053
:1098500089FF3C4A3346032144F0D8F8286810B108
:1098600003685B68984700232B60022E07F11807F6
:1098700008F1800805F10405CBD00226A8E72820CE
:10988000019208F089FA81460028D7D0019A214632
:1098900070F04EFCD2E76820019208F07DFA814614
:1098A0000028CBD0FF23019A21466FF0BFFEC5E709
:1098B0006820019208F070FA81460028BED000238B
:1098C000F1E76820019208F067FA81460028B5D0D8
:1098D0000123E8E74420019208F05EFA814600285F
:1098E000ACD0019A21466FF0C1F9C9F800A000235D
:1098F000C9F84030A2E74420019208F04DFA8146B1
:1099000000289BD0019A21466FF0B0F90E4BC9F8A0
:109910000030ECE76020019208F03EFA8146002812
:109920008CD0019A21466FF0A1F9084BC9F800309C
:109930000023C9F8243081E72B68002B95D084F8E8
:109940004FB192E79E830B08FCC20C0874860B088B
:1099500030C50C0813B50446FFF7E0FE204638F08A
:1099600037F868B994F9283013B994F940303BB10D
:1099700001230DF1070120468DF8073039F0B0FAC8
:1099800094F90030002B08DD94F928302BB12046E3
:1099900002B0BDE81040FFF70DBF02B010BD0000DF
:1099A0000346406C012807D0032805D0986C012895
:1099B00002D0032818BF02207047000090F9003041
:1099C000002B0ADD012908D8182303FB010090F9B8
:1099D0002800003818BF01207047002070470000A1
:1099E00037B50446FFF7EAFF9FED0B0A0D4680B13D
:1099F00004EB81038DED010AD3F8540138B10368FB
:109A000001A9DB68984704EBC51484F865009DED57
:109A1000010A03B030BD00BF0000000070B504466D
:109A2000FFF7CCFF50B104EB8104D4F8540128B106
:109A30000368BDE870401B6911461847002070BDDF
:109A40002DE9F04F2DED028B90F90030002B83B003
:109A50000646894653DD2C4B1B68D86A03685B6851
:109A60009847044650B14AF07DFE284A062103B0CB
:109A7000BDEC028BBDE8F04F43F0C8BF9FED248AD8
:109A8000DFF890A0DFF890B0354606F14407B04605
:109A900021463046FFF792FF20B195F8643043B17C
:109AA00088ED068A8035043708F118083CBB01248C
:109AB000EEE7B9F1000F03D098F92630002BF1D171
:109AC000D7F81021631C01933AB94AF04BFE019B71
:109AD0005A46032143F09AFFE4E76EF04DFF00225F
:109AE000A5F87020A5F872200122A86685ED1B8AD2
:109AF0003A604AF037FE019B52460621EAE703B07E
:109B0000BDEC028BBDE8F08F58260020CC830B08FB
:109B1000000000000A840B08E3830B082DE9F043E2
:109B20002DED028B85B004460D46B0EE408AFFF75E
:109B300045FF98B304EBC119CF01D9F868306BB376
:109B40006EF01AFFD9F86830C01AB0F57A7F03D3E7
:109B5000B9F872300F2B0CD8E31993F86520002A5E
:109B600040F08C803C44B4F872300133A4F8723079
:109B700014E0B9F8703005F1010805F1100693B949
:109B80004AF0F0FD04EB86064346454A042143F0C3
:109B90003DFF032373603C440023A36605B0BDEC86
:109BA000028BBDE8F08307EE903AD9ED1B6AD4F83A
:109BB0005C21F8EEE77A86EEA77A8DED037ACAB3D8
:109BC00094F90230002B35DD07EE903AB2F90C2003
:109BD0009FED345AF8EEE75AF7EE007AE5EE857A13
:109BE000182101FB054506EE902AF8EEE66A95ED90
:109BF000066A67EEA67A37EE467A67EEA77AB0EE87
:109C0000C77AE6EEE67AF6EE006A67EEA67AF4EE3A
:109C1000C77AF1EE10FA0DD5B0EEC66AB5EEC06A9D
:109C2000F1EE10FA06DD4AF09DFD1F4A434604217D
:109C300043F0ECFE182003A900FB084004EB860665
:109C400039F0E4F8022373606368DB060ED54AF04E
:109C500089FD05460398F6F74FFC144ACDE900014B
:109C600043460621284643F0D1FE94E74AF07AFDA8
:109C70000F4A4346062143F0C9FE8CE7B3F8722031
:109C8000052A7FF66FAFD3ED1B7AB3F8702037EE5D
:109C9000880A013283ED1B0AA3F8702062E700BF37
:109CA0002C840B080AD7233C42840B086F840B08D2
:109CB00096840B0810B590F90030002B02460C4634
:109CC0001CDD90F84D31CBB9FFF778FEA8B1182113
:109CD00001FB042292F9243093B1022B0DD14620CE
:109CE0004DF08EF9DFED077AB0EEC00AB4EEE70A68
:109CF000F1EE10FA4CBF0120002010BD0020FCE75F
:109D00001846FAE7000000342DE9F8432DED028BE8
:109D100004460E46FFF752FEE8B104EB81090DB28E
:109D2000D9F85431BBB16EF027FE04EBC6174FEAE9
:109D3000C6183866D9F8540103685B69984770B152
:109D4000D9F85401036839469B69503198473B6DF7
:109D500087F86500FB64BDEC028BBDE8F8833146F3
:109D6000204697F86590FFF73BFE182303FB064358
:109D700093ED068ABB6E30EE488A87ED178A1BB1D9
:109D800031462046FFF7CAFEB9F1000F43D0DFEDA0
:109D9000447A9FED447A04EB080368EE277AD3ED0A
:109DA000166AE6EE877A182104EB080701FB0646DF
:109DB000C7ED167A96F9273083B3012B53D1DFED27
:109DC0003A8AF1EE487A05EB4505B4EEE88AC7ED2C
:109DD000157A04EBC505F1EE10FA95ED070A58BFA8
:109DE000F0EE687A27EE800A92F09CFB87ED130A6A
:109DF00097ED160AB4EEE80AF1EE10FA48BFF1EE5C
:109E0000408A95ED070A28EE800A92F08BFB4444C5
:109E100084ED140A9FE7F0EE487AC4E7B5EEC08AF5
:109E200005EB4505F1EE10FA87ED158A04EBC50543
:109E3000D8BF9FED1D8A95ED070A28EE000A92F023
:109E400071FB04EB0803D3ED167A83ED130AF5EEEC
:109E5000C07AF1EE10FAD8BFDFED137A95ED070A5C
:109E600027EE800AD1E7B0EEC88A05EB450587EDFD
:109E7000158A04EBC50494ED070A28EE000A92F057
:109E800051FBD7ED167A87ED130A94ED070AF0EE31
:109E9000E77A27EE800A92F045FB87ED140A5AE72D
:109EA0009A99993E3333333F0000000038B50A4693
:109EB0000446FFF783FD10B304EBC113CD0193F803
:109EC000653033B104EB8103D3F85431003B18BF44
:109ED0000123182101FB0242D2ED067AF0EEE77A67
:109EE000F5EEC07AF1EE10FA08DC2C4494F8640028
:109EF00020B992F92600003818BF0120184038BD5B
:109F000010B500210446FFF759FD18B12046FFF7B0
:109F1000CDFF50B101212046FFF750FD30B1204662
:109F2000FFF7C4FF003818BF012010BD0846FCE74A
:109F300010B50246FFF742FD20B102EBC11292EDCF
:109F4000140A10BDBFEE000AFBE7000010B5024680
:109F5000FFF734FD20B102EBC11292ED130A10BDE0
:109F6000BFEE000AFBE7000010B50246FFF726FD32
:109F700020B102EBC11292ED150A10BD9FED010A4E
:109F8000FBE700BF0000000010B50246FFF716FD1A
:109F900020B102EBC11292ED170A10BD9FED010A2C
:109FA000FBE700BF000000002DE9F04F2DED028B14
:109FB0008DB004466EF0E8FC9FED3C8ADFED3C8AF4
:109FC00080468946274625464FF0000B04F5AA7ABD
:109FD0005FFA8BF631462046FFF7F0FC002858D098
:109FE0005AF82B30002B54D06A462046FFF716FD56
:109FF00008B9CDED008A1D22002104A894F042FB8F
:10A00000A3238DF80430952331468DF80530204682
:10A0100072238DF80630CDF80780CDF80B908DF8BF
:10A020000F60FFF793FF20468DED040AFFF79CFFBA
:10A03000DDED007A8DED050A67EE887A2046FDEEAB
:10A04000E77A17EE903AADF81830FFF79DFF10EE63
:10A05000103A2046CDF81A30BB69CDF81E30FFF714
:10A0600029FE31468DF822002046FFF71FFFD5F864
:10A07000BC300993D5F8C0300A9394F84E318DF86E
:10A0800023008DF82C3041F01BFD292201A940F05E
:10A0900069FE18378035BBF1000F04D00DB0BDEC60
:10A0A000028BBDE8F08F4FF0010B91E70000C84232
:10A0B00000000000F8B590F90030002B04464DDD9B
:10A0C0000021FFF721FE01212046FFF71DFE94F934
:10A0D0000030002B0DDD94F9403053B14AF042FBC3
:10A0E000012105462046FFF723FF1D49284643F07E
:10A0F00003FF667894F84E7131462046FFF7D6FE8E
:10A10000054668B901462046FFF7D0FE28B901216F
:10A110002046FFF7CBFE28B1012584F84E5101E01F
:10A1200084F84E6120466EF07FFF94F84E31BB42BA
:10A1300004D041F0C5FC5A2141F0FEFBD4F8503167
:10A1400001330BD041F0BCFCD4F8501141F082FC3B
:10A1500020B12046BDE8F840FFF726BFF8BD00BF9C
:10A16000B0840B08014B1868704700BFA48600201C
:10A17000002070477047000001207047436AC3B158
:10A18000B0F850301BB9436D0B600120704707EEEB
:10A19000903AD0ED136AF8EEE77A002386EEA77ABC
:10A1A00081ED007AA0F85030002380ED157AC36469
:10A1B000EBE718467047000070B504463FF008FA18
:10A1C0000022222105463FF05FF8606220B30023A1
:10A1D0001A461946062014F0A5FA014620466EF0EC
:10A1E0007FFD002222212846666A3FF06DF8014675
:10A1F000304614F0F5FC94F82020E369182101FBA7
:10A200000233002283F82420E36994F8202003EB32
:10A21000C213012083F8640070BD000010B5034B29
:10A22000036004466EF032FD204610BD74860B08B4
:10A2300010B50446FFF7F2FF204607F0B5FD2046B3
:10A2400010BD000073B590F8455004463DB301239E
:10A2500080F846300DF10601002390F828008DF8B3
:10A2600006308DF8073007F019FA18B9002528468E
:10A2700002B070BD94F829000DF1070107F00EFA45
:10A280000028F3D09DF806509DF8073043EA0513E7
:10A2900094F84450DBB2EB1A5D425D41E7E790F879
:10A2A0003830FBB990F82830413B192BDFD890F8B3
:10A2B0002930413B192BDAD800F12A0617493046DC
:10A2C000F7F7DEF810B984F84850D0E71449304663
:10A2D000F7F7D6F818B9012384F84830C7E784F8AF
:10A2E0004750C4E790F8482042B9012BBFD1294616
:10A2F000283095F0EDFC84ED100AB8E7012AB6D1BC
:10A30000072BB4D12946283095F0E2FCDFED057A21
:10A3100020EE270A84ED0F0AA9E700BF64860B0828
:10A3200068860B08E4388E3E242970B504460D4635
:10A3300040D016DC0A291ED00D291CD094F83730E5
:10A340000D2B9FBF5A1C1B1984F8372083F8285007
:10A3500094F8450090B994F844104D4084F8445066
:10A360000DE02A2907D02C29E8D190F8443083F059
:10A370002C0380F8443094F846600EB1002070BD84
:10A3800094F84730002BF9D094F837302344204616
:10A3900083F82860FFF756FF94F8383084F8376068
:10A3A000013384F83830A5F12A035D425D4184F819
:10A3B0004550E4E700204FF0807384F8380084F8BB
:10A3C00037006364DBE700002DE9F0412DED028BDF
:10A3D000436A0446884623B90020BDEC028BBDE8E1
:10A3E000F0816EF0C9FA0546606A9FED248A036821
:10A3F0005B699847002687B23BB2002B26DD606A76
:10A4000003689B699847431CE6D041B22046FFF79A
:10A410008BFF50B194F84830E565012B08D1D4ED9D
:10A420000F7A013638EE278AB6B2013FBFB2E3E7B2
:10A43000D4ED137A94ED107AB4F8503077EE877A31
:10A440000133C4ED137AA4F85030EEE756B9A36D8A
:10A45000C8F80030E06D281AB0F5FA6F2CBF002064
:10A460000120BAE707EE906AF8EEE77A88EE277ADD
:10A4700088ED007A84ED167AECE700BF000000005A
:10A4800010B50349044637F0E7FE204610BD00BF73
:10A4900094860B08F0B52DED048B91B004466D4603
:10A4A000284607F049F994F8BC33002B72D004F524
:10A4B0007A730FCB85E80F0094F8F833D4EDEC8A6B
:10A4C00094EDED8A94EDEE9A002B63D094F8D0339E
:10A4D000002B5FD02D22002104A8D4F8C073D4F83B
:10A4E000C463D4F8C853D4F8CC4394F0CBF8A32376
:10A4F0008DF8103095238DF8113046238DF81230E9
:10A500006EF042FA9FED250A9FED257ACDF81710DF
:10A5100068EE807ACDF8130067EE877AFDEEE77A71
:10A5200017EE903A68EE007A29EE000A67EE877A15
:10A53000ADF81B30FDEEE77A20EE070A17EE903AF1
:10A54000ADF81D3017F03AFEDDED017A9FED157A7A
:10A55000CDF82D70BCEEC00AF8EEE77A10EE103A96
:10A5600067EE877AADF81F3017EE903ACDF82130BC
:10A57000029BCDF82530039BCDF82930CDF8316012
:10A58000CDF83550CDF8394041F09AFA2D2204A982
:10A5900040F0E8FB11B0BDEC048BF0BDE02E65424D
:10A5A0000000C8420AD7233C30B52DED028B8BB09A
:10A5B000044624220D4601A8002194F063F8A32349
:10A5C0008DF8043095238DF8053048239FED1F8AC0
:10A5D0008DF806306EF0D8F9D4ED817A2B68CDF87D
:10A5E0000F3067EE887A95ED020ACDF80B1017EE62
:10A5F000903AD4ED827ACDF8133067EE887A6B68A2
:10A60000CDF8173017EE903ACDF80700CDF81B3093
:10A6100017F0AAFD10EE103A94ED830ACDF81F3022
:10A6200020EE080A17F0A0FD10EE103ACDF8233006
:10A6300094F80C338DF8273041F042FA242201A916
:10A6400040F090FB0BB0BDEC028B30BDE02E6542BC
:10A6500030B587B014460D4618220021684694F0A4
:10A6600011F8A3238DF8003095238DF8013049238C
:10A670008DF802306EF088F9A3680393E3680493C1
:10A680006368CDF807100593CDF803008DF80B50E3
:10A6900041F016FA1822694640F064FB07B030BD5D
:10A6A00010B58EB0044602A807F046F802A920466D
:10A6B00001F00EFB002845D001F048FD694601F08D
:10A6C0009FF91F22002106A893F0DCFFA3238DF839
:10A6D000183095238DF819304A238DF81A306EF012
:10A6E00053F9DDED037A9FED1B7A049BCDF82330FF
:10A6F000F8EEE77A059BCDF8273067EE877ACDF83C
:10A700001B0017EE903ADDED007ACDF82B30F1EE1C
:10A71000677A17EE903ACDF81F10204601A9CDF8C0
:10A720002F3000F083FC78B1DDED017AF1EE677A2D
:10A7300017EE903ACDF8333041F0C2F91F2206A946
:10A7400040F010FB0EB010BD41F0BAF9DFED027A17
:10A75000EEE700BF0AD7233C5241C07F10B594B04A
:10A760004FF07E5303A903930023044606930593F9
:10A77000049300F061FA17F085F890F813330C2277
:10A7800002FB030004F5577100F5C4701AF08CFC4D
:10A790003322002107A88DED000ACDED010A8DEDD1
:10A7A000021A93F06FFFA3238DF81C3095238DF8C8
:10A7B0001D30CC238DF81E306EF0E6F8D4F814333B
:10A7C000CDF82730D4F81833CDF82B30D4F81C331B
:10A7D000CDF82F30009BCDF83330019BCDF83730CA
:10A7E000029BCDF83B30039BCDF83F30049BCDF866
:10A7F0004330059BCDF84730069BCDF82310CDF8AC
:10A800004B30CDF81F0041F05BF9332207A940F02F
:10A81000A9FA14B010BD00000023036043608360F8
:10A82000C360036143618361C361036270470000D9
:10A8300090F8C432B02202FB030390F8082393F887
:10A84000A13012B1012B28BF012318467047000028
:10A850002DE9F04F04468BB04FF0000A0D461EF074
:10A860009FFE84F814A204F506704FF07E576DF039
:10A8700039FA4FF47A73A4F8623284F86852C4F853
:10A880004872C4F84C72C4F8507204F51B7000256D
:10A8900006F052FF04F52B790323C4F8803204F547
:10A8A0003476C4F89452C4F89852C4F89C52C4F850
:10A8B000A052C4F8A452C4F8A8524846FFF7ACFF0F
:10A8C00004F5487B3046FFF7A7FFC4F81453C4F8DB
:10A8D0001853C4F81C535846FFF79EFFC4F844535E
:10A8E000C4F84853C4F84C53C4F85053C4F85453F4
:10A8F000C4F85853C4F85C53C4F86053C4F86453A4
:10A90000C4F86853C4F86C53C4F87053C4F88C533B
:10A91000C4F89053C4F89453C4F8A853C4F8A4538B
:10A92000C4F8A053C4F8B053C4F8B453C4F8B8532F
:10A93000C4F8CC53C4F8C853C4F8C453C4F89C73C7
:10A94000C4F8C07304F5757006F0F6FE04F57A706D
:10A9500006F0F2FE04F58063C4F8FC531D6004F5B4
:10A96000816304F583601D605D609D6006F0E4FE18
:10A9700004F22C4304F264481D605D609D60684BE6
:10A98000C4F83C3404F50D73C4F8403404F50E7378
:10A99000C4F8443404F50F73C4F8483404F5107354
:10A9A000C4F84C3404F24523C4F8503404F5117350
:10A9B000C4F8543404F58B6340461D605D609D60AF
:10A9C000FFF72AFF04F59160FFF726FF04F5976370
:10A9D00004F23C421D605D609D6004F2C44304F2D9
:10A9E000A4501D605D609D6004F59A631D605D600C
:10A9F0009D6004F2DC431D605D609D6004F2EC43E9
:10AA00001D605D609D6004F2FC431D605D609D60A3
:10AA100004F5A463C2F8D470C2F8D8701D605D60FC
:10AA20009D6004F22C531D605D609D6004F5A96378
:10AA30001F605D6004F26C531D605D609D6004F5F5
:10AA4000AF631D605D609D6004F5B2631D605D6075
:10AA50009D6006F071FE04F2B45324221D605D6017
:10AA600004F2BC5351461D605D6004F2C45340467D
:10AA70001D605D6093F006FE04F2E450C8F820709B
:10AA8000C8F81070C8F80070FFF7C6FE04F5C1637F
:10AA900004F5C7601D605D609D6004F214631D6075
:10AAA0005D609D6004F5C4631D605D609D6004F29F
:10AAB0002C631D605D609D6006F03EFE194B1A49D7
:10AAC0001C60204637F0C8FB51462422584693F0BC
:10AAD000D9FDC4F84073C4F83073C4F8207304F58A
:10AAE000257207CA04F5287383E80700484694EDE9
:10AAF000AA1AD4EDA90A94EDA80A18F0CFFB35469E
:10AB0000494668466E4618F0EBFA0FCE0FC50FCED9
:10AB10000FC533682B6020460BB0BDE8F08F00BF37
:10AB2000AC890B08A886002068880B0810B504467D
:10AB300088B001F095FB94F93232012B02D12748FD
:10AB400004F040FD022B0AD1032384F8323204A919
:10AB5000012304F111008DF8103038F083F994F8D6
:10AB6000323284F8903204F23C4001F02FFB94F929
:10AB70003132642B30D1652304A904F231208DF8E1
:10AB8000103038F0ADF904A9204636F003FE18B3B2
:10AB900004238DF818300023CDE9013303930F23EC
:10ABA0000593694604A836F0C7FF059B28B108AA9B
:10ABB00002EB8302009942F8581C0133112B0593D4
:10ABC000EFD966F07DF99DED031ADDED020A9DEDEA
:10ABD000010A652166F032F908B010BD54870B08F0
:10ABE00070B500F5257600F528758CB00446314621
:10ABF00028461AF0F9F9E0B996E8070085E8070059
:10AC000004F52B7194EDAA1AD4EDA90A94EDA80AC3
:10AC10000191084618F042FB02AD019902A818F014
:10AC20005FFA0FCD04F534740FC40FCD0FC42B6839
:10AC300023600CB070BD00000B4600F5487118464B
:10AC400019F0F6B984B000F5487004B018F088B96E
:10AC500013B540F2411200F50671044601A813F045
:10AC600007FF04F23C4001F0C1FC20461EF0F0FE5C
:10AC700001A813F01FFF02B010BD0000F8B50B686B
:10AC8000C0F804324B68C0F808328B68C0F80C3248
:10AC900001F10C0607460C4600F548750FCE0FC5AE
:10ACA0000FCE0FC533682B6004F1300207CA07F5D9
:10ACB000457383E8070004F13C0207CA07F55173A6
:10ACC00083E8070004F1480207CA07F5547383E8D4
:10ACD0000700543494E8070007F5577383E807002A
:10ACE000384601F0D1FB3846BDE8F84001F0B4BB6E
:10ACF00013B5044600F23C40019003F06DF804F5F2
:10AD0000BB610198009102F0C5FB0099204602B09A
:10AD1000BDE81040FFF7B2BF4A78064BC2F34012BD
:10AD20001A754A78C2F380125A750A78C2F3001273
:10AD30009A7570473D87002013B540F2F52204460E
:10AD400000F5067101A813F093FE002104F23C40C7
:10AD500001F0BEFE94F8603223B120461FF080F867
:10AD600084F8600201A813F0A5FE02B010BD000037
:10AD700038B590F80C3305460C462BB1032B0BD09D
:10AD800095F86832DB070CD405F5C7630FCB84E870
:10AD90000F0095F8480603E01EF0B0FE0028EFD043
:10ADA00038BD0020FCE7000000F23C4090ED350A81
:10ADB0007047000000F23C4090ED360A70470000FA
:10ADC00010B490F80C230C462AB1032A0AD00020B4
:10ADD0005DF8044B704700F5B26007C884E80700CF
:10ADE0000120F5E75DF8044B1EF070BE90F8840377
:10ADF000431E58425841704738B590F80C330D4601
:10AE00008BB900F23C4001F063FC044610B9002409
:10AE1000204638BD01F0B0FBD5ED007A27EE800A60
:10AE200085ED000AF4E7D0EDE07AC1ED007A90F804
:10AE30007C43002CEBD090EDDE7ADFED086AB4EEB7
:10AE4000E67AF1EE10FAF7EE006AB8BFB0EE667A75
:10AE500067EE877AC1ED007ADAE700BF00000034C0
:10AE600090F80C33032B01D11EF0A0BD00207047D9
:10AE700010B490F80C43032C03D15DF8044B1EF082
:10AE8000A1BD00205DF8044B7047000090F80C2332
:10AE9000032A01D11EF0DCBE00F23C4002F07AB879
:10AEA00030B590F80C3385B004460D468BB1032BBA
:10AEB00018D004F525701AF0D1F8284601A98DEDB7
:10AEC000010ACDED020A8DED031A19F067FC01208D
:10AED00006E000F23C4001F0A5FB0028E9D100208B
:10AEE00005B030BD90F86032002BF8D01EF098FE0F
:10AEF000DFE700007FB590F80C2332B1032A4FF052
:10AF0000000309D0039304930CE000F23C4007B027
:10AF10005DF804EB01F060BC03A90393049305936F
:10AF20001EF03AFD9DED030ADDED040A07B05DF861
:10AF300004FB000007B590F80C3333B100F57F70C7
:10AF400003B05DF804EB19F0D5BD00F23C4001F010
:10AF500043FC68468DED000ACDED010A19F0CAFDEB
:10AF600003B05DF804FB000090F80C03003818BF34
:10AF70000120704708B590F80C23032A05D0BDE8DE
:10AF8000084000F23C4001F011BC1EF005FD01201C
:10AF900008BD000010B590F80C230C461AB1032A26
:10AFA00007D0002010BDBDE8104000F23C4001F089
:10AFB000A1BB1EF017FD012084ED000AF2E700009E
:10AFC00030B590F80C3385B005460C4623B1032B01
:10AFD00009D0002005B030BD00F23C4005B0BDE80E
:10AFE000304002F087BA002302A9029303931EF0B7
:10AFF000BBFC0028EDD001A928461EF0C1FC0028AA
:10B00000E7D0029B2360039B6360019BA360E1E7A1
:10B0100090F80C231AB1032A05D00020704700F2E3
:10B020003C4002F09BBA1EF09FBC000090F80C233D
:10B030001AB1032A05D00020704700F23C4002F00C
:10B040007FBA1EF09DBC000090F932323BB990F8F7
:10B05000683213F0010F14BF032000207047032053
:10B0600070470000F7B50446FFF7EEFF05460028DD
:10B0700062D0032839D194F860326BB394F8683207
:10B08000D8072BD501A920461FF014F8BDF80430CD
:10B09000002B18BF002594F8146206F0FD06012E5F
:10B0A0004AD10023032D019307D101A920461FF0A7
:10B0B0000DF820461EF0E4FD064604F23C4002F086
:10B0C000CBFA08B994F809039DF80430D90703D5E1
:10B0D0005A0701D59F0632D400252DE020461EF0E8
:10B0E000B3FB002808BF0025D5E70025D3E713F000
:10B0F000020F2EE094F9443223B99DF80430DB09A5
:10B100002FD0E9E7002EF8D00FF08EFFFFF790FB6D
:10B11000022807D99DF805309806DDD59DF8043042
:10B12000D906D9D5FB6A93F89C30002BE5D118E0FD
:10B13000DA0601D41B0718D5284603B0F0BD002855
:10B14000FAD094F80923B4F94C36002ACFD013F082
:10B15000010FF1D1154B1F68FB6A93F89C30002B4F
:10B16000C8D19DF804309C07E2D407F09DFB07F09E
:10B1700099FA0028B0D10FF057FFFFF759FB0228CA
:10B18000AAD90FF051FF90F8C432B02202FB03009D
:10B1900090ED2F7AF0EE007AB4EEE77AF1EE10FA45
:10B1A0009AD59DF80530DB09C6D195E758260020D1
:10B1B0002DE9F04790F8603292B00446002B00F081
:10B1C000948020461FF0C6F82046FFF74BFF032867
:10B1D0007BD104F548780027414620460097019727
:10B1E00002971EF0F3FC694620461EF0E5FC009B2A
:10B1F000C4F80432019BC4F80832029BC4F80C3234
:10B20000204601F041F9204601F026F916F03AFBFC
:10B21000054620461EF09AFB0028A8BFC6B203AA26
:10B220004FF0FF312046BCBF95F8129395F8136399
:10B230000397A8BFB146049705971EF0E1FB03A84A
:10B2400019F00CFF4FF00C0A0AFB095084EDD10AEB
:10B25000C4EDD20A84EDD31A04F5517100F51170D2
:10B2600019F00CFF04F557770AFB065584EDC50A63
:10B27000C4EDC60A84EDC71A3A464FF0FF312046A6
:10B2800005F5C4751EF0D0FB95E8070006AE86E80C
:10B2900007003946304619F057FF04F52B72414636
:10B2A00009A817F0ADFE314609A817F02BFE09A931
:10B2B000204684EDD40AC4EDD50A84EDD61A1EF0DA
:10B2C00005FF09A92046FFF727FD94F84E36002B0D
:10B2D0003AD109A806F030FA09A920461EF01AFC56
:10B2E00090B3012384F84E362EE0D0F864321BB9B7
:10B2F0006DF042FBC4F86402154B1B68D86A036802
:10B300005B68984788B16DF037FBD4F86432C01A97
:10B31000B4F86232984204D920461EF0A1FD84F8A8
:10B32000600294F860327BB14BE76DF025FBD4F8F6
:10B330006432C01A41F287339842E4D840F0C0FB2F
:10B3400040F0A4FB0028DED112B0BDE8F08700BFBA
:10B350005826002090F80C3323B1032B4FF0000047
:10B3600007D0704790F93222032A04D10A700120D5
:10B3700070470870FBE718467047000073B50D462C
:10B380000DF107010446FFF7E5FF064628B19DF8D9
:10B3900007302BB1032B09D00026304602B070BD18
:10B3A00004F5C7630FCB85E80F00F6E72946204672
:10B3B0001EF0A4FB94F86062EFE700007FB50E4634
:10B3C0000DF103010446FFF7C5FF054618B9002536
:10B3D000284604B070BD9DF8033083B1032B16D00E
:10B3E00004F5257019F03AFE01A930468DED010AE9
:10B3F000CDED020A8DED031A19F0D0F9E8E73146D8
:10B4000004F23C4001F00EF90028E9D1DFE794F89E
:10B410006032002BDBD0314620461EF001FCDFE716
:10B4200037B50D460DF107010446FFF793FF28B12C
:10B430009DF8073023B1032B0FD0002003B030BD9F
:10B4400004F5BB631B682B6004F2DC5304F5BC6499
:10B450001B686B602368AB60F0E7204629461EF04E
:10B46000ABFB94F86002E9E710B50446FFF7ECFD8A
:10B4700018B1032807D0002010BD04F23C40BDE8FD
:10B48000104001F0F9B894F86032002BF3D0204658
:10B490001EF0DAF90028EED094F8143203F0FD0320
:10B4A000012BE9D194F80C03C31E58425841E3E73D
:10B4B00010B50446FFF7C8FD80B1032810D194F8F9
:10B4C000600250B16DF058FAD4F86432C01A44F6F4
:10B4D0002063984294BF0020012010BD0120FCE7AA
:10B4E0000020FAE708B50246FFF7AEFD032804D1B5
:10B4F00010461EF0EBFD012008BD0020FCE7000017
:10B5000030B585B004460191FEF72CFE0199054641
:10B5100010B9002005B030BD0191FEF7CBFB0199B9
:10B520000028F6D02846FEF7C1FC0028F1D0B4F878
:10B530004C365907EED494F80933002BEAD00B4A65
:10B540001268D26A92F89C506DB103A92046FFF7A9
:10B55000C9FF30B19DF80E309A07DBD5C3F38000E8
:10B56000D8E72846D6E71846D4E700BF582600207B
:10B570002DE9F04190F80C338CB00027032B0646E0
:10B580000C46154600970197029719D11EF0DEF977
:10B590006A4680464FF0FF3130461EF045FAB8F15A
:10B5A000FF3FA760676027600DD116F06BF92B464F
:10B5B00090F81313224615F0D9F90CB0BDE8F081CC
:10B5C0004FF0FF38EBE716F05DF92B4622465FFAA5
:10B5D00088F115F0CBF995ED000A684619F07AFD6F
:10B5E00003A920468DED051A8DED030ACDED040A61
:10B5F00019F0AAFD06F52B7206F5487103A817F09D
:10B60000FFFC214603A817F07DFC84ED021A84EDAF
:10B61000000AC4ED010A95ED007ADFED037AA7EE8A
:10B62000271A84ED021AC8E70AE81C411FB5DFEDAE
:10B630000B7A20EE270A0C461946094BCDE9004249
:10B64000BDEEC00A18688DED020A064B9DF8182061
:10B65000C06A13F0EDFB04B010BD00BFE02E6542E0
:10B660005826002068870B082DE9F0472DED028B46
:10B6700092B0002504460F464FF07E5A00F54871FF
:10B6800006A89046CDF818A009950895079518F0DA
:10B69000CFFC07F009F907F005F881462046FFF7CF
:10B6A000D3FC032803D094F80C33032B4FD19FED28
:10B6B000558ADFED558A00262379F2B2934247D9A5
:10B6C0000AAA71B22046CDF828A00D950C950B95CD
:10B6D0001EF086FA0AA906A819F0D2F8B4EEC80A34
:10B6E000F1EE10FA0DDD494ACDF800803B4648499D
:10B6F0002046FFF79BFF002012B0BDEC028BBDE897
:10B70000F0870AA906A803950495059519F0A2F8F3
:10B7100003A90EA88DED0E0ACDED0F0A8DED101ABE
:10B72000CDED111A18F00AFEB9F1000F0DD09DED04
:10B73000050AB0EEC00AB4EEE80AF1EE10FA04DD34
:10B74000344ACDF800803B46D1E70136B4E7002308
:10B7500094F8686216F0010001D0012BCCD104F2FC
:10B76000E4510AA8CDF828A00D950C950B9518F07A
:10B770005FFC0AA906A819F083F8DFED227AB4EE7F
:10B78000E70AF1EE10FA05DD204ACDF800803B46CD
:10B790002149ADE72046FFF757FC03282DD120466D
:10B7A0001EF062FA94F86832DB0728D438BB0AA985
:10B7B00006A803950495059519F04CF803A90EA861
:10B7C0008DED0E0ACDED0F0A8DED101ACDED111A8B
:10B7D00018F0B4FDB9F1000F11D09DED050ADFEDB1
:10B7E0000A7AB0EEC00AB4EEE70AF1EE10FA06DD0E
:10B7F000084ACDF800803B46CAE70020D2E7012086
:10B800007AE700BFC2B8323EC2B8B23E94870B0896
:10B810009F870B08B6DC0B08A4870B082DE9F743BC
:10B820001446054688460193FFF71EFE019A074617
:10B8300038B92448244B00682146C06A13F0F8FA4E
:10B84000019A019221462846FFF70EFF064630B3C3
:10B850002846FFF7F9FB95F80C33019A83420DD087
:10B8600007F022F806F01EFF019A38B1174B154871
:10B8700000682146C06A13F0DBFA10E02846FFF7A3
:10B88000E3FB18B103280FD0114BF0E713464146F4
:10B89000224605F23C4000F003FF00B107B9002644
:10B8A000304603B0BDE8F08395F86092B9F1000F1F
:10B8B00001D1084BDBE713464146224628461DF0DE
:10B8C000D3FFEAE758260020A8870B08B4870B08A7
:10B8D000E4870B08D3870B0890F80C33032B01D1B6
:10B8E0001EF00ABC0020704737B5054600F506710A
:10B8F00040F6033201A813F0BBF82846FFF7A4FB7B
:10B90000044640B103280AD0002401A813F0D2F85D
:10B91000204603B030BD28461EF0B4F8F5E72846AF
:10B920001EF0B0F80446F0E708B50246FFF78CFBBE
:10B9300010B1032806D008BDBDE8084002F23C4023
:10B9400000F064BEBDE8084010461EF0CBBB00000E
:10B950000B4610B411462BB1032B09D000205DF823
:10B96000044B70475DF8044B00F23C4000F064BEAD
:10B970005DF8044B1EF0CEB813B50446FFF764FB28
:10B980000A46014620460192FFF7E2FF70B9084BD4
:10B99000019A1B68DB6A93F89C0038B194F80C1389
:10B9A000204602B0BDE81040FFF7D2BF02B010BD84
:10B9B0005826002037B504460D4640F2B25200F535
:10B9C000067101A813F054F8294620461EF0C0F86D
:10B9D00094F80C33032B054610D148B104F583616C
:10B9E0002046FFF7C9FF84F82804204600F0A4FD94
:10B9F00001A813F05FF8284603B030BD0025F7E733
:10BA000070B590F87C32DB0786B004460D460CD446
:10BA100002F08CFF437C242202FB0300D0ED0B7A62
:10BA2000F1EE677AC5ED007A3BE002A805F084FEEE
:10BA300001A92046FFF7FAFAE8B90FF0F5FA94F9F0
:10BA40004432022B0646E3D1FEF7F2FE0228DFD98C
:10BA500096F8C4029FED147AB02303FB0066D4F875
:10BA60007032D6F8B0209B1A07EE903AF8EEE77ADB
:10BA700067EE877AD6E702A92046FFF77DFF002808
:10BA8000DBD0D4F87022039BDFED076A9DED017ACD
:10BA90009B1A07EE903AF8EEE77AA7EEE67A85ED84
:10BAA000007A06B070BD00BF0AD7233CF0B50C4643
:10BAB00087B000F50671064640F6863201A812F0FE
:10BAC000D7FFA36853B9E36843B9636833B9002764
:10BAD00001A812F0EFFF384607B0F0BD204605F090
:10BAE00001FF0028F3D094E80F0002AD85E80F00B5
:10BAF0000021284605F0B8FE07460028E7D096F852
:10BB00007C32DB0704D43FF0DBFF19213FF014FF48
:10BB100095E80F0006F51B7C8CE80F0096F87C3248
:10BB200043F0010386F87C32304600F005FD48F012
:10BB300019FE462149F010FA48F014FE452149F05B
:10BB40000BFA054BA2681B68DB6A1A61E2685A614E
:10BB500062689A61BCE700BF5826002038B5144BD4
:10BB60001B68DD6A2B6804465B6828469847F0B17D
:10BB70002B690BB96A69D2B1C4F874326B69C4F825
:10BB80007832A969002204F51B7005F0DBFD94F8FA
:10BB90007C3223F0030343F0030384F87C3248F043
:10BBA000E1FDBDE83840034A062141F02FBF38BD12
:10BBB00058260020F8870B0810B588B00446059376
:10BBC000FFF742FA0328059B4FF000000AD10690C8
:10BBD000079006A802900B9801900A9800902046C2
:10BBE0001EF028F808B010BD38B50446FEF7BAFAC2
:10BBF0000546D0B194F80C33032B03D095F84E4191
:10BC0000204638BD20461DF06DFFFF280446F5D0C4
:10BC100001462846FEF74AF90028EFD0214628467B
:10BC2000FEF748F80028E9D0EAE70446E8E7000014
:10BC300008B590F80C33032B05D015F023FE90F9CE
:10BC40001203C0B208BD1DF081FE431CF9D1F4E718
:10BC500008B590F80C3383B1032B03D1BDE808403D
:10BC60001DF06CBE3EF038FA40F6ED424FF4801104
:10BC70003EF0EAF94FF0FF3008BD1846FCE700003F
:10BC800090F80C33032B01D11EF0B0BC70470000BC
:10BC900090F80C33032B01D11DF034BD7047000028
:10BCA0001DF0BABD10B5044620F06CFD2046FEF72D
:10BCB000F1FB2046BDE81040FEF7F2BC90F80C33D3
:10BCC0000BB1032B01D11EF00DBD00207047000009
:10BCD00030B500F5757304460D460FCB85E80F00AF
:10BCE00094F8E40330BD00007FB5054668460E4673
:10BCF00005F022FD95F87C32DB0703D400242046B2
:10BD000004B070BD69462846FFF7E2FF04460028EC
:10BD1000F4D0694605F51B7005F0F4FE86ED000AC7
:10BD2000C6ED010AEBE70000D0F880330B6090F815
:10BD30007C037047D0F888330B6090F88503704718
:10BD400030B500F5677304460D460FCB85E80F004C
:10BD500094F8AC0330BD000030B500F583630446B1
:10BD60000D460FCB85E80F0094F8280430BD000085
:10BD700010B500F22C4203460C4607CA84E80700BF
:10BD800093F8380410BD00002DE9F0432DED028B2F
:10BD90008BB005460E461746FFF726FF0146804644
:10BDA0002846FFF7ADFB0446002848D0FEF7DAF935
:10BDB0004146FEF7BDF886ED000A95F93032002BBA
:10BDC0003ADD0FF031F9FEF733FD012834D90FF0D9
:10BDD0002BF990F8C432D5EDDE7ADFED5D8A96ED71
:10BDE000000AB02202FB030095F93032D0ED2F0A91
:10BDF00007EE103AF4EEE87AB8EEC77AF1EE10FAF0
:10BE0000B7EE008AB8BFF0EE487A37EE201A20EE7F
:10BE1000270A70EEC70A40F2B63016F03BFAD5EDAD
:10BE2000DE7AF4EEE87AF1EE10FAB8BFF0EE487A76
:10BE300080EE277A86ED007A01233B7003E095F8C7
:10BE4000083333B9387020460BB0BDEC028BBDE827
:10BE5000F08395F80C334FF00009CDF80490CDF83D
:10BE60000890CDF80C9043B1032B10D0CDF8109072
:10BE7000CDF81490CDF818907CB902233B7032466F
:10BE8000414605F23C4001F0ABFB0446DBE701A96B
:10BE900028461DF01BFE0446E8E795F80C33002BFE
:10BEA000EBD004A92846FFF763FF04460028E4D03E
:10BEB00001A904A819F0F8F807A8CDED080A8DED3E
:10BEC000091A8DED070A19F003FD04A8B0EE408AA7
:10BED00019F0FEFC95F93032002B30DD07EE903A78
:10BEE000F8EEE77A4FF47F7070EE670A37EE801A4B
:10BEF000F5EEC00AF1EE10FA48BFDFED160AF4EED7
:10BF0000410AF1EE10FAB0EE480AC8BFB0EE601A6E
:10BF100016F0C0F9B0EE408AD5EDDE7A9FED0C7ACE
:10BF2000F4EEC77AF1EE10FAB7EE007AB8BFF0EE91
:10BF3000477A88EE277A032386ED007A7DE7B5EE0F
:10BF4000C08AF1EE10FA48BF9FED028AE4E700BF15
:10BF5000000000340000000010B50446FFF768FE42
:10BF600084F80D032046FFF763FE84F80E03204695
:10BF7000FFF75EFE84F80F032046FFF769FE04F525
:10BF80005A7184F810032046FEF71AFF84F87403F0
:10BF900000F0F2FA04F5617284EDDE0A04F56071D6
:10BFA0002046FFF7F1FE04F5627184F87C03204619
:10BFB000FEF722FF04F5637184F885032046FEF73F
:10BFC0004FFF04F5677184F898032046FEF768FF79
:10BFD00004F56C7184F8AC032046FFF721FA04F5F0
:10BFE000707184F8BC032046FFF7E8F904F5757119
:10BFF00084F8D0032046FEF7BBFE04F57A7184F87E
:10C00000E4032046FFF7BAF984F8F8032046FEF768
:10C0100071FF04F5806384EDFF0A2046C3ED000A3A
:10C02000FEF788FF04F2044383ED000A04F2144291
:10C0300004F581612046FFF79BFA04F583612046F1
:10C04000FFF79AFC04F22C4184F828042046FEF7FE
:10C0500091FF84F8380410BD37B50D46044600F052
:10C06000FFF81DB915F00EFC14F0B0FB4FF4BE72D2
:10C0700004F5067101A812F0FBFC94F869322BB9A3
:10C080002046FFF76BFD012384F86932224B1D68BF
:10C09000A86A03689B6998472046FEF7A1FD2046E1
:10C0A000FEF726FE204600F079FA2046FFF780F8DA
:10C0B000286B30B10368D4EDD20ADB6894EDD10A65
:10C0C0009847D4F8100208B16EF0B8FF204600F08F
:10C0D0007DF82046FEF7C6FF94F8903284F80C03F2
:10C0E00083420ED084F8900298B10C4D0C4B03287B
:10C0F00008BF1D4648F036FB0A4A2B46062141F090
:10C1000085FC2046FFF728FF01A812F0D3FC03B0FE
:10C1100030BD054DEEE700BF58260020CF3F0B088D
:10C120009F870B0810880B08A4870B08D0EDDE7AD8
:10C130009FED057AF4EEC77AF1EE10FAB7EE000A39
:10C14000A8BFB0EE670A704700000034014B1868C2
:10C15000704700BFA88600204FF0FF3070470000F6
:10C160000120704770470000002070470020704792
:10C1700070470000704700000020704700207047A3
:10C180000020704700207047002070470020704753
:10C1900000207047012070470368D3F89430184797
:10C1A0000020704700207047002070470020704733
:10C1B0000020704700207047002070470020704723
:10C1C0000020704700207047704700007047000053
:10C1D00008B515F057FB90F8130308BD08B515F026
:10C1E00051FB90F8120308BD30B52DED028B9FED89
:10C1F0001A1ADFED1A0A91ED000A87B005462D20C4
:10C200000C468DED011ACDED000A16F043F89DEDB8
:10C21000011ADDED000AF0EE408A2E2094ED010AAD
:10C2200016F038F89DED011ADDED000AB0EE408AF7
:10C230002F2094ED020A16F02DF803A905F52570BC
:10C24000CDED038A8DED048A8DED050A36F02CFFC5
:10C2500007B0BDEC028B30BDC2B8323EC2B832BEB0
:10C2600010B504466CF088FBD4F8F4321BB1C21A46
:10C27000B2F57A7F12D30A4A1268D26A92F89C20E9
:10C2800002B15BB9C4F8F40294F8314215F0FAFA3D
:10C2900080F80D4306F008FB80F8254010BD00BF74
:10C2A000582600202DE9F0432DED028B91ED007A08
:10C2B000D1ED037A87B08DED047AB0EEC77AB5EE92
:10C2C000C07AF1EE10FADDE91087DDF84C90CDED83
:10C2D000057A0C4615461E4606DCF0EEE77AF5EECA
:10C2E000C07AF1EE10FA02DD04A818F081FC6B2090
:10C2F000B7EE001AFFEE000A9DED050A15F0CAFF21
:10C300006C2089ED000AB7EE001AFFEE000A9DEDE1
:10C31000040A15F0BFFF04A888ED000A18F0C4FB5A
:10C32000B7EE008A002852D00023C9F8003088ED0B
:10C33000008AD4ED067A67EEA77AF4EEC87AF1EEB9
:10C3400010FA4ADB0023336085ED008ADFED3F0AF7
:10C3500096ED000A7C20B7EE001A15F09BFF86EDE3
:10C36000000A95ED000A7D20B7EE001AFFEE000AE4
:10C3700015F090FF85ED000AD4ED067A129BDFEDF3
:10C38000346AF1EE677AC3ED007A96ED007AF0EE4A
:10C39000C77AF4EEE67AF1EE10FA2BD503AB02AAD7
:10C3A00001A9204616F0DAFF9DED018AB0EE480A99
:10C3B0008FF04CFD85ED000AB0EE480A8FF09CFE30
:10C3C00087ED000A07B0BDEC028BBDE8F08304A83E
:10C3D00018F056FB0028A7D1ABE738EE670A15F036
:10C3E00089FE86ED000A94ED087AC7EE007AC5ED65
:10C3F000007AABE794ED076AC6EE077AC7ED007ADC
:10C4000096ED007AB0EEC77AB4EEE67AF1EE10FA65
:10C41000C4D495ED007ADFED0F6AB0EEC76AB4EED2
:10C42000666AF1EE10FAB9DCB4EE477AF1EE10FA72
:10C43000B4D6B0EEE77AB4EE667AF1EE10FAADDC7F
:10C44000F4EE677AF1EE10FABCD7A7E7000000001F
:10C4500000000034FFFF7F7F1FB500F517730393C3
:10C4600000F51673029300F51573019300F514732C
:10C47000009300F5127200F5137300F54871FFF791
:10C4800011FF05B05DF804FB9FED156A90ED817A10
:10C49000DFED146AD0ED837A27EE067A67EE867AAE
:10C4A00027EE267A67EEA67ABDEEC77AFDEEE77A2A
:10C4B00080ED7E7A90ED827A27EE067A17EE903A3A
:10C4C00027EE267A002BB8BF03F50C43BDEEC77AE2
:10C4D000B8BFA03380ED7F7AC0F80032704700BF4C
:10C4E000E02E65420000C842D0ED946AD1ED010A09
:10C4F000D0ED977A91ED007A20EEA70A66EEA00AB9
:10C50000A7EE260A84B0E7EE670A04B07047000081
:10C51000D0ED946AD1ED010AD0ED977A91ED007AD1
:10C5200027EEE00A66EEA00AA7EE260A84B0E7EE40
:10C53000270A04B0704700001FB50E4B1B68044665
:10C54000B3B1684605F0F8F869462046FFF704FCE9
:10C5500020B16A4600212046FEF77AF894F87C3232
:10C56000DB0705D504F51B7201212046FEF770F8A4
:10C5700004B010BD6489002008B502F0D7F9BDE809
:10C58000084001F06FBD000010B580F8F8120446B5
:10C590006CF0F2F9C4F8FC0210BD000010B590F880
:10C5A000F832044653B16CF0E7F9D4F8FC32C01A03
:10C5B000B0F57A7F84BF002384F8F83294F8003312
:10C5C00053B16CF0D9F9D4F80433C01AB0F57A7FBE
:10C5D00084BF002384F8003310BD000000F5AA706A
:10C5E0000B4607C883E80700012070470023C0F806
:10C5F0009C30C0F89830C0F89430C0F8A830C0F82B
:10C60000A430C0F8A030C0F8AC30704770470000CC
:10C61000024B0B604FF07C531360704700004842A0
:10C620007047000008B50B4600F12801184617F0C6
:10C63000FFFC012008BD000010B500F5B4700C46E9
:10C640000FC884E80F00204605F066F830B1FFF708
:10C650007DFD00F51B700FC884E80F00204605F033
:10C660005BF880F00100C0B210BD000010B50446B8
:10C6700005F09AFB204610BD10B5D0F86031044695
:10C680005BB16CF079F9D4F86031C01A41F28833AB
:10C69000984294BF0020012010BD0120FCE700005B
:10C6A00013B5009303680192D3F890309847DDE901
:10C6B0000021044628B90448044B0068C06A12F0FF
:10C6C000B7FB204602B010BD58260020A8870B08F3
:10C6D00013B504460191FDF745FD2368019A1B6DD2
:10C6E000014608B190F84E11204602B0BDE8104056
:10C6F0001847000030B585B00023019302930393DF
:10C7000003680D46DB6D01A99847044620B1039BE1
:10C710002B60204605B030BD02F008F9417C01F0E5
:10C72000DDFD04460028F4D002F000F901F03CFDE4
:10C73000B1EE400A85ED000AEBE7000090ED007ACB
:10C74000DFED0F7AB0EEC77AB4EEE77AF1EE10FAC9
:10C7500014D590ED017AB0EEC77AB4EEE77AF1EE37
:10C7600010FA0BD590ED027AB0EEC77AB4EEE77A04
:10C77000F1EE10FA4CBF01200020704700207047F6
:10C780000000003410B5FDF7EDFC044658B190F8F8
:10C790004E11FDF78FFA30B194F84E112046BDE8E6
:10C7A0001040FDF783BB002010BD000038B50D46DA
:10C7B0000EF03AFC0446FEF73BF8022881BF94F8DD
:10C7C000C402B02303FB0040D43089BF07C8002057
:10C7D00085E80700012038BD2DE9F0432DED028BDF
:10C7E0008FB003680025DB6C0395049505950695CD
:10C7F000029502A904469847064638B1FFF7BCFEE9
:10C80000DDED027A27EE800A8DED020A0EF00CFCB7
:10C81000FEF70EF80746002E50D0DDED027AD4ED7B
:10C82000646A94ED657A23680B9527EE877A67EE44
:10C83000A67A8DED097ACDED0A7A0C950D959B6C53
:10C840000BA9204609AD98470BA9284618F086F891
:10C85000012F8DED030ACDED040A40F2B3800EF0F6
:10C86000E3FB90F8C432DFED5B7AB02505FB0300F3
:10C8700090ED308A28EE278AB0EE480A8FF0E6FA6B
:10C88000F0EE408AB0EE480A8FF036FCCDED0B8A10
:10C890008DED0C0A0EF0C8FB90F8C43205FB0300C6
:10C8A00090ED2F0A0BA818F079F809AD8DED050A67
:10C8B000CDED060A05A896BB03C885E00128CED8B1
:10C8C0009DED020AB5EEC00AF1EE10FA7FDD07AE6B
:10C8D000D4F89421D4F8903107923046089318F098
:10C8E00087F823680B950C950D959B6C0BA920463A
:10C8F0009847DDED077A9DED0B7A77EE877A9DED0F
:10C900000C7ACDED077ADDED087A77EE877A09AB00
:10C91000CDED087A96E8030083E8030049E0236937
:10C9200093ED000AB7EE008A38EE408A18F036F828
:10C9300004F5BC798DED090A4846B0EE480ACDED04
:10C940000A0A18F02BF80BA92846CDED0C0A8DED3C
:10C950000B0A18F003F804F5C47603AFC4ED5F0AC0
:10C96000314684ED5E0A384618F008F804F5C078C0
:10C970008DED090A4046B0EE480ACDED0A0A18F0DE
:10C980000DF80BA928468DED0B0ACDED0C0A17F01A
:10C99000E5FF97E8030084ED600AC4ED610A86E8CC
:10C9A00003004946404617F0D9FF8DED090ACDED49
:10C9B0000A0A9DED090ADDED0A0A0FB0BDEC028BF3
:10C9C000BDE8F083DDE9030185E80300F1E709959F
:10C9D0000A95EEE735FA8E3C10B590F842130446FE
:10C9E00005F07CFB7C23C0B203FB0044D4F8A0001C
:10C9F00010BD0000044B026F1B68DB6A5A60426F77
:10CA00009A60826FDA60704758260020F0B58FB0C8
:10CA1000044614F037FF002302930393049390F825
:10CA2000121301AB02AA054613F046FF04F1940766
:10CA3000D8B39DED010AB5EEC00AF1EE10FA34DD6F
:10CA400002A818F057FB04F1B00684ED2C0AC4EDDF
:10CA50002D0A84ED2E1A3946304618F05BFB04F19E
:10CA60007C01304618F00AFB04F1880105A88DED21
:10CA7000050ACDED060A8DED071A18F0FFFA08A891
:10CA80008DED080A9DED010ACDED090A8DED0A1A1A
:10CA900018F020FB0BA904F128008DED0B0ACDED59
:10CAA0000C0A8DED0D1A16F005FD95F812030C23F6
:10CAB00003FB0050394600F5117018F0DFFA84EDE1
:10CAC0002C0AC4ED2D0A84ED2E1A0FB0F0BD000023
:10CAD0002DE9F047824B00251F682DED028BC0F831
:10CAE0009C50C0F89850C0F89450C0F88450C0F8DA
:10CAF0008050C567C0F89050C0F88C50C0F888507E
:10CB0000C0F8B850C0F8B450C0F8B0500446F86A45
:10CB100003688AB05B680E46984704F1280900282C
:10CB200054D06BF029FF42F20F7398424ED8FB6A43
:10CB30009FED6C8A93ED010A84ED1C0AD3ED020A85
:10CB4000C4ED1D0A93ED031A484684ED1E1A16F033
:10CB5000A5FB47F007FED4ED1E7A67EE887A0546FE
:10CB600017EE900AF3F7C8FCD4ED1D7A67EE887AC9
:10CB7000CDE9040117EE900AF3F7BEFCD4ED1C7A60
:10CB800067EE887ACDE9020117EE900AF3F7B4FC5C
:10CB9000554ACDE900010621284640F037FF94EDC3
:10CBA0001E8AB0EE480A8FF051F984ED650AB0EEA6
:10CBB000480A8FF0A1FA84ED640A6BF0DDFEC4F838
:10CBC00064010AB0BDEC028BBDE8F087A6B194ED1C
:10CBD0001C0AB4EE400AF1EE10FA0DD6D4ED1D0A8F
:10CBE000F4EE600AF1EE10FA06D694ED1E1AB4EED9
:10CBF000411AF1EE10FA52D714F044FE90F81333B4
:10CC00004FF00C0A0AFB030303F5C473074693E8CD
:10CC1000070007AE86E807004FF01508B2EE028A5B
:10CC2000F2EE068A304618F053FEB4EEC80AF1EE72
:10CC300010FA38D508F1FF3818F0FF083CD130461B
:10CC400018F046FEF1EE047AB4EEE70AF1EE10FABF
:10CC500043DD9DED090ADDED087A9DED078A20EEA2
:10CC6000000AA7EEA70A8FF05DFCF0EE400AB0EED6
:10CC7000480A8FF00DFBDDED090A84ED1D0A9DEDDC
:10CC8000080AF1EE600AB1EE400A8FF001FB84ED74
:10CC90001C0A9FED161AD4ED1D0A94ED1C0A484695
:10CCA00016F0FCFA7BE7304618F012FEB4EEE80A04
:10CCB000F1EE10FABEDCC2E7384613F0BFFC38468E
:10CCC00013F084FD97F813330AFB037303F5C47361
:10CCD00093E8070086E80700A4E725676567D8E7BB
:10CCE00058260020E02E654228890B08000000002D
:10CCF0000021FFF7EDBE000037B504460846154693
:10CD0000019118F0E5FDB7EE007AC7EE007AB4F8AD
:10CD1000D03001980133A4F8D03094ED337A37EE57
:10CD2000277A84ED337AB0EE007AF4EEC77AF1EE2A
:10CD300010FA06D5B6EE007AF4EEC77AF1EE10FAE4
:10CD40000DDC9FED0E7AF4EEC77AF1EE10FA13D5F2
:10CD50009FED0B7AF4EEC77AF1EE10FA0CDDB0EE2F
:10CD6000670A18F0B7F9012085ED000AC5ED010A40
:10CD700085ED021A03B030BD0020FBE700247449A2
:10CD8000BD37863570B52DED028B00F1280600F118
:10CD900034058AB029460446304618F017FAB6EE34
:10CDA000008A20EE088A2846B0EE480A18F092F968
:10CDB00007A93046CDED080A8DED091A8DED070A59
:10CDC00018F072F930468DED010AB0EE480ACDED4B
:10CDD000020A8DED031A18F07DF907A928468DED9A
:10CDE000070ACDED080A8DED091A18F05DF904A9BE
:10CDF00001A88DED040ACDED050A8DED061A18F097
:10CE0000F9F9324601A920468DED070ACDED080A51
:10CE10008DED091AFFF770FF58B96BF0ADFD0121D8
:10CE2000C4F860012046FFF753FE0AB0BDEC028B48
:10CE300070BD2A4604A92046FFF75EFF0028ECD00B
:10CE400004F1400207A92046FFF756FF0028E4D06E
:10CE5000EBE7000030B52DED028B0D4683B091F865
:10CE600042130446284605F039F9C1B27C2000FB84
:10CE70000151903104F1280016F0A0F868468DEDBC
:10CE8000000ACDED010A17F035FEDFED1C7AB4EE95
:10CE9000E70AF1EE10FA05D59FED190A03B0BDECD3
:10CEA000028B30BD684617F0A3FE684617F0FCFD04
:10CEB0000028F1D1284694ED428A05F083FAF0EE7D
:10CEC000400AB0EE480A15F0E1F880B9284605F0AE
:10CED00079FA84ED420AB0EE408A8EF0B7FF84ED15
:10CEE000430AB0EE480A8FF007F984ED440A04F5CE
:10CEF0008671684617F0A6FDD0E700BF0000003439
:10CF0000000000009FED0C7AB4EEC70AF1EE10FAB3
:10CF10000BD4DFED0A7AB4EEE70AF1EE10FA07DC83
:10CF2000C0EE077AB0EE670A7047F7EE007AF9E7CD
:10CF3000F2EE047AF6E700BFF3665F3F58A00B41BC
:10CF400008B51C3017F0D6FDF1EE007AB4EEE70A12
:10CF5000F1EE10FA9DBFF1EE027A37EEC00ADFED76
:10CF6000047A9FED040A98BF20EE270A08BD00BF8F
:10CF7000CDCC4C3ECDCCCC3D08B5836993F90000B7
:10CF800038B10EF051F8FDF753FC012894BF002092
:10CF9000012008BDF8B52DED028B054605F084FC97
:10CFA00005F080FB0446B8B3FFF7D0F890F80933DA
:10CFB00093B32846FFF7E0FF064668B30EF034F857
:10CFC00090F8C432B02707FB030090ED2F7AF0EE03
:10CFD000087AB4EEE77AF1EE10FA1DD495ED1E8AC8
:10CFE0000EF022F890F8C432DFED1E7A07FB030042
:10CFF00090ED300A98EE270A15F0CCF8DFED1A7A9A
:10D00000B0EEC00AB4EEE70AF1EE10FA08DC6BF0FD
:10D01000B3FC3446C5F85001BDEC028B2046F8BD88
:10D0200005F5AA7018F054FCB0EE408A0DF0FCFF34
:10D0300090F8C4329FED0D7A07FB0303D3ED2F7AEE
:10D0400067EE877AB4EEE78AF1EE10FADFD56BF07F
:10D0500093FCD5F85041001BB0F5FA6F8CBF00244B
:10D060000124D9E7E02E654200003442CDCC4C3F8C
:10D0700010B50A4B1B68DB6A93F89C3004465BB919
:10D080006BF07AFCD4F86431C01A44F61F639842FE
:10D090008CBF0020012010BD0020FCE75826002096
:10D0A000F8B52DED068B04460DF0BEFF054605F0E4
:10D0B000FBFB064608F0E4F8002840F0AA80204672
:10D0C000FFF768FF002800F0A7803046FFF784FCD8
:10D0D000D4F8DC30984200F018813046FFF77CFC31
:10D0E000D4F8DC30DFED8E7AC31A08EE903AF8EE11
:10D0F000688A304668EEA78AFFF76EFC94F8BC3069
:10D10000C4F8DC00F3B9304605F0DEFAD0B104F122
:10D11000280796F842233946304605F057F9D4EDF2
:10D120001D0AB0EE401A384694ED1C0A16F0B6F807
:10D130000023C4F89030C4F88C30C4F88830012340
:10D1400084F8BC3020463146FFF784FE95F8C402CF
:10D1500005EB0015B0EE408A2B6FC4F8E03004F107
:10D16000B000D4ED129A18F0B3FB6368DFED6D7A6E
:10D1700093ED007AB4EEE77AF1EE10FA68EE299AB0
:10D18000B0EE40AA01D5C3ED007A2046B0EE4A0ABF
:10D19000FFF7B8FE636820EE299A93ED000A29EEA6
:10D1A000009AFFF7CDFE29EE009A204684ED249ADE
:10D1B000FFF75EFF38B1D4ED247AB2EE007A67EE65
:10D1C000877AC4ED247AF0EE007AF4EEE78AF1EE85
:10D1D00010FA10D5DFED547AB4EEE7AAF1EE10FAAA
:10D1E00009D5DFED527A69EEA79AD4ED2A7AE9EEF5
:10D1F000A87AC4ED2A7A9FED4E0A94ED367ADFEDD7
:10D200004D7AB0EEC88A28EE008AA7EE278A84ED10
:10D21000368ABDEC068BF8BDFEF798FF90F809330F
:10D22000002B72D02046FFF7A7FE00286DD095F89E
:10D23000C42205EB0213196FD4F8E0308B4264D09E
:10D24000B02606FB025292ED2F7AF0EE087AB4EE89
:10D25000E77AF1EE10FA58DBCB1AC4F8E01008EECA
:10D26000903A95F8C4329FED341A94ED1E0ADFED22
:10D27000337A06FB0353D3ED309A69EE819AF8EEC8
:10D28000688A39EEC00A68EEA78A14F0EFFFB0EEA4
:10D29000409A8EF031FF94F8BC30B0EE408AF3B182
:10D2A000F3EE047AF4EEE78AF1EE10FA17DC95F863
:10D2B000C40206FB005595ED2F7AF2EE027AB4EE29
:10D2C000E77AF1EE10FAFFF64AAFDFED1D7AB0EE25
:10D2D000C99AB4EEE79AF1EE10FAFFF640AF9FED6F
:10D2E000198AD4ED1D0A94ED1C0AB0EE691A04F1F6
:10D2F000280015F0D3FF012384ED248A84ED238ACE
:10D3000084ED228A84F8BC3029E7BDEC068B04F159
:10D3100088009FED0D0ABDE8F84017F02FBF00BF51
:10D32000BD378635CDCC4C3DC2B8B23E0AD7233C82
:10D33000CDCC4C3ECDCC4C3F35FA8E3C6F12833A6F
:10D340001904863F00000000EC51783F30B50C23F3
:10D3500003FB010101F1C003144693E807008BB001
:10D3600004AD85E8070094E8070083E80700284635
:10D37000FFF7E4F907AB58B194E8070083E807002A
:10D380009DED070ADDED080A9DED091A0BB030BDD1
:10D3900095E80700F2E70000F0B52DED028BD0F81C
:10D3A00018318B60D0F81C31CB6085B004460D4637
:10D3B00001F0BCFA06460DF037FEA36993F9003080
:10D3C000022B07464BD1FDF733FA022847D997F8CD
:10D3D000C432B02202FB0373D3F8B01000222846F7
:10D3E00004F0B0F9D4ED4A0A94ED490A284604F055
:10D3F000A3FC94F82C3163B36BF0BEFA9FED228A44
:10D4000097F8C4128DED018A01AA064638460CF041
:10D410008FFED4F820019FED1D0A361A07EE906AA0
:10D42000F8EE677A4FF4876027EE800AB6EE001AAE
:10D43000F0EE480A14F02EFFDDED017A30EE270AF7
:10D4400004F1F0008DED010A17F0A8FA284604F067
:10D4500073FC94F82C0105B0BDEC028BF0BD707C20
:10D46000242303FB006696ED0B8AFEF76FFED0EDDA
:10D470009C7A9FED077AF8EEE77AE8EE077AFDEE00
:10D48000E77A17EE901AA9E7000000006F12833ABE
:10D490000000C842F8B5036F0B60436F4B60836FA9
:10D4A0008B6000F14C050E46074601F10C040FCDD0
:10D4B0000FC40FCD0FC42B68236007F1B00207CA59
:10D4C00006F1300383E8070007F1940207CA06F16A
:10D4D0003C0383E8070007F11C0207CA06F1480372
:10D4E00083E8070006F160013846FFF755FF86F82C
:10D4F0007000F8BD30B589B0044668460D4604F0AA
:10D500001BF969462046FFF797F818B90024204612
:10D5100009B030BD04A804F00FF9204604A9FFF7B4
:10D520003BFF04460028F1D004A9684604F05CFBE8
:10D5300085ED000AC5ED010A85ED021AE7E7000056
:10D540001FB500230C4601A9019302930393FFF733
:10D55000D1FF08B1039B236004B010BD30B585B086
:10D5600001AD00230C462946019302930393FFF774
:10D57000C1FF034618B195E8030084E8030018468C
:10D5800005B030BDF8B506460F461546FCF7EAFD76
:10D59000044690B13946FCF78DFB70B12046394600
:10D5A000FCF784FC044640B1FCF7DCFD3946FCF78F
:10D5B000BFFC85ED000A2046F8BDFEF7C7FD90F8D8
:10D5C000083343B13046FFF7D7FC044618B1D6F80C
:10D5D0004C312B60EFE7D6F84C312B600024EAE7A2
:10D5E00070B52DED048B1646FFF7CCFF054670B3E2
:10D5F000FEF7ACFD90F930424CB30DF015FDFDF790
:10D6000017F9012823D9E4B207EE904AB8EE678AE9
:10D610000DF00AFD90F8C43296ED009AB02202FB9C
:10D620000300D0ED2F8AFEF7A7FF38EE281A78EE18
:10D63000C80A40F2614029EE000A14F02BFEB0EE59
:10D64000408AFEF799FFC8EE007AC6ED007ABDEC7D
:10D65000048B284670BD000008B505F025F9BDE82B
:10D66000084005F01FB8000010B5044617F0DEFDB5
:10D6700050B904F10C0017F0D9FD28B904F11800D5
:10D68000BDE8104017F0D2BD012010BD38B500F143
:10D69000280504462846FFF7E7FF28B12046012168
:10D6A000BDE83840FFF714BAD4ED107AB7EE007A2F
:10D6B000F4EEC77AF1EE10FA06D5BFEE007AF4EE7A
:10D6C000C77AF1EE10FA12DC2046FFF75BFB284622
:10D6D000FFF7CAFF0028E1D1D4ED107AB2EE047A48
:10D6E000F0EEE77AF4EEC77AF1EE10FAD6DC38BD48
:10D6F00010B5044618F0ECF82046BDE8104017F0CD
:10D7000051BD00002DE9F04F2DED048B9FEDC48A33
:10D7100095B00446F0EE408A8DED028A8DED038AC5
:10D720008DED048AFFF7BCFC14F0ACF8002305462D
:10D7300095F87921012AA8BF012293423FD2002106
:10D74000284612F0E7FE01230028F1D008AB0BAA0F
:10D75000002128468DED0B8A8DED0C8A8DED0D8A0A
:10D7600013F004F99DED080AB5EEC00AF1EE10FAC7
:10D7700023DD0BA817F0BEFC11A904F128008DEDE4
:10D78000110ACDED120A8DED131A15F0BBFB0EA890
:10D790008DED0E0AB0EE680ACDED0F0A8DED101A70
:10D7A00017F098FC11A904F1E4008DED110ACDEDFC
:10D7B000120A8DED131A17F0ADFC0123B8E795F8A6
:10D7C00013130C2303FB015104F1280B01F5C47161
:10D7D000584615F097FB84ED070A94ED3F0AC4ED17
:10D7E000080A70EE288A84ED091AC4ED3F8A0DF00C
:10D7F0001BFC0646FEF7AAFC90F80933009320466E
:10D80000FFF7BAFB80B13046FDF712F802280BD9BA
:10D8100096F8C4226169B02303FB026391F90010FA
:10D8200093F8D20088425FDA94ED3F7ADFED7D7A9B
:10D83000B4EEE77AF1EE10FA5DD4D4ED538AFEF738
:10D84000A1FF38B1FCF78EFC90F84E11FCF770FB8D
:10D85000F0EE408A236C626BA16A1393B0EE680A03
:10D8600011A81292119117F035FC04F5AA7102A8C3
:10D870008DED020ACDED030A8DED041A17F04AFC76
:10D880006BF07AF80023074684F814312046FFF73E
:10D8900073FB002865D096F8C422B02302FB033244
:10D8A00032445268C4F8182196F8C42202FB0333AC
:10D8B00033449B68C4F81C316BF05EF80123C4F854
:10D8C000200184ED498A84ED4A8A84F82C31D4F809
:10D8D0000031002B58D102AB93E80700C4F8007167
:10D8E000F03484E8070006E006EB0212176FD4F864
:10D8F0000021BA4204D115B0BDEC048BBDE8F08F15
:10D90000D43393E8070094F814310DF1080C8CE837
:10D9100007001BB904F1F00383E807000123604608
:10D9200084F8143104F5AA7117F0BEFB11A904F1B3
:10D930004C008DED110ACDED120A8DED131A15F084
:10D940000FFBB5EEC00AF1EE10FA8DED110AD8BF4B
:10D950009FED330ACDED120A8DED131A84ED530AB3
:10D9600094E794ED3F7AD4ED497ADDED026AE6EE74
:10D97000877ADDED036AC4ED497AD4ED4A7AE7EEA1
:10D98000267AC4ED4A7AA2E7D4ED3F7A224B8DED98
:10D99000058AF5EEC07AF1EE10FA8DED068A07934E
:10D9A000A9D99FED1E7A94F8143167EE877AB7EE05
:10D9B000007AC7EE279A1BB9009B002B00F0AA80C3
:10D9C000E36804F1F00102A8D3ED008A17F06CFBC4
:10D9D00069EEA88A8DED110A11A8B0EE680ACDEDA6
:10D9E000120A8DED131A17F075FB0EA905A88DED1F
:10D9F0000E0ACDED0F0A8DED101A17F08BFB05A85E
:10DA0000FFF776FE05A817F02BFCD8B16AF0B4FF3B
:10DA1000C4F860016FE700BF000080BF0AE81C4146
:10DA200000000000CDCC4C3ECDCC4C3FCDCC4C3D8D
:10DA3000920A06BF920A063FC2B8B23E728A0E3CF4
:10DA40005B821839012301930023CDE90833CDE926
:10DA50000A33CDE90C335FED0E8A4FF0FF3A04F143
:10DA6000E40895F87921012A1046A8BF01208342D5
:10DA700057D20123002AFAD095F835130029F6D0A1
:10DA8000B0EE690A404617F079FB019B0DF12C09B5
:10DA9000002B41D0424600212046FFF757FC8DED78
:10DAA0000B0ACDED0C0A8DED0D1A4846FEF746FE29
:10DAB00070BB4846FFF71CFE484617F0D1FB38BB49
:10DAC00005A9484617F096FB484605A98DED080ABA
:10DAD000CDED090A8DED0A1A17F078FB08A8B0EE13
:10DAE000409A17F0F5FEBAF1000F06D1F4EEC08AA5
:10DAF000F1EE10FAD8BFB0EE680AB5EEC09AF1EEBA
:10DB000010FAF7EE008A58BFF0EE408A4FF0000A94
:10DB10000123A6E7009B96E798E8070089E807003D
:10DB2000C3E7BAF1000F7FF471AF002384F804312A
:10DB30002046FFF72FFA38B12046FFF71DFA0028DC
:10DB400040F025818DED0A8A95F8123395F87821F9
:10DB50009A4240F233812B4493F83433002B00F087
:10DB60002D8195F8133395F879219A4240F2268158
:10DB70002B4493F83533002B00F0208108A9584638
:10DB800015F0EEF98DED080ACDED090A8DED0A1AB2
:10DB900008A817F04BFB002840F0178108A817F0E1
:10DBA0005FFB002840F011815FED627A94ED357AD9
:10DBB00068EEA78A5FED647AE7EE278A04F1B00089
:10DBC000C4ED358A17F084FEA3685FED687A93EDA3
:10DBD000007AB4EEE77AF1EE10FAF0EE408A00F146
:10DBE000F8802046B0EE680AFFF78CF908A817F015
:10DBF00071FAA3688DED110ACDED120A8DED131A9D
:10DC000093ED000A11A817F065FA204684ED1F0A6B
:10DC1000C4ED200A84ED211AFFF72AFA28B1B2EEEA
:10DC2000000A04F17C0017F0A9FA009BB3B3304658
:10DC3000FCF7FEFD012831D996F8C402B02303FB9E
:10DC4000006696ED2F7AF0EE087AB4EEE77AF1EE00
:10DC500010FA23D595F813030C2303FB005595ED1B
:10DC6000627AF1EE0C7AB4EEE77AF1EE10FA15DB97
:10DC7000D4ED1D7A1FED927AF4EEC77AF1EE10FA28
:10DC80000CDD1FED947AF4EEC77AF1EE10FA05D5AB
:10DC9000B6EE000A04F17C0017F070FA5FED9A7A94
:10DCA000F4EEE78AF1EE10FA22D51FED9C0A08A8DF
:10DCB00017F010FA0EA88DED0E0A94ED3F0ACDED87
:10DCC0000F0A8DED101A17F005FA11A904F1A00042
:10DCD0008DED110ACDED120A8DED131A17F01AFA17
:10DCE000D4ED2B7A94ED3F7A77EE877AC4ED2B7AD8
:10DCF00094ED2B7AF1EE047AB4EEE77AF1EE10FAB5
:10DD00003BDB13F0BFFD5FEDB27A94ED2B1A94ED7F
:10DD1000280A21EE271A40F2C530F1EE410A8DEDB6
:10DD2000011ACDED000A14F0B5FA9DED011ADDEDF2
:10DD3000000A84ED280A40F2C63094ED290A14F056
:10DD4000A9FA9DED011ADDED000A84ED290A40F2E1
:10DD5000C73094ED2A0A14F09DFA04F1A00184ED75
:10DD60002A0A04F1940017F0D5F984ED2A8A84ED8B
:10DD7000298A84ED288A84ED2B8A0023C4F8E430B4
:10DD8000C4F8E830C4F8EC3084ED3F8AA3E5E368DA
:10DD9000F7EE000A93ED000A14F078F900283FF43A
:10DDA000D1AE94ED1C0AB0EEC00A8EF0A5F9DDEDFF
:10DDB0000A7A27EE800A8DED0A0AC5E68DED0A8AF9
:10DDC0008DED098A8DED088AE2E62046FFF75EFCBC
:10DDD0001CE6C3ED007A04E72DE9F04D2DED048B30
:10DDE0009EB0044613F04EFDD0EDC87A90ED618AE6
:10DDF000F4EE487AF1EE10FA48BFB0EE678ADFED34
:10DE00005C7AB4EEE78AF1EE10FA0EDD0023C4F876
:10DE1000E430C4F8E830C4F8EC300023C4F8FC3037
:10DE20001EB0BDEC048BBDE8F08D2046FEF7EEFD84
:10DE30002046FEF7A7FFB0EE480A2046FFF762FC37
:10DE40002046FFF723FCFEF781F914AD00F534728C
:10DE500004F1280114A815F0D3F80FCD04F14C06F5
:10DE60000FC60FCD0FC62B68336004F1740204F1A6
:10DE7000780304F1700104F14C0015F06FFA94ED91
:10DE80001E8AB0EE480A8DF0E1FF84ED650AB0EE1F
:10DE9000480A8EF031F9204684ED640AFEF7AAFDA7
:10DEA000FEF754F904F5B471FDF756FF6AF064FD0E
:10DEB000D4F89831C31A632BB2D9C4F898013DF055
:10DEC000FFFD9FED2C9A05466AF05EFDD4ED1C7AAD
:10DED00067EE897A074617EE900A0E46F2F70CFBBA
:10DEE000D4ED1D7A67EE897A824617EE900A8B464A
:10DEF000F2F702FB94ED1E0A20EE090A41EC180B22
:10DF000014F032F9D4F85C0110EE108AF2F7F4FA4A
:10DF1000CDE91201D4F85801F2F7EEFACDE910017B
:10DF2000D4F85401F2F7E8FACDE90E01D4F8D8009C
:10DF3000F2F7E2FACDE90C01D4F8D400F2F7DCFAFA
:10DF4000CDE90A014046F2F7D7FA0B4B01930B4B90
:10DF50000093CDE908018DED068BCDE904ABCDE949
:10DF60000276074B074A084928463DF035FB57E73C
:10DF7000CDCC4C3EE02E65428D890B0897890B086D
:10DF800054890B085E890B08A4870B0808B52DED92
:10DF9000048BB0EE609AF0EE408A00F011F9B0EE1A
:10DFA000408A89EE280A8EF0DDF9DFED0B7A20EE4B
:10DFB000270A8EF06FF9DFED097A38EE278ADFED58
:10DFC000087A28EE278AF7EE007A37EEC00A28EEA4
:10DFD000000ABDEC048B08BD41D3423E3393884315
:10DFE000A1D81943FFF7D2BF08B52DED048B9FEDE3
:10DFF000189AF0EEE07AF4EEC97AF1EE10FAF0EE4B
:10E00000408AB0EE608A1ED400F0DAF8DFED117AB3
:10E010009FED117A70EE277A9FED100AE8EEC77A2D
:10E020009FED0F7A27EE800AC8EE007A87EE270A66
:10E03000B4EEC90AF1EE10FA05DBBDEC048BBDE8C5
:10E0400008408EF06FBABDEC048BB7EE000A08BD35
:10E050000000003433938843F4FDD43B48A18F4340
:10E06000CDCC9C3F427CD0ED257A242101FB0202DD
:10E0700092ED0B0AD2ED090A30EE270AFFF7B4BF82
:10E0800038B52DED088BDFED21AA9FED21AA9FED7C
:10E0900021BA0546B0EE409AF0EE609AB0EE408AA2
:10E0A0001524013CA4B25CB3F0EE490A2846B0EE58
:10E0B000480AFFF76BFFF0EE490A70EE698A2846BE
:10E0C00038EE2A0AFFF762FFB0EEE87A70EE697A5E
:10E0D000B4EECA7AF1EE10FA77EEE87A10D468EE70
:10E0E000AA8A40F2631088EEA70AB0EE4B1A38EE07
:10E0F000400AF0EE4A0A14F0CDF8B0EE408AD0E7BC
:10E10000B0EE480ABDEC088B38BD00BFCDCCCC3D8D
:10E110000AD7233C00247449002343608360C36012
:10E12000036143618361C361002380F8203070473D
:10E1300090F82020531CDBB2062B80F8203000EB37
:10E14000820288BF002382ED010A88BF80F8203058
:10E15000704700004FF0FF3310B543610E4BC0F81D
:10E16000A8300023044680F8C830A830FFF7D4FF59
:10E170000A4BC4F8A83004F5867069F0B3FD084B6B
:10E1800008491C60204634F067F8D4F89030C4F891
:10E190009430204610BD00BFC08B0B08D08B0B08FD
:10E1A000AC860020608C0B0808B5A8303EF0CEFC91
:10E1B000DFED027A20EE270A08BD00BF00007A4496
:10E1C00090ED3C0ADFED057AB0EEC07AB4EEE77A66
:10E1D000F1EE10FA48BF90ED3D0A704700000034A0
:10E1E00073B5D0F8A43004460E4663B16AF0C4FBA0
:10E1F000D4F8A430C01A42F20F73984203D894EDB9
:10E20000280A02B070BD114B1D687DB195F84E1102
:10E210002846FBF74BFE48B195F84E1101AA284657
:10E22000FBF7FCFB10B19DED010AEAE7242101FB9D
:10E23000064494ED0A0ADFED067AB4EEE70AF1EE41
:10E2400010FA58BFB0EE670ADBE700BFA4860020D3
:10E2500000000C4208B561B10378022B02D90648D0
:10E260006AF058FB5A1C027000EB830041600120E9
:10E2700008BD0846FCE700BF7C8A0B082DE9F8437F
:10E2800005460E469146002400F13C082B78A34237
:10E2900011DD00234A463146012010F043FA2423C1
:10E2A00063430746002158F8030010F04BFA8742F9
:10E2B00004D00134EAE70020BDE8F8830120FBE741
:10E2C000054B1B682BB141694A1C02D018463DF032
:10E2D000C1BB0020704700BF6489002002290BD811
:10E2E000242303FB010191F8390030B191F83A0081
:10E2F00018B191F83B007047002070472DE9F047B6
:10E3000004466AF039FBD4F8F86042F21073861BB9
:10E310009E4288BFC4F8F80000274FF0240942F25B
:10E32000107A237CFDB2AB421CD929462046FFF768
:10E33000D5FF70B109FB054898ED0D0AD8ED097AB3
:10E34000D4ED250A30EE270A2046FFF799FE88ED26
:10E350000C0A564504D909FB0540303034F054F915
:10E360000137DEE7617C2046FFF73AFF84ED3D0A86
:10E37000BDE8F08770B5044686B06AF0FDFAD4F8BF
:10E380009830C31AB3F57A7F05464FD3344B94EDDA
:10E39000257A1B68DFED336ADB6AD4ED247A93F8C3
:10E3A0009C60B0EEC76AB4EEE66AF1EE10FA32D5C0
:10E3B000B0EEE76AB4EEE66AF1EE10FA2BD502A8E9
:10E3C00003F0BAF996BBFDF7C1FE02A9FDF7C4FC44
:10E3D00060B3DDED037A9FED247AF8EEE77A67EE1D
:10E3E000877AC4ED257AC4F89850FDF7AFFEFDF7A3
:10E3F0007BFA2046FFF782FF46F0B4F90546D4F8D1
:10E400009400F2F779F8194ACDE90001062128466F
:10E410003FF0FCFA0AE037EE676AF7EE005AB0EE1A
:10E42000C66AB4EEE56AF1EE10FA01DC06B070BD22
:10E43000B0EEE76AB4EEE66AF1EE10FAF6D4002E1A
:10E44000CFD02046903080ED007A34F0DDF846F0F1
:10E4500089F9074A012106B0BDE870403FF0D6BAFD
:10E4600058260020000000340AD7233CBD8A0B0840
:10E47000988A0B08F0B52DED048B85B004464FF457
:10E48000537200F5867103A810F0F2FAD4ED227AE7
:10E49000D4ED236A9FED796A637C37EEE67A242215
